:100000000C94BF140C94F0140C94F0140C94F01491
:100010000C94F0140C94F0140C94F0140C94F01450
:100020000C94F0140C94F0140C94F0140C94F01440
:100030000C94F0140C94A6900C94F0140C94F014FE
:100040000C94F0140C940CB60C94F0140C94F01462
:100050000C94F0140C94F0140C94E8980C940EC5C5
:100060000C94F0140C94D1550C94F0140C94F014DE
:100070000C94F0140C94F0140C94F0140C94F014F0
:100080000C94F0140C94F0140C94F0140C94F014E0
:100090000C94F0140C94F0140C94F0140C94F014D0
:1000A0000C94F0140C94F0140C94F0140C94F014C0
:1000B0000C94F0140C94F0140C94F0140C94F014B0
:1000C0000C94F0140C94F0140C94F0140C94F014A0
:1000D0000C94F0140C94F0140C9470560C9431564B
:1000E0000C94F014F9321633473364337933A23366
:1000F0000F3475341E35663974396D399439983931
:10010000B239183EC739133A453A6C3A953AEB3A48
:10011000FC3A0D3B1E3B2F3B403B183E233D183E17
:100120002E3D9E3DA43DC43D27C12AC119C11DC11C
:1001300023C161C12EC132C138C13CC140C146C1D9
:100140004AC14EC161C154C158C15CC12AC42FC447
:1001500034C43EC448C4C1C452C45AC462C46CC48A
:1001600076C480C48FC499C4C1C4A3C4ADC4B7C489
:10017000084AD73B3BCE016E84BCBFFDC12F3D6C0E
:1001800074319ABD56833DDA3D00C77F11BED9E474
:10019000BB4C3E916BAAAABE000000803F05A84C54
:1001A000CDB2D44EB93836A9020C50B99186880820
:1001B0003CA6AAAA2ABE000000803F004E414E493C
:1001C0004E495459494E46CDCCCC3D0AD7233C1715
:1001D000B7D13877CC2B329595E6241FB14F0A0062
:1001E0000020410000C84200401C4620BCBE4CCA52
:1001F0001B0E5AAEC59D74434F4D4D554E4943415C
:1002000054494F4E0044525952554E004552524F98
:10021000525300494E464F004543484F0047322F46
:1002200047332062616420706172616D657465722C
:10023000730A00206F6620004D424C20473239205F
:10024000706F696E74200059206F7574206F66207E
:1002500072616E67652028312D35292E0A005820DD
:100260006F7574206F662072616E67652028312D6E
:1002700035292E0A004D6573682070726F62696EB1
:100280006720646F6E652E0A005374617274206D6E
:100290006573682070726F62696E67207769746831
:1002A0002022473239205331222066697273742E1E
:1002B0000A004732380A47323920533200537461FA
:1002C00074653A20004D65736820626564206C6532
:1002D00076656C696E6720686173206E6F2064615B
:1002E00074612E0A0053206F7574206F662072614E
:1002F0006E67652028302D35292E0A004D657368FC
:1003000020706F696E742063616E6E6F7420626519
:10031000207265736F6C7665640A00456E642066B2
:10032000696C65206C6973740A00426567696E20A8
:1003300066696C65206C6973740A00286E6F2066AC
:10034000696C6529005344207072696E74696E6728
:10035000206279746520004E6F74205344207072BF
:10036000696E74696E670A0043757272656E7420F7
:1003700066696C653A20002569730025696D202542
:100380006973002569682025696D2025697300253A
:100390006964202569682025696D20256973002519
:1003A000697920256964202569682025696D2025E3
:1003B0006973005072696E742074696D653A20002B
:1003C000180213020C020502F7016F66660044452D
:1003D0004255473A004B494C4C45442E20004D3184
:1003E00031332053006F6B002C20002C2000544828
:1003F00045524D414C5F50524F54454354494F4E26
:10040000004155544F5245504F52545F53445F532F
:10041000544154555300454D455247454E43595F4D
:1004200050415253455200434153455F4C49474860
:10043000545F4252494748544E45535300544F4726
:10044000474C455F4C494748545300534F46545717
:100450004152455F504F574552004255494C445F09
:1004600050455243454E54004C4556454C494E4725
:100470005F44415441005A5F50524F42450041553C
:10048000544F4C4556454C005052494E545F4A4FCC
:10049000420050524F4752455353004155544F521A
:1004A00045504F52545F54454D5000564F4C554D9A
:1004B000455452494300454550524F4D0053455213
:1004C00049414C5F584F4E5F584F4646004649528F
:1004D0004D574152455F4E414D453A4D61726C69F1
:1004E0006E20312E312E39202847697468756229B3
:1004F00020534F555243455F434F44455F55524C3F
:100500003A68747470733A2F2F6769746875622E35
:10051000636F6D2F4D61726C696E4669726D7761A4
:1005200072652F4D61726C696E2050524F544F436B
:100530004F4C5F56455253494F4E3A312E30204D65
:10054000414348494E455F545950453A3344205041
:1005500072696E7465722045585452554445525F15
:10056000434F554E543A3120555549443A636564DA
:1005700065326132662D343161322D343734382D95
:10058000396231322D63353563363266333637663C
:10059000660A002F2F200020540020520041636380
:1005A000656C65726174696F6E3A20500020466C0C
:1005B0006F773A20000001363726032BFFFFFF3C00
:1005C0003D382AFFFFFFFF2E303E12FFFFFFFFFFE7
:1005D000FFFF0809FF2C071A1C18FFFFFF08440A39
:1005E0002C4324221E20643A0020693A0020703AED
:1005F00000496E76616C6964206578747275646513
:10060000720A0043290A0061626C656420286D69E2
:100610006E2074656D702000436F6C642065787483
:10062000727564657320617265200020643A002051
:10063000693A0020703A004E6F2063617365206C48
:10064000696768740A00454550524F4D204F4B0A68
:1006500000205A004475616C20456E6473746F709D
:100660002041646A7573746D656E7420286D6D2900
:100670003A20003F4B2076616C7565206F757420C1
:100680006F662072616E67652028302D3130292E0B
:100690000A00416476616E6365204B3D00416374DE
:1006A0006976652045787472756465723A200049F0
:1006B0006E76616C69642065787472756465720A1F
:1006C0000043616E6E6F7420656E74657220737581
:1006D000626469723A20004739310A4731205A2D45
:1006E000302E30320A473930005370656369616CCF
:1006F000204D656E753A205A20446F776E20302E5B
:10070000310A004739310A4731205A2D302E303214
:100710000A473930005370656369616C204D656E1E
:10072000753A205A20446F776E20302E30320A00FE
:100730004739310A4731205A2B302E30320A473997
:1007400030005370656369616C204D656E753A20A9
:100750005A20557020302E30320A004739310A476E
:1007600031205A2B302E310A4739300053706563DF
:1007700069616C204D656E753A205A2055702030A5
:100780002E310A00473239205332005370656369B5
:10079000616C204D656E753A204E657874204D650C
:1007A000736820506F696E740A00473239205331E4
:1007B000005370656369616C204D656E753A205316
:1007C00074617274204D657368204C6576656C6940
:1007D0006E670A004D313430205336300053706557
:1007E0006369616C204D656E753A2050726568656D
:1007F0006174204265640A004D35303100537065E4
:100800006369616C204D656E753A205265616420A4
:10081000454550524F4D0A004D35303000537065FC
:100820006369616C204D656E753A20536176652071
:10083000454550524F4D0A004D33303320452D3140
:100840002053383020433820553100537065636998
:10085000616C204D656E753A204175746F2054753A
:100860006E6520486F74626564205069640A004DAB
:100870003330332045302053323330204338205535
:1008800031005370656369616C204D656E753A2067
:100890004175746F2054756E6520486F74656E6481
:1008A000205049440A003C5370656369616C5F4D98
:1008B000656E753E003C5370656369616C5F4D65A4
:1008C0006E753E002F002F002F002F2E2E0A002FB6
:1008D0002E2E002F2E2E003C5370656369616C5FD5
:1008E0004D656E753E0A003C5370656369616C200E
:1008F0004D656E753E003C5370656369616C204DBB
:10090000656E753E003C5265616420454550524F0E
:100910004D3E003C5265616420454550524F4D3E6E
:10092000003C4175746F2054756E6520486F746289
:100930006564205049443E003C4175746F205475F5
:100940006E6520486F74626564205049443E003CE7
:100950004175746F2054756E6520486F74656E64C0
:10096000205049443E003C4175746F2054756E65BB
:1009700020486F74656E64205049443E003C4578C1
:1009800069743E003C457869743E003C536176656D
:1009900020454550524F4D3E003C53617665204501
:1009A0004550524F4D3E003C4E657874204D657366
:1009B0006820506F696E743E003C4E657874204D1F
:1009C00065736820506F696E743E003C53746172A9
:1009D00074204D657368204C6576656C696E673E62
:1009E000003C5374617274204D657368204C6576C9
:1009F000656C696E673E003C507265686561742085
:100A00006265643E003C5072656865617420626591
:100A1000643E003C5A20446F776E20302E313E00F9
:100A20003C5A20446F776E20302E313E003C5A20D5
:100A3000446F776E20302E30323E003C5A20446F97
:100A4000776E20302E30323E003C5A2055702030D8
:100A50002E30323E003C5A20557020302E30323E2F
:100A6000003C5A20557020302E313E003C5A205513
:100A70007020302E313E0056313136004A3333205B
:100A8000004D3530300A4D3432302053310A473171
:100A9000205A313020463234300A47312058302035
:100AA0005930204636303030004A3232004A323235
:100AB000004731205A3520463234300A4731205819
:100AC000313930205932302046363030300A473103
:100AD000205A302046323430004731205A352046E3
:100AE0003234300A473120583139302059313930C9
:100AF0002046363030300A4731205A3020463234D2
:100B000030004731205A3520463234300A473120F0
:100B100058313930205932302046363030300A478B
:100B200031205A302046323430004739310A4731BB
:100B3000205A313020463234300A4739300A4732A1
:100B4000380A4732390A473120583230205932307A
:100B50002046363030300A4731205A302046323471
:100B600030004A3032004A3132004731205A3130A9
:100B7000004F4B004731205A313000473930004791
:100B800031204525694635303000473120452D302C
:100B90002E314625690047312045302E31462569E2
:100BA000004731205A2569462569004731205A2DD2
:100BB000302E31462569004731205A302E314625E6
:100BC0006900473120592569462569004731205978
:100BD0002D302E314625690047312059302E3146BF
:100BE000256900473120582569462569004731208D
:100BF000582D302E314625690047312058302E318E
:100C000046256900473931004732380047323820DD
:100C10005A004732382059004732382058004132B4
:100C2000305620004731205A3130004A3034004AD3
:100C30003231004A3230004B494C4C45442E2000A2
:100C40004A303400454E4400464E20004A303200BF
:100C50003939393A393939004D0048004137562081
:100C600000413656202D2D2D004A30320041365697
:100C700020005A3A2000593A2000583A20004135C5
:100C80005600413456200041335620004132562050
:100C900000413156200041305620004D3834004A82
:100CA0003136004A3138004739310A4731205A314C
:100CB0003020463234300A473930004A3134004A55
:100CC0003030004A3031004A31300024F4D4305002
:100CD000C38E20C2A24017828B7011127A910D81AF
:100CE0006CD90AA861E108C7586607615143061E1E
:100CF0004B5D05C145A7041A411104093D980371D4
:100D00003931034036DB0265339102D4305402801E
:100D10002E1D02632CEE01752AC501B028A001101A
:100D20002781018F2564012B244B01E0223401AC83
:100D3000211F018D200D01801FFC00841EED0097F6
:100D40001DDF00B81CD200E61BC600201BBC0064DF
:100D50001AB200B219A8000A19A0006A189900D1A5
:100D600017910040178B00B516840031167E00B332
:100D70001579003A157300C7146F0058146A00EE15
:100D80001366008813630025135E00C7125B006CB6
:100D900012570015125400C111510070114F00215B
:100DA000114B00D61049008D104700461044000238
:100DB000104200C00F4000800F3E00420F3C000672
:100DC0000F3B00CB0E3800930E37005C0E3500272A
:100DD0000E3400F30D3200C10D3100900D30006073
:100DE0000D2E00320D2D00050D2C00D90C2B00AE60
:100DF0000C2900850C29005C0C2700350C27000EFF
:100E00000C2600E80B2400C40B2400A00B23007D5B
:100E10000B23005A0B2100390B2100180B2000F87E
:100E20000A1F00D90A1E00BB0A1E009D0A1D008071
:100E30000A1D00630A1C00470A1B002C0A1B001134
:100E40000A1A00F7091A00DD091900C4091900ABD4
:100E5000091900920917007B091800630917004C53
:100E600009160036091600200916000A091500F5B2
:100E7000081500E0081400CC081400B8081400A4F9
:100E8000081400900813007D0812006B0813005826
:100E9000081200460812003408110023081100123D
:100EA00008110001081100F0071000E0071000D041
:100EB000071000C0071000B0070F00A10710009135
:100EC000070E0083070F0074070F0065070E005719
:100ED000070E0049070E003B070D002E070E0020ED
:100EE000070D0013070D0006070D00F9060C00EDB5
:100EF000060D00E0060C00D4060C00C8060C00BC71
:100F0000060C00B0060C00A4060B0099060C008D20
:100F1000060B0082060B0077060B006C060B0061C7
:100F2000060A0057060B004C060A0042060A003863
:100F3000060A002E060A0024060A001A060A0010F5
:100F400006090007060A00FD050900F4050900EB83
:100F5000050900E2050900D9050900D0050900C707
:100F6000050900BE050900B5050800AD050800A586
:100F70000509009C050800940508008C05080084FC
:100F80000508007C050800740508006C050700656D
:100F90000508005D050700560508004E05070047D7
:100FA0000507004005080038050700310507002A3D
:100FB000050700230507001C050600160507000F9E
:100FC0000507000805060002050700FB040600F5FA
:100FD000040700EE040600E8040600E2040700DB54
:100FE000040600D5040600CF040600C9040600C3A9
:100FF000040600BD040600B7040600B1040500ACF9
:10100000040600A6040600A00405009B0406009543
:10101000040500900406008A04050085040500808C
:101020000406007A04050075040500700405006BD1
:1010300004050066040500610405005C0405005712
:10104000040500520405004D040500480405004352
:101050000405003E0404003A040500350405003090
:101060000404002C04050027040400230405001ECA
:101070000404001A04040016040500110404000D01
:10108000040400090405000404040000040400FC36
:10109000030400F8030400F4030400F0030400EC6C
:1010A000030400E8030400E4030400E0030400DC9C
:1010B000030400D8030400D4030400D0030400CCCC
:1010C000030400C8030300C503030024F404D9206B
:1010D0001BC40C5C0E9804C4095F0265077101F41F
:1010E00005F900FB04B30048048700C103690058F8
:1010F00003550003034500BE023A00840231005349
:10110000022A002902250004022000E4011C00C874
:10111000011900AF01170098011400840113007138
:101120000110006101100051010E0043010D003655
:10113000010B002B010B0020010B00150109000C15
:1011400001090003010800FB000800F3000800EBA0
:10115000000700E4000600DE000600D8000600D20A
:10116000000600CC000500C7000500C2000500BD58
:10117000000400B9000400B5000400B1000400AD93
:10118000000400A9000400A5000300A20003009FC2
:101190000004009B000300980003009500020093E8
:1011A000000300900003008D0002008B0003008804
:1011B0000002008600020084000300810002007F1C
:1011C0000002007D0002007B00020079000200772F
:1011D000000100760002007400020072000100713C
:1011E0000002006F0002006D0001006C0002006A46
:1011F000000100690002006700010066000100654F
:101200000001006400020062000100610001006052
:101210000001005F0002005D0001005C0001005B56
:101220000001005A00010059000100580001005758
:101230000001005600010055000100540001005358
:101240000000005300010052000100510001005055
:101250000001004F0001004E0000004E0001004D53
:101260000001004C0001004B0000004B0001004A4F
:10127000000100490001004800000048000100474B
:101280000001004600000046000100450000004546
:10129000000100440001004300000043000100423F
:1012A0000000004200010041000000410001004038
:1012B0000001003F0000003F0001003E0000003E32
:1012C0000001003D0000003D0001003C0000003C2A
:1012D0000000003C0001003B0000003B0001003A20
:1012E0000000003A00010039000000390001003818
:1012F000000000380000003800010037000000370F
:101300000001003600000036000000360001003504
:1013100000000035000000350001003400000034FA
:1013200000000034000100330000003300000033EF
:1013300000010032000000320000003200010031E4
:1013400000000031000000310001003000000030DA
:10135000000000300001002F0000002F0000002FCF
:101360000000002F0001002E0000002E0000002EC3
:101370000001002D0000002D0000002D0000002DB8
:101380000001002C0000002C0000002C0000002CAC
:101390000001002B0000002B0000002B0000002BA0
:1013A0000001002A0000002A0000002A0000002A94
:1013B0000001002900000029000000290000002988
:1013C000000000290001002800000028000000287B
:1013D000000000280000002800010027000000276E
:1013E0000000002700000027000000270001002661
:1013F0000000002600000026000000260000002655
:101400000001002500000025000000250000002547
:101410000000002500000025000100240000002439
:10142000000000240000002400000024000100232C
:101430000000002300000023000000230000002320
:101440000000002300000023000100220000002211
:101450000000002200000022000000220000002204
:1014600000010021000000210000002100000021F7
:1014700000000021000000210000002100010020E8
:1014800000000020000000200000002000000020DC
:101490000000002000000020000000200001001FCC
:1014A0000000001F0000001F0000001F0000001FC0
:1014B0000000001F0000001F0001001E0000001EB1
:1014C0000000001E0000001E000000232C0000B8D9
:1014D000220000561800003A0F0000B8080000B1C2
:1014E000040000710200003E010000656E71756528
:1014F0007565696E672022004B494C4C45442E208F
:10150000005072696E7465722073746F70706564D8
:101510002064756520746F206572726F72732E205F
:1015200046697820746865206572726F7220616EFA
:101530006420757365204D39393920746F207265C8
:1015400073746172742E202854656D7065726174B5
:101550007572652069732072657365742E205365FA
:101560007420697420616674657220726573746199
:101570007274696E67290A004E6F20436865636B59
:1015800073756D2077697468206C696E65206E755F
:101590006D6265722C204C617374204C696E653AE3
:1015A00020004E6F20436865636B73756D2077690B
:1015B0007468206C696E65206E756D6265722C2092
:1015C0004C617374204C696E653A200063686563F2
:1015D0006B73756D206D69736D617463682C204C3D
:1015E000617374204C696E653A20004C696E652009
:1015F0004E756D626572206973206E6F74204C6148
:101600007374204C696E65204E756D6265722B3166
:101610002C204C617374204C696E653A20004D316A
:101620003130004D333100534420726561642065D0
:1016300072726F720A00446F6E65207072696E7408
:10164000696E672066696C650A00526573656E6431
:101650003A20006F6B0020746F6F206C6F6E6720F4
:10166000657874727573696F6E2070726576656ED9
:101670007465640A0020636F6C6420657874727509
:1016800073696F6E2070726576656E7465640A00AA
:10169000627573793A2070617573656420666F7244
:1016A00020696E7075740A00627573793A207061F2
:1016B0007573656420666F7220757365720A0062C7
:1016C0007573793A2070726F63657373696E670A18
:1016D000004A3135004B494C4C45442E20004B49C3
:1016E0004C4C20636175736564206279204B494CD2
:1016F0004C20627574746F6E2F70696E0A004B49CE
:101700004C4C45442E20004B494C4C206361757372
:10171000656420627920746F6F206D75636820693D
:101720006E6163746976652074696D65202D206330
:10173000757272656E7420636F6D6D616E643A20B0
:10174000004A3131005072696E7465722068616CB4
:101750007465642E206B696C6C28292063616C6C45
:101760006564210A000000A0C00000000000000025
:10177000005761726E696E673A20486F6D696E67D7
:101780002042756D702044697669736F72203C2029
:10179000310A000202040000A0400000A040000046
:1017A000004000005C430000574300004E43FFFF31
:1017B000FF20746F6F206C6F6E6720657874727590
:1017C00073696F6E2070726576656E7465640A0069
:1017D00020636F6C6420657874727573696F6E2016
:1017E00070726576656E7465640A003A00436170D4
:1017F0003A005741524E494E4721204C6F77205AAC
:10180000204A65726B206D6179206C65616420747B
:101810006F20756E77616E74656420706175736595
:10182000732E0A00205A00205900580020204D61D4
:10183000783A2000205A00205900580020204D6995
:101840006E3A20004F6E20004F666600536F66743C
:1018500020656E6473746F70733A20004B642000CF
:1018600023646566696E652044454641554C545F66
:10187000004B69200023646566696E652044454617
:1018800041554C545F004B70200023646566696EBF
:10189000652044454641554C545F00504944204121
:1018A00075746F74756E652066696E6973686564BA
:1018B000212050757420746865206C617374204B0E
:1018C000702C204B6920616E64204B6420636F6E26
:1018D0007374616E74732066726F6D2062656C6FD5
:1018E0007720696E746F20436F6E666967757261E9
:1018F00074696F6E2E680A00504944204175746FF8
:1019000074756E65206661696C6564212074696D0B
:10191000656F75740A00453120544845524D414C5D
:101920002052554E415741590042454420544845A4
:10193000524D414C2052554E415741590054686513
:10194000726D616C2052756E61776179004531204E
:1019500048656174696E67206661696C6564004200
:1019600065642068656174696E67206661696C658D
:10197000640048656174696E67206661696C6564BE
:1019800000504944204175746F74756E652066611E
:10199000696C6564212054656D706572617475723F
:1019A0006520746F6F20686967680A00204B643A8D
:1019B0002000204B693A2000204B703A20000A207A
:1019C000436C617373696320504944200A002054BA
:1019D000753A2000204B753A2000206D61783A203E
:1019E00000206D696E3A200020643A200020626970
:1019F00061733A2000504944204175746F74756ECC
:101A000065206661696C65642120426164206578A7
:101A1000747275646572206E756D6265720A00502D
:101A20004944204175746F74756E652073746172DA
:101A3000740A004F66660A0046616465204865695D
:101A40006768742000426564204C6576656C696E39
:101A50006720004661696C656420746F20656E6163
:101A6000626C6520426564204C6576656C696E67C2
:101A70000A004D65736820426564204C6576656C8C
:101A800020646174613A0A004D65736820706F6963
:101A90006E742063616E6E6F742062652072657370
:101AA0006F6C7665640A004D34323120696E636F65
:101AB000727265637420706172616D657465722005
:101AC00075736167650A002066697273740A005A4B
:101AD0000059005800486F6D652000546F6F2066F4
:101AE00061722066726F6D207265666572656E63E5
:101AF0006520706F696E740A0020496E76616C69AA
:101B00006420657874727564657220000000A0C05E
:101B10000000000000000000000057430000574391
:101B200000004E43486F6D696E67206661696C65A1
:101B30006400206E6F7420656E74657265642E0A91
:101B40000046696C652064656C657465643A0044A0
:101B5000656C6574696F6E206661696C65642C20C4
:101B600046696C653A200050726F746563746564F1
:101B70002050696E0A004A3036004A3034004A303C
:101B8000370020573A004A3038004A303900205791
:101B90003A00205A3A0020593A0020436F756E747B
:101BA00020583A0020453A00205A3A0020593A007D
:101BB000583A00454550524F4D2064617461736935
:101BC0007A65206572726F722E0A00290A002062FF
:101BD000797465733B206372632000536574746984
:101BE0006E67732053746F726564202800290A00A1
:101BF0002062797465733B206372632000207374E4
:101C00006F7265642073657474696E6773207265A2
:101C100074726965766564202800202863616C63AE
:101C2000756C6174656429210A0020213D200045FE
:101C30004550524F4D20435243206D69736D61747E
:101C40006368202D202873746F726564292000203A
:101C500053697A653A2000496E6465783A2000201D
:101C60004D61726C696E3D563535290A002845452F
:101C700050524F4D3D00454550524F4D20766572B4
:101C800073696F6E206D69736D6174636820000203
:101C90004A3135004A3132004A3137002020506C39
:101CA000616E6E65724275666665724279746573BF
:101CB0003A20002046726565204D656D6F72793A55
:101CC0002000436F6D70696C65643A204E6F76201A
:101CD000323820323031380A00207C204175746857
:101CE0006F723A2028646176696472616D69726FFF
:101CF0002C20666F7220416E79637562696320697A
:101D000033204D656761290A00323031392D313178
:101D10002D323800204C61737420557064617465F5
:101D2000643A2000312E312E390A004D61726C69FF
:101D30006E0020536F66747761726520526573651B
:101D4000740A00205761746368646F67205265737A
:101D500065740A002042726F776E206F757420528E
:101D6000657365740A002045787465726E616C2035
:101D700052657365740A00506F77657255700A007A
:101D800073746172740A004D3234004D3233202571
:101D900073006175746F25692E67006572726F72CA
:101DA0002077726974696E6720746F2066696C654C
:101DB0000A00205A3A0020593A0020583A00656E2D
:101DC0006473746F7073206869743A2000446F6E96
:101DD0006520736176696E672066696C652E0A00FE
:101DE0004D3239006F70656E206661696C65642CD8
:101DF0002046696C653A200043616E6E6F74206FF7
:101E000070656E2073756264697220004A30350017
:101E10004A3233004739310A4731205A2D313020B8
:101E2000463234300A4739300053442063617264CB
:101E3000206F6B0A006F70656E526F6F7420666161
:101E4000696C65640A00766F6C756D652E696E69E4
:101E500074206661696C65640A004572726F723A3B
:101E600000534420696E6974206661696C0A0065DC
:101E700063686F3A001000C90210012C0140012272
:101E80000170011801B0010E01F00104015002FAC5
:101E900000B002F0003003E600D003DC009004D272
:101EA000007005C800A006BE000008B400B009AA72
:101EB00000D00BA000600E960060118C000015820F
:101EC0000020197800C01D6E00A0226400B0275ABF
:101ED00000902C500000314600E0343C00103832B5
:101EE00000903A2800603C1E00A03D1400803E0A8D
:101EF00000203F00002CFFFFFFFFFF000101010158
:101F0000016265640A002C2073797374656D207317
:101F1000746F7070656421204865617465725F49F3
:101F2000443A20004265642068656174696E6720E8
:101F30006661696C65640048656174696E672066F6
:101F400061696C65640045312048656174696E673C
:101F5000206661696C65640048656174696E67201C
:101F60006661696C65640070012C0190012701B005
:101F7000012201C0011D01F00118011002130130FE
:101F8000020E016002090190020401C002FF00007C
:101F900003FA004003F5008003F000D003EB0020BB
:101FA00004E6007004E100E004DC004005D700C056
:101FB00005D2004006CD00D006C8008007C300301F
:101FC00008BE00F008B900C009B400B00AAF00B004
:101FD0000BAA00D00CA500000EA000500F9B00C063
:101FE0001096005012910000148C00C0158700B0AC
:101FF000178200B0197D00D01B7800001E730040CE
:10200000206E0090226900F024640040275F009059
:10201000295A00E02B5500102E500020304B0010A4
:10202000324600E033410090353C001037370070F5
:10203000383200A0392D00B03A2800A03B230060C0
:102040003C1E00103D1900903D1400103E0F007022
:102050003E0A00C03E0500003F0000403FFBFF80FD
:102060003FF6FFC03FF1FF453120544845524D41F6
:102070004C2052554E415741590042454420544846
:1020800045524D414C2052554E41574159005468DC
:1020900065726D616C2052756E61776179004531B2
:1020A000204572723A204D415854454D50004572BA
:1020B000723A204D415854454D5020424544004D00
:1020C000415854454D502074726967676572656464
:1020D000004531204572723A204D494E54454D50CD
:1020E000004572723A204D494E54454D50204245AC
:1020F00044004D494E54454D5020747269676765E0
:10210000726564004D383420582059205A2045000B
:10211000202F002042403A0020403A007C3C3E5EA6
:102120002B3D3F2F5B5D3B2C2A225C0054524947DC
:102130004745524544006F70656E003A20007A3280
:102140005F6D696E007A5F6D696E00795F6D696EB3
:1021500000785F6D696E005265706F7274696E67AA
:1021600020656E6473746F70207374617475730A84
:10217000000A4D6561737572656420706F696E74D5
:10218000733A0A005A206F66667365743A20004EEF
:10219000756D20582C593A20352C350A0000000066
:1021A000010000000100008000555555000000406E
:1021B0000033333300AAAA2A0049922400000020E9
:1021C00000C7711C0099991900D145170055551584
:1021D000003BB1130024491200111111000000103E
:1021E000000F0F0F00E3380E0043790D00CCCC0C2C
:1021F00000C3300C00E8A20B0064210B00AAAA0A5D
:1022000000703D0A009DD80900427B090092240914
:1022100000DCD3080088880800104208000000088D
:1022200000F0C107008787070075500700711C0781
:10223000003EEB0600A1BC0600699006006666063B
:1022400000703E06006118060017F4050074D10501
:10225000005BB00500B2900500627205005555059F
:102260000078390500B81E0500050505004EEC0490
:102270000087D40400A1BD040090A7040049920483
:1022800000C17D0400EE690400C756040044440404
:10229000005C320400082104004110040000000426
:1022A000003FF00300F8E0030026D20300C3C3039D
:1022B00000CCB503003AA803000A9B0300388E0344
:1022C00000C08103009F750300D0690300505E03C6
:1022D000001D53030034480300913D0300333303D2
:1022E0000016290300381F030097150300300C0364
:1022F00000030303000BFA020049F10200BAE802EE
:10230000005CE002002DD802002DD0020059C80266
:1023100000B0C0020031B90200DAB10200AAAA027C
:1023200000A0A30200BC9C0200FA9502005C8F0290
:1023300000DF88020082820200457C0200277602CC
:102340000027700200436A02007C640200D05E0233
:10235000003F590200C853020048617264636F6411
:1023600065642044656661756C7420536574746996
:102370006E6773204C6F616465640A00B80B0000DF
:10238000B80B00003C000000102700000000FA43DA
:102390000000FA430000C040000070420000A0426C
:1023A0000000A0420000C843E17AD24220286D6DAF
:1023B000290020204D393030204B004C696E65617A
:1023C0007220416476616E63653A0A002044002001
:1023D000490020204D333034205000204400204953
:1023E0000020204D33303120500050494420736587
:1023F0007474696E67733A0A00205A0020204D36C3
:10240000363600456E6473746F702061646A75734C
:10241000746D656E743A0A00205A0020590020201D
:10242000473239205333205800205A0020204D34A1
:1024300032302053004D65736820426564204C653E
:1024400076656C696E673A0A00205A0020590020B0
:10245000204D323036205800486F6D65206F66661B
:102460007365743A0A00204500205A002059002064
:10247000580020540020530020204D323035205188
:102480000020453C6D61785F655F6A65726B3E0058
:1024900020583C6D61785F785F6A65726B3E2059A9
:1024A0003C6D61785F795F6A65726B3E205A3C6D66
:1024B00061785F7A5F6A65726B3E00416476616E37
:1024C0006365643A20513C6D696E5F7365676D6545
:1024D0006E745F74696D655F75733E20533C6D6902
:1024E0006E5F66656564726174653E20543C6D691B
:1024F0006E5F74726176656C5F6665656472617447
:10250000653E0020540020520020204D32303420FF
:102510005000416363656C65726174696F6E202859
:10252000756E6974732F7332293A20503C7072694A
:102530006E745F616363656C3E20523C72657472B9
:102540006163745F616363656C3E20543C747261C7
:1025500076656C5F616363656C3E0A002045002010
:102560005A0020590020204D3230312058004D6152
:1025700078696D756D20416363656C65726174691E
:102580006F6E2028756E6974732F7332293A0A00B2
:10259000204500205A0020590020204D32303320A1
:1025A00058004D6178696D756D206665656472616E
:1025B0007465732028756E6974732F73293A0A0045
:1025C000204500205A0020590020204D3932205843
:1025D0000053746570732070657220756E69743A6B
:1025E0000A0020204D3230302044300A0020204D97
:1025F0003230302044002044697361626C65640AA3
:102600000046696C616D656E742073657474696EE3
:1026100067733A002020473231202020203B00FF02
:10262000FDFCFAF8F6F4F2F0EEECEAE9E7E5E3E1B6
:10263000E0DEDCDAD9D7D5D4D2D0CFCDCBCAC8C76B
:10264000C5C3C2C0BFBDBCBAB9B7B6B4B3B2B0AFF0
:10265000ADACAAA9A8A6A5A4A2A1A09E9D9C9A994A
:10266000989795949392908F8E8D8B8A8988878680
:1026700084838281807F7E7D7B7A7978777675749A
:10268000737271706F6E6D6C6B6A69686766656492
:10269000636261605F5E5D5C5B5A5958585756557E
:1026A0005453525150504F4E4D4C4B4A4A49484753
:1026B0004646454443424241403F3E3E3D3C3B3B13
:1026C0003A39383837363535343332323130302FC5
:1026D0002E2E2D2C2B2B2A29292827272625252469
:1026E000232322212120201F1E1E1D1C1C1B1B1A00
:1026F000191918181716161515141313121211118B
:10270000100F0F0E0E0D0D0C0C0B0A0A090908080C
:10271000070706060505040403030202010000453D
:1027200072726F722077726974696E6720746F209D
:10273000454550524F4D210A00000021002400273A
:10274000002A002D003000330001010000040107C1
:10275000010A0100002200250028002B002E003174
:1027600000340002010000050108010B01000020F7
:10277000002300260029002C002F00320000010059
:1027800000030106010901050505050705080808FC
:1027900008020202020A0A080804040404010101F2
:1027A00001010101010303030303030303040707FA
:1027B000070C0C0C0C0C0C0C0C0202020206060698
:1027C00006060606060B0B0B0B0B0B0B0B01021080
:1027D000202008081020401020408002010201083B
:1027E00004020101020408102040808040201008EB
:1027F0000402018004020180402010080402010844
:1028000004020101020408102040800102040810A3
:1028100020408000000A0B02090C0D0E080703047B
:1028200001000000000000000000000000000000A7
:102830000000000000000000000000000000001286
:102840001110000000000000000000000000000067
:10285000000000000000000000556E6B6E6F776E88
:1028600020636F6D6D616E643A2022000000484263
:102870000000484200008040000000005772697468
:10288000696E6720746F2066696C653A20006F700E
:10289000656E206661696C65642C2046696C653ADA
:1028A00020006F70656E206661696C65642C20463F
:1028B000696C653A200046696C652073656C6563D8
:1028C0007465640A002053697A653A200046696C91
:1028D00065206F70656E65643A20002066696C65DE
:1028E0003A2000646F696E67006672657368004E17
:1028F0006F772000454E4420535542524F5554495E
:102900004E450A002220706F7300222070617265AC
:102910006E743A2200535542524F5554494E452049
:1029200043414C4C207461726765743A22004B49F4
:102930004C4C45442E2000747279696E6720746F88
:102940002063616C6C207375622D67636F64652012
:1029500066696C6573207769746820746F6F206D89
:10296000616E79206C6576656C732E204D41582020
:102970006C6576656C2069733A00D8CFF2C9112472
:102980001FBECFEFD1E2DEBFCDBF00E00CBF14E031
:10299000A0E0B2E0EEEEFAEB01E00BBF02C0079060
:1029A0000D92AC30B107D9F728E1ACE0B4E001C03A
:1029B0001D92AD33B207E1F714E1CEEBD4E100E0B4
:1029C00006C021970109802FFE010E94CFDCCD3B7C
:1029D000D10780E00807A9F70E943ECA0C9466DD83
:1029E0000C9400002F923F924F925F926F927F92D1
:1029F0008F929F92AF92BF92CF92DF92EF92FF920F
:102A00000F931F93CF93DF93CDB7DEB7C45AD1098D
:102A10000FB6F894DEBF0FBECDBF91E09093C50511
:102A2000809136188D3411F40C94D024843511F42F
:102A30000C945230873411F00C949E30209034184E
:102A40003090351825E02216310409F43EC66CF4A6
:102A500044E0241631040CF0F9C552E02516310487
:102A6000B4F537FE2DC00C94CC246AE2261631044E
:102A700011F40C946C2374F48CE12816310411F4D5
:102A80000C9471219DE12916310411F40C947621E6
:102A90000C94CC24ABE52A16310411F40C94F723E2
:102AA000BCE52B16310411F40C94FB23EAE52E1639
:102AB000310411F00C94CC2410921E040C94A0301C
:102AC0008091350281110C94A5300C94A030809136
:102AD0003502882311F40C94A0300E94687F82E5AF
:102AE0000E949D51882309F454C10E941D514B013D
:102AF0005C0120E030E0A9010E948DD5882309F413
:102B000078C1C0902904D0902A04E0902B04F09062
:102B10002C04CCAEDDAEEEAEFFAEC0902D04D09056
:102B20002E04E0902F04F09030042496CCAEDDAE5D
:102B3000EEAEFFAE2497C090E005D090E105E090A6
:102B4000E205F090E3052C96CCAEDDAEEEAEFFAE26
:102B50002C97C090E405D090E505E090E605F09054
:102B6000E7052896CCAEDDAEEEAEFFAE28972C96EC
:102B70002CAD3DAD4EAD5FAD2C976CAD7DAD8EAD4A
:102B80009FAD0E948DD581110DC0A701960124969D
:102B90006CAD7DAD8EAD9FAD24970E948DD5882301
:102BA00009F427C111E022E02216310409F010E0F7
:102BB00020E030E0A901C501B4010E948DD5881F35
:102BC0008827881F181739F0C12CD12C90E8E92EDE
:102BD0009FEBF92E06C0C12CD12C80E8E82E8FE3A4
:102BE000F82E6896CCAEDDAEEEAEFFAE68972CAD9B
:102BF0003DAD4EAD5FAD2C966CAD7DAD8EAD9FAD58
:102C00002C970E94B6D964966CAF7DAF8EAF9FAF04
:102C1000649724962CAD3DAD4EAD5FAD24972896BC
:102C20006CAD7DAD8EAD9FAD28970E94B6D96B017E
:102C30007C0164962CAD3DAD4EAD5FAD6497CA018D
:102C4000B9010E94F2D52B013C01A7019601C701F1
:102C5000B6010E94F2D59B01AC01C301B2010E94F2
:102C6000B7D90E9422DC60966CAF7DAF8EAF9FAF6C
:102C7000609720E030E040E05FE30E94F2D52B0156
:102C80003C01A5019401C501B4010E94F2D54B019C
:102C90005C01A3019201C301B2010E94F2D59B0124
:102CA000AC01C501B4010E94B6D90E9422DC68962D
:102CB0002CAD3DAD4EAD5FAD68970E94F2D54B0196
:102CC0005C01C701B601905860962CAD3DAD4EAD8C
:102CD0005FAD60970E9493DAA50194010E94F2D53E
:102CE0006B017C012C962CAD3DAD4EAD5FAD2C97AC
:102CF0006CAD7DAD8EAD9FAD0E94B7D920E030E0C8
:102D000040E05FE30E94F2D59B01AC01C701B60130
:102D10000E94B7D92CAD3DAD4EAD5FAD0E94B6D986
:102D20006B017C0128962CAD3DAD4EAD5FAD289773
:102D300024966CAD7DAD8EAD9FAD24970E94B7D922
:102D400020E030E040E05FE30E94F2D52B013C013F
:102D500060962CAD3DAD4EAD5FAD609764966CADA9
:102D60007DAD8EAD9FAD64970E9493DAA50194016D
:102D70000E94F2D59B01AC01C301B2010E94B7D9F8
:102D800024962CAD3DAD4EAD5FAD24970E94B6D9D3
:102D900014C089E40E949D51882329F00E941D518E
:102DA0006B017C0103C0C12CD12C76018AE40E9406
:102DB0009D51882309F10E941D512C966CAF7DAF67
:102DC0008EAF9FAF2C9720E030E0A901C701B6017C
:102DD0000E948DD581111FC020E030E0A9012C9602
:102DE0006CAD7DAD8EAD9FAD2C970E948DD58111C0
:102DF00012C0EAE5FEE116C420E030E0A901C701F7
:102E0000B6010E948DD58823A1F32C961CAE1DAE71
:102E10001EAE1FAE2C97A701960150582CAF3DAFA8
:102E20004EAF5FAF2C964CAD5DAD6EAD7FAD2C97C8
:102E3000705824964CAF5DAF6EAF7FAF24972CAD2A
:102E40003DAD4EAD5FADCA01B9010E94F2D54B0157
:102E50005C0124962CAD3DAD4EAD5FAD2497CA010B
:102E6000B9010E94F2D59B01AC01C501B4010E94D9
:102E7000B7D90E9422DCA8966CAF7DAF8EAF9FAF12
:102E8000A8976091290470912A0480912B04909155
:102E90002C0428966CAF7DAF8EAF9FAF2897A7010B
:102EA00096010E94B7D968966CAF7DAF8EAF9FAF89
:102EB0006897C0902D04D0902E04E0902F04F090DD
:102EC00030046496CCAEDDAEEEAEFFAE64972C96C9
:102ED0002CAD3DAD4EAD5FAD2C97C701B6010E9444
:102EE000B7D9A4966CAF7DAF8EAF9FAFA497C090BB
:102EF000E005D090E105E090E205F090E3056C96E6
:102F0000CCAEDDAEEEAEFFAE6C9768962CAD3DADAF
:102F10004EAD5FAD6897C701B6010E94B6D96B018F
:102F20007C012091E4053091E5054091E605509142
:102F3000E705A0962CAF3DAF4EAF5FAFA097A4962C
:102F40002CAD3DAD4EAD5FADA497A0966CAD7DAD03
:102F50008EAD9FADA0970E94B6D94B015C01409108
:102F60003104509132046091330470913404AC9672
:102F70004CAF5DAF6EAF7FAFAC979A01AB01609184
:102F8000E8057091E9058091EA059091EB050E94B2
:102F9000B6D960966CAF7DAF8EAF9FAF6097A7013B
:102FA00096016CAD7DAD8EAD9FAD0E94F2D52B012B
:102FB0003C01A501940124966CAD7DAD8EAD9FAD15
:102FC00024970E94F2D59B01AC01C301B2010E947B
:102FD000B7D92B013C01A50194016CAD7DAD8EAD3F
:102FE0009FAD0E94F2D54B015C01A701960124968A
:102FF0006CAD7DAD8EAD9FAD24970E94F2D59B0147
:10300000AC01C501B4010E94B6D9A30192010E948E
:103010002ADA6B017C0120E030E0A9010E948DD505
:1030200087FF0AC02BED3FE049EC50E4C701B60131
:103030000E94B7D96B017C0152E02516310451F48E
:103040002BED3FE049EC50E4C701B6010E94B6D930
:103050006B017C0120E030E0A901C701B6010E94AC
:103060008DD5811128C06C962CAD3DAD4EAD5FADB8
:103070006C9728966CAD7DAD8EAD9FAD28970E9464
:103080008DD5811118C0A0962CAD3DAD4EAD5FAD74
:10309000A09764966CAD7DAD8EAD9FAD64970E9498
:1030A0008DD5811108C00BEDC02E0FE0D02E09EC9C
:1030B000E02E00E4F02EA7019601A8966CAD7DAD40
:1030C0008EAD9FADA8970E94F2D54B015C0120E028
:1030D00030E0A90160966CAD7DAD8EAD9FAD60977F
:1030E0000E948DD58823E9F0A5019401C501B401A2
:1030F0000E94F2D54B015C0160962CAD3DAD4EAD0A
:103100005FAD6097CA01B9010E94F2D59B01AC0185
:10311000C501B4010E94B7D90E9422DC4B015C01B9
:103120000DC020E030E0A901C501B4010E94DDDB43
:1031300087FF04C0B7FAB094B7F8B0942FE632E135
:1031400043E85AE3C501B4010E948DD587FF02C050
:103150000C94A030C501B4010E942CDB0E9400DB5E
:1031600062967FAF6EAF6297672B31F461E070E0DB
:1031700062967FAF6EAF62974090350450903604F0
:1031800060903704709038046296AEADBFAD629720
:10319000BD0180E090E00E9491D54B015C019B0154
:1031A000AC01C701B6010E9493DA28966CAF7DAFDF
:1031B0008EAF9FAF2897A501940160966CAD7DAD51
:1031C0008EAD9FAD60970E9493DAA8966CAF7DAFED
:1031D0008EAF9FAFA897A30192016091EC0570910B
:1031E000ED058091EE059091EF050E94B6D9A501FD
:1031F00094010E9493DAE0966CAF7DAF8EAF9FAFE3
:10320000E09728962CAD3DAD4EAD5FAD2897CA0135
:10321000B9010E94F2D520E030E040E05FE30E9477
:10322000F2D59B01AC0160E070E080E89FE30E9472
:10323000B6D96C966CAF7DAF8EAF9FAF6C97AC96E6
:10324000CCACDDACEEACFFACAC97C986DA86EB86D5
:10325000FC864D865E866F86788A60910202709148
:103260000302072E000C880B990B0E9493D5209126
:103270004B0230914C0240914D0250914E020E94FF
:10328000F2D52AE037ED43E25CE30E94F2D56CA769
:103290007DA78EA79FA70E9402C59B01AC01285362
:1032A0003F4F4F4F5F4FA0962CAF3DAF4EAF5FAF3C
:1032B000A0974CAC5DAC6EAC7FAC22242394312C37
:1032C00039E12D963FAF2D9762964EAD5FAD629777
:1032D0004215530509F453C10E94239E0E9402C562
:1032E000DC01CB01A096CCACDDACEEACFFACA09782
:1032F0008C199D09AE09BF09B7FD10C00E9402C517
:103300009B01AC0128533F4F4F4F5F4FA0962CAF0E
:103310003DAF4EAF5FAFA0970E9452582D963FAD84
:103320002D9731502D963FAF2D97332309F44BC085
:1033300024962CAD3DAD4EAD5FAD24976C966CAD33
:103340007DAD8EAD9FAD6C970E94F2D56B017C0177
:103350009201A30128966CAD7DAD8EAD9FAD2897EF
:103360000E94F2D5A70196010E94B7D97B018C017A
:103370009201A3016C966CAD7DAD8EAD9FAD6C9747
:103380000E94F2D54B015C0124962CAD3DAD4EADB3
:103390005FAD249728966CAD7DAD8EAD9FAD28971F
:1033A0000E94F2D59B01AC01C501B4010E94B6D9BF
:1033B0002B013C01C701D80124968CAF9DAFAEAF65
:1033C000BFAF249757C0B10180E090E00E9491D533
:1033D00028962CAD3DAD4EAD5FAD28970E94F2D53D
:1033E0004B015C010E9490DA6B017C01C501B401C4
:1033F0000E9418DC4B015C01A70196016CAD7DAD0C
:103400008EAD9FAD0E94F2D52B013C012C962CADC8
:103410003DAD4EAD5FAD2C97C501B4010E94F2D514
:10342000A30192010E94B7D92B013C01A50194018F
:103430006CAD7DAD8EAD9FAD0E94F2D54B015C01B0
:103440002C962CAD3DAD4EAD5FAD2C97C701B601AE
:103450000E94F2D59B01AC01C501B4010E94B6D90E
:1034600024966CAF7DAF8EAF9FAF249749E12D9628
:103470004FAF2D979201A30168966CAD7DAD8EADD7
:103480009FAD68970E94B7D969837A838B839C83A9
:1034900024962CAD3DAD4EAD5FAD2497A4966CAD9A
:1034A0007DAD8EAD9FADA4970E94B7D96D837E830D
:1034B0008F839887A8962CAD3DAD4EAD5FADA89794
:1034C00069857A858B859C850E94B7D969877A87BB
:1034D0008B879C87E0962CAD3DAD4EAD5FADE09700
:1034E0006D857E858F8598890E94B7D96D877E8787
:1034F0008F87988BCE0101960E94315CE090C405C5
:103500001CAA1DAA1EAA1FAA89819A81AB81BC810F
:1035100088A399A3AAA3BBA38D819E81AF81B885FF
:103520008CA39DA3AEA3BFA389859A85AB85BC85DB
:1035300088A799A7AAA7BBA7AE01485D5F4FBE01A8
:103540006C5D7F4FCE0180960E94B2AEBE016C5C76
:103550007F4F6B018E01045D1F4F9E01235F3F4F24
:10356000AE01485D5F4F60517109CE0180960E94A7
:10357000E460882321F07FEF271A370AA5CEE09078
:10358000C40518AE19AE1AAE1BAE8091E00590913D
:10359000E105A091E205B091E30588A399A3AAA350
:1035A000BBA38091E4059091E505A091E605B0915B
:1035B000E7058CA39DA3AEA3BFA38091E8059091DE
:1035C000E905A091EA05B091EB0588A799A7AAA7FC
:1035D000BBA7AE01485D5F4FBE016C5D7F4FCE0162
:1035E00080960E94B2AECE01C8966C018E01045D39
:1035F0001F4F2CEE35E0AE01485D5F4FBE016C5DA4
:103600007F4F48970E94E46080E1E0EEF5E0A9E298
:10361000B4E001900D928A95E1F70C94A0300E94DD
:10362000B951F80184918F010F5F1F4F8111F7CFBE
:10363000EDE1F2E084918F010F5F1F4F882311F4B9
:103640000C94A0300E94B951F801F4CF80E50E949B
:103650009D51882379F080910C0490910D0400977E
:1036600049F04AE050E060E070E00E940CD46B0149
:103670007C0103C0C12CD12C760183E50E949D51B1
:10368000882361F00E941D5120E030E04AE754E4B5
:103690000E94F2D50E9400DB6B017C010E94087140
:1036A0000E9402C5C60ED71EE81EF91E0E9402C562
:1036B000DC01CB018C199D09AE09BF09B7FD02C021
:1036C0000C94A0300E945258F1CF8091350288238B
:1036D00011F40C94A0300E94687F89E40E949D51EF
:1036E000882329F00E941D512B013C0103C0412C6D
:1036F000512C32018AE40E949D51882329F00E94B6
:103700001D514B015C0103C0812C912C540180E5BB
:103710000E949D51882329F00E941D516B017C015C
:1037200003C0C12CD12C760181E50E949D518823D4
:1037300039F00E941D516CAF7DAF8EAF9FAF04C0BA
:103740001CAE1DAE1EAE1FAE9091C405CC55DF4F12
:103750009883C45AD0406091020270910302072EF0
:10376000000C880B990B0E9493D520914B0230914D
:103770004C0240914D0250914E020E94F2D52AE037
:1037800037ED43E25CE30E94F2D568AB79AB8AABDC
:103790009BAB2091290430912A0440912B04509135
:1037A0002C0424962CAF3DAF4EAF5FAF2497C301DE
:1037B000B2010E94B7D9EB966CAF7DAF8EAF9FAFD1
:1037C000EB9740902D0450902E0460902F04709041
:1037D0003004A3019201C501B4010E94B7D9EF964C
:1037E0006CAF7DAF8EAF9FAFEF972091E00530912A
:1037F000E1054091E2055091E305C701B6010E9441
:10380000B7D9C158DF4F688379838A839B83CF57A9
:10381000D0402091E4053091E5054091E6055091B6
:10382000E7056CAD7DAD8EAD9FAD0E94B7D9CD578C
:10383000DF4F688379838A839B83C358D040249663
:10384000CCACDDACEEACFFAC2497C982DA82EB8263
:10385000FC824D825E826F8278860E9402C59B0147
:10386000AC0128533F4F4F4F5F4FC156DF4F288366
:1038700039834A835B83CF59D040BDEC8B2EBCEC9F
:103880009B2EA92CBDE3BB2E2D961FAE2D976196C6
:103890001FAE619765961FAE6597A1961FAEA19763
:1038A0000E94239E0E9402C58B019C01C156DF4FDE
:1038B000C880D980EA80FB80CF59D0400C191D09FF
:1038C0002E093F0937FD10C09B01AC0128533F4F23
:1038D0004F4F5F4FC156DF4F288339834A835B8345
:1038E000CF59D0400E945258A50194012D96BFADEA
:1038F0002D976196AFAD61976596FFAD6597A196DF
:10390000EFADA1976B2F7A2F8F2F9E2F0E94B7D9E3
:103910006CAF21967FAF219729968FAF2997259677
:103920009FAF259720E030E040E85FE30E94DDDBB9
:10393000181664F41CAE21961FAE219730E8299624
:103940003FAF29974FE325964FAF25976091E0054C
:103950007091E1058091E2059091E305C957DF4F31
:10396000688379838A839B83C758D04080912904D8
:1039700090912A04A0912B04B0912C04C557DF4FDD
:1039800088839983AA83BB83CB58D04025969FAD6B
:1039900025979F932996AFAD2997AF932196BFADF9
:1039A0002197BF93ECADEF93C957DF4FA880B98043
:1039B000CA80DB80C758D040C158DF4FE880F9800B
:1039C0000A811B81CF57D040EB962CAD3DAD4EAD5B
:1039D0005FADEB97C557DF4F688179818A819B8105
:1039E000CB58D0400E946EB70F900F900F900F9061
:1039F00069966FAF69976D967FAF6D97A9968FAFF8
:103A0000A997A5969FAFA597C090E405D090E5052E
:103A1000E090E605F090E705C157DF4FC882D982F4
:103A2000EA82FB82CF58D04020912D0430912E04A1
:103A300040912F0450913004CD56DF4F28833983B5
:103A40004A835B83C359D04025963FAD25973F936A
:103A500029964FAD29974F9321965FAD21975F939C
:103A60006CAD6F93C157DF4FA880B980CA80DB80EF
:103A7000CF58D040CD57DF4FE880F9800A811B81B5
:103A8000C358D040EF962CAD3DAD4EAD5FADEF9736
:103A9000CD56DF4F688179818A819B81C359D0409F
:103AA0000E946EB70F900F900F900F90AD966FAF72
:103AB000AD97E1967FAFE197E2968FAFE297E396FD
:103AC0009FAFE39789819A81AB81BC81C956DF4F53
:103AD00088839983AA83BB83C759D040CD80DE8079
:103AE000EF80F884C556DF4FC882D982EA82FB8214
:103AF000CB59D040E4961FAEE4972D967FAD2D971D
:103B000061966FAD619765969FAD6597A1968FADF4
:103B1000A197272F362F492F582FBCAD2196AFAD37
:103B200021972996FFAD29972596EFAD25976B2F05
:103B30007A2F8F2F9E2F0E94B6D92FE632E143E0D5
:103B40005BE30E948DD587FD3DC17CAD21966FADB5
:103B5000219729969FAD299725968FAD2597272FD9
:103B6000362F492F582F2D96BFAD2D976196AFADAB
:103B700061976596FFAD6597A196EFADA1976B2F05
:103B80007A2F8F2F9E2F0E94B7D920E030E040E09F
:103B90005FE30E94F2D5662E972E882E792E9F9392
:103BA0008F937F936F93C957DF4FA880B980CA80E6
:103BB000DB80C758D040C158DF4FE880F9800A81C8
:103BC0001B81CF57D040EB962CAD3DAD4EAD5FADD8
:103BD000EB97C557DF4F688179818A819B81CB58EC
:103BE000D0400E946EB70F900F900F900F90E59607
:103BF0006FAFE597E6967FAFE697E7968FAFE797CB
:103C0000CD55DF4F9883C35AD0407F928F929F92B9
:103C10006F92C157DF4FA880B980CA80DB80CF5830
:103C2000D040CD57DF4FE880F9800A811B81C3580F
:103C3000D040EF962CAD3DAD4EAD5FADEF97CD567C
:103C4000DF4F688179818A819B81C359D0400E946E
:103C50006EB70F900F900F900F90162F072FB82E62
:103C6000A92EAD962FADAD97E1963FADE197E296C7
:103C70004FADE297E3965FADE397C556DF4F68819E
:103C800079818A819B81CB59D0400E94B7D920E0AD
:103C900030E040E05FE30E94F2D51B012C01699601
:103CA0002FAD69976D963FAD6D97A9964FADA997CA
:103CB000A5965FADA597C956DF4F688179818A8146
:103CC0009B81C759D0400E94B7D920E030E040E046
:103CD0005FE30E94F2D59B01AC01E5966FADE597DD
:103CE000E6967FADE697E7968FADE797CD55DF4F28
:103CF0009881C35AD0400E94B6D96B017C0120E064
:103D000030E0A9010E94DDDB87FF04C0F7FAF094E0
:103D1000F7F8F094A2019101612F702F8B2D9A2D4D
:103D20000E94B6D91B012C0120E030E0A9010E94BD
:103D3000DDDB87FF04C057FA509457F85094A20176
:103D40009101C701B6010E94B7D92DEC3CEC4CECB7
:103D50005DE30E948DD51816ACF5AD961FAFAD97FB
:103D6000E1960FAFE197E296BFAEE297E396AFAE72
:103D7000E397E596DFACE5976996DFAE6997E6963F
:103D8000EFACE6976D96EFAE6D97E796FFACE797D1
:103D9000A996FFAEA997CD55DF4F2881C35AD040D1
:103DA000A5962FAFA5976CAE21969FAE2197299629
:103DB0008FAE299725967FAE259731E0E4963FAFE9
:103DC000E4979BCEE4964FADE497411158C12D96F0
:103DD0007FAD2D9761966FAD619765969FAD6597A5
:103DE000A1968FADA197272F362F492F582FBCAD05
:103DF0002196AFAD21972996FFAD29972596EFAD76
:103E000025976B2F7A2F8F2F9E2F0E94B6D96B018B
:103E10007C012DEC3CEC4CEC5DE30E94DDDB1816E4
:103E20000CF42DC1A7019601C701B6010E94B7D9B4
:103E30002D96EFAD2D976196BFAD61976596AFADAD
:103E40006597A196FFADA1972E2F3B2F4A2F5F2F8D
:103E50000E94B7D9662E972E882E792E20E030E06A
:103E600040E85FE30E94DDDB87FF09C17F928F920C
:103E70009F926F92C957DF4FA880B980CA80DB80BC
:103E8000C758D040C158DF4FE880F9800A811B81B4
:103E9000CF57D040EB962CAD3DAD4EAD5FADEB971F
:103EA000C557DF4F688179818A819B81CB58D0408B
:103EB0000E946EB70F900F900F900F90E4966FAF27
:103EC000E497E5967FAFE597E6968FAFE697E7969E
:103ED0009FAFE7977F928F929F926F92C157DF4F6C
:103EE000A880B980CA80DB80CF58D040CD57DF4F43
:103EF000E880F9800A811B81C358D040EF962CAD31
:103F00003DAD4EAD5FADEF97CD56DF4F6881798106
:103F10008A819B81C359D0400E946EB70F900F9049
:103F20000F900F90162F072FB82EA92E262F372F60
:103F3000482F592FC556DF4F688179818A819B812F
:103F4000CB59D0400E94B7D920E030E040E05FE399
:103F50000E94F2D56B017C01E4962FADE497E596C3
:103F60003FADE597E6964FADE697E7965FADE797ED
:103F7000C956DF4F688179818A819B81C759D040BA
:103F80000E94B7D920E030E040E05FE30E94F2D524
:103F90009B01AC0169966FAD69976D967FAD6D978A
:103FA000A9968FADA997A5969FADA5970E94B6D962
:103FB0001B012C0120E030E0A9010E94DDDB87FF1E
:103FC00004C057FA509457F85094A7019601AD9643
:103FD0006FADAD97E1967FADE197E2968FADE29739
:103FE000E3969FADE3970E94B6D96B017C0120E078
:103FF00030E0A9010E94DDDB87FF04C0F7FAF094EE
:10400000F7F8F094A2019101C701B6010E94B7D957
:104010002DEC3CEC4CEC5DE30E94DDDB18167CF1F2
:10402000AD961FAFAD97E1960FAFE197E296BFAEA9
:10403000E297E396AFAEE397E4965FADE4976996B7
:104040005FAF6997E5966FADE5976D966FAF6D972A
:10405000E6967FADE697A9967FAFA997E7968FADD5
:10406000E797A5968FAFA5976CAE21969FAE219747
:1040700029968FAE299725967FAE2597A8CE2D96A7
:104080007FAD2D9761966FAD619765969FAD6597F2
:10409000A1968FADA197272F362F492F582FBCAD52
:1040A0002196AFAD21972996FFAD29972596EFADC3
:1040B00025976B2F7A2F8F2F9E2F0E94B6D94B01F9
:1040C0005C0169968FAD69976D969FAD6D97A996C6
:1040D000AFADA997A596BFADA59789839A83AB830A
:1040E000BC83AD968FADAD97E1969FADE197E2961B
:1040F000AFADE297E396BFADE3978D839E83AF8329
:10410000B8877CAD21966FAD219729969FAD2997F1
:1041100025968FAD2597272F362F492F582F60E0F2
:1041200070E080E89FE30E94B6D96B017C0120918A
:1041300031043091320440913304509134040E9490
:10414000F2D52B013C012091E8053091E905409121
:10415000EA055091EB05BCAD2196AFAD21972996AC
:10416000FFAD29972596EFAD25976B2F7A2F8F2FCF
:104170009E2F0E94F2D59B01AC01C301B2010E94A7
:10418000B7D969877A878B879C87209135043091CE
:1041900036044091370450913804C701B6010E949B
:1041A000F2D56B017C012091EC053091ED05409139
:1041B000EE055091EF05BCAD2196AFAD2197299644
:1041C000FFAD29972596EFAD25976B2F7A2F8F2F6F
:1041D0009E2F0E94F2D59B01AC01C701B6010E943F
:1041E000B7D96D877E878F87988BCE0101960E9405
:1041F000315C1CA61DA61EA61FA689819A81AB81D3
:10420000BC8188A399A3AAA3BBA38D819E81AF8102
:10421000B8858CA39DA3AEA3BFA389859A85AB85E2
:10422000BC8588A799A7AAA7BBA7AE01485D5F4F29
:10423000BE016C5D7F4FCE0180960E94B2AEDE0162
:104240009C966D01CC55DF4FE880C45AD0408E015A
:10425000005D1F4F9E01235F3F4FAE01485D5F4FE2
:10426000BE016C5D7F4FCE0180960E94E460882382
:1042700069F120E030E040E85FE3BCAD2196AFADEE
:1042800021972996FFAD29972596EFAD25976B2F9E
:104290007A2F8F2F9E2F0E948DD587FF17C03CADA0
:1042A0002D963FAF2D9721964FAD219761964FAF39
:1042B000619729965FAD299765965FAF65972596BB
:1042C0006FAD2597A1966FAFA197EACA80E1E0EEA6
:1042D000F5E0A9E2B4E001900D928A95E1F70C9423
:1042E000A03080E00E9408810C94A03083E50E94F9
:1042F0009D51882321F10E94FD50182F863070F0C7
:10430000E5EEF2E084918F010F5F1F4F882311F4D7
:104310000C94A0300E94B951F801F4CF833009F415
:104320004AC130F4813091F1823009F43FC008C0B5
:10433000843009F49FC1853009F4ACC101C010E09C
:104340000E94BB80811103C0E5ECF2E013C08091B4
:10435000FD17882319F06BE073E002C06FE073E093
:104360008DEB92E00E9453B78AE00E94B9510E94FF
:10437000ECAE96C184917F01BFEFEB1AFB0A882354
:1043800009F48EC10E94B951F701F4CF0E949FAF8A
:10439000109201021092000282EB92E09093FC07CF
:1043A0008093FB070E94E5510C94A030809100029D
:1043B0009091010297FF0EC0E9E8F2E084918F012D
:1043C0000F5F1F4F882311F40C94A0300E94B95145
:1043D000F801F4CF0097A1F48091210280931F048B
:1043E00019821A821B821C8218A219A21AA21BA26D
:1043F000BE016F5F7F4FCE0180960E946DC227C0C5
:10440000815065E00E947FDC80FF03C024E0291B0F
:10441000922F25E09202F0011124E80FF11D87FD93
:10442000FA95EE0FFF1FEE0FFF1FEB54FF4E80912A
:10443000310490913204A0913304B091340480830C
:104440009183A283B38380911F0480932102809182
:10445000000290910102893191050CF067C0109221
:1044600021029C012F5F3F4F3093010220930002F5
:1044700065E00E947FDC80FF03C024E0291B922FAF
:1044800040913104509132046091330470913404AE
:1044900048A359A36AA37BA319821A821B821C8298
:1044A00044E0840290011124B9016F5B754F4B0108
:1044B000DB012D913D914D915C91B4E09B02C001D7
:1044C0001124FC01EB5AF54F5F01608171818281FB
:1044D0009381DE0111966D01E12CF12C00EA10E4CC
:1044E0000E949DC119821A821B821C82B601CE01D4
:1044F00080960E946DC2F50180819181A281B38175
:104500008093290490932A04A0932B04B0932C0445
:10451000F40180819181A281B38180932D049093D5
:104520002E04A0932F04B0933004BCC080E090E030
:10453000A0EAB0E48093310490933204A093330452
:10454000B09334040E94F5810E9408718FEF9FEFB1
:104550009093010280930002E5E7F2E084918F01DD
:104560000F5F1F4F882321F00E94B951F801F6CF49
:1045700083E992E09A83898304E610E019A308A3F3
:10458000BE016F5F7F4FCE0180960E9420C38AEBF1
:1045900092E09A83898319A308A3BE016F5F7F4FBE
:1045A000CE0180960E9420C381E00E94088181E0B4
:1045B0000E94E88077C088E50E949D518823A1F081
:1045C0000E94ED501FEF160F1530A8F0EEE5F2E057
:1045D00084918F010F5F1F4F882311F40C94A0303A
:1045E0000E94B951F801F4CF88E50E94B9510E94A8
:1045F0002ECA0C94A03089E50E949D518823A1F019
:104600000E94ED500FEF060F0530A8F0E7E4F2E04E
:1046100084918F010F5F1F4F882311F40C94A030F9
:104620000E94B951F801F4CF89E50E94B9510E9466
:104630002ECA0C94A0308AE50E949D51882399F0DF
:104640000E941D5125E0129FF0011124E00FF11D81
:10465000EE0FFF1FEE0FFF1FEB54FF4E60837183C1
:104660008283938335C08AE50E94B9510E942ECA85
:104670000C94A0308AE50E949D518823A1F30E94EA
:104680001D516093B1107093B2108093B31090934A
:10469000B4101EC080E00E94E8800E949FAF18C046
:1046A0001230B1F46091000270910102693171051C
:1046B00014F069E170E088E392E00E943AB769E1A2
:1046C00070E083E392E00E943AB78AE00E94B95119
:1046D0000E94637C0C94A03080913502882311F4F1
:1046E0000C94A03089E40E949D51E82E882321F08B
:1046F0000E94ED50062F01C000E08AE40E949D5107
:10470000F82E882321F00E94ED50162F01C010E0F2
:10471000EE2011F0053020F4FF2081F0153070F00C
:10472000ECEFF2E084918F010F5F1F4F882311F4AB
:104730000C94A0300E94B951F801F4CF0E94AF51FF
:10474000EE2091F034E00302F0011124EB5AF54F12
:1047500080819181A281B3818093E0059093E105EE
:10476000A093E205B093E305FF2091F044E014022A
:10477000F0011124EF5BF54F80819181A281B3811B
:104780008093E4059093E505A093E605B093E705D3
:1047900080E50E949D51882319F00E940E5103C0AC
:1047A00080E50E94545186E40E949D518823D9F0EF
:1047B0000E941D516B017C0120E030E0A9010E94A4
:1047C000DDDB181684F420E030E040E752E4C70156
:1047D000B6010E9493DA60934B0270934C0280936F
:1047E0004D0290934E020E94C85C0C94A0309093AE
:1047F0001E040C94A0309FE4292E92E0392E23ED64
:10480000E22E25E0F22E69E274E07DAF6CAF3EE06F
:10481000C32E34E0D32E00E010E0D1018D911D01B4
:104820000E949D51882309F44BC00E941D512B0109
:104830003C01133049F0F6012081318142815381DE
:104840000E94B6D92B013C01ACADBDAD2D913D917F
:104850004D915C91C301B2010E94B6D94B015C013C
:104860002DEB37E346E855EB0E94DDDB87FD0AC000
:104870002DEB37E346E855E3C501B4010E948DD521
:104880001816F4F4133051F4409235045092360463
:10489000609237047092380401E012C0A5019401BF
:1048A000F70160817181828193810E94B7D9D7011C
:1048B0006D937D938D939C931397812F0E944C82CF
:1048C0001F5FB4E0EB0EF11CECADFDAD3496FDAF17
:1048D000ECAFF4E0CF0ED11C143009F09ECF0023D2
:1048E00009F4F6CEC0903504D0903604E090370439
:1048F000F090380420E030E0A901C701B6010E9421
:10490000B7D920916A1130916B1140916C1150917F
:104910006D110E94F2D50E94E8DB60933D0A70930E
:104920003E0A80933F0A9093400AC0922D0AD0928B
:104930002E0AE0922F0AF092300A90910B0A809191
:104940000C0A981719F00E94AA70C2CE0E94087132
:1049500080916F00982F927081FF05C080916F0049
:104960008D7F80936F0040913D0A50913E0A609187
:104970003F0A7091400A4093311050933210609377
:10498000331070933410992309F4A2CE80916F00F4
:10499000826080936F009CCE0E9454C30C94A03020
:1049A00080913418909135188637910509F4CDC659
:1049B0000CF0C9C08D34910509F42BC40CF055C01E
:1049C0008A31910509F431C224F58531910509F444
:1049D000EAC184F48231910509F484C584319105DA
:1049E00009F4A1C1419711F00C944F300E940A5C68
:1049F0000C94A0308731910509F4DFC10CF4D7C1C4
:104A00008831910509F4EFC1499709F4F7C10C9475
:104A10004F308F31910509F404C39CF48C3191051A
:104A200009F4A9C20CF40FC28D31910511F40C9454
:104A3000A0304E9711F00C944F300E94CB840C9410
:104A4000A0308A32910509F49EC32CF4809709F4B2
:104A50009CC20C944F308B34910509F4C4C38C3440
:104A6000910509F4C3C30C944F308B36910509F4BA
:104A70000BC50CF042C08535910509F436C5FCF430
:104A80008235910509F427C584F48135910511F02B
:104A90000C944F300E94639B0E9494A910923A0498
:104AA0001092390400E010E0FFC48335910509F449
:104AB00015C58435910509F415C50C944F30883619
:104AC000910509F4A9C37CF48C35910511F00C947F
:104AD0004F30FFE4CF2EF2E0DF2EAEE5EA2EA1E16B
:104AE000FA2E10E01BC58936910509F452C48A36A6
:104AF000910509F4ADC40C944F308037910509F449
:104B000017C484F48D36910509F482C40CF40DC4E5
:104B10008E36910509F4A5C38F36910509F4B2C309
:104B20000C944F308237910509F477C50CF407C413
:104B30008337910509F4F4C08537910511F40C947D
:104B4000A0300C944F308E3221E0920711F40C9477
:104B50008B2E0CF068C08B3C910509F4B5C6ACF502
:104B60008C38910509F457C48CF48837910509F401
:104B70003CC60CF437C68937910511F00C944F30C0
:104B800010926806109267060C94A0308E3B910537
:104B900009F45BC434F48B39910509F414C40C9402
:104BA0004F30883C910509F426C6893C910511F0E7
:104BB0000C944F307FE4E72E72E0F72E0EE311E104
:104BC000EEE4CE2EE1E1DE2E66C68C3D910509F4C1
:104BD00035C79CF48D3C910509F407C70CF490C6C9
:104BE0008E3C910509F404C7833D910511F00C94A6
:104BF0004F300E94BF7A0C94A030823E910509F498
:104C000097C734F48D3D910509F425C70C944F30B6
:104C10008C3241E0940709F4B5C78D32914009F414
:104C2000DAC70C944F30853F61E0960711F40C947D
:104C3000782FDCF58A39A1E09A0709F47DC3BCF42A
:104C40008033E1E09E0711F40C94E22E14F40C94EE
:104C5000DF2E833621E0920709F45EC0803991404F
:104C600011F00C944F300E9408710C94A030853ADA
:104C700041E0940711F40C94752F4CF4843A914060
:104C800011F00C944F300E945C730C94A0308C3A5D
:104C900071E0970709F4CFC6843F914011F00C945E
:104CA0004F300E94A88B0C94A0308A39B2E09B0749
:104CB00011F40C94B72FB4F4873FF1E09F0711F47F
:104CC0000C947E2F14F40C947B2F883F31E09307D3
:104CD00011F40C948A2F8C30924011F40C94AE2F66
:104CE0000C944F308B3853E0950711F40C94A0309E
:104CF0003CF48438934011F40C94E42F0C944F301E
:104D0000803AA3E09A0709F47FC1873E934011F4EB
:104D10000C943C300C944F30EAE5FEE10C94622F89
:104D2000EDECF4E0B7C4EAE2F3E084918F010F5FA9
:104D30001F4F882321F00E94B951F801F6CF10923D
:104D4000070D8AEB9AE00E9411A48BE1EAEBFAE0EE
:104D5000DE01159601900D928A95E1F78091B80ACF
:104D60009091B90A9C838B8385EE92E09A83898324
:104D700040E050E0BE016F5F7F4F80E090E00E9416
:104D8000DD94CE0101960E94EB57EBE1F3E08491B4
:104D90008F010F5F1F4F882311F40C94A0300E94E5
:104DA000B951F801F4CF0E94AC920C94A03010924B
:104DB000890A10928A0A0C94A030E0913218F0917E
:104DC00033188081882329F0803209F410823196CB
:104DD000F8CF40E061E080913218909133180E9442
:104DE0006AC50C94A03080918A0A882319F081E06A
:104DF0008093890A0E942C9B0C94A0301092890AFF
:104E000080913910813011F00C94A03082E08093B1
:104E100039100E9402C5609335107093361080934C
:104E20003710909338100C94A03080918A0A882310
:104E300011F40C94A03083E50E949D5181110C94D3
:104E4000AA300C94A03083E40E945451882309F4C2
:104E500050C0E8E6F3E084918F010F5F1F4F882375
:104E600021F00E94B951F801F6CF8091550C8111C3
:104E700003C0EBE3F3E012C0BE016F5F7F4F82E53A
:104E80009CE00E94D9A28E010F5F1F4FF801819113
:104E90008F01882349F10E94B951F8CF84918F0185
:104EA0000F5F1F4F882301F10E94B951F801F6CF1F
:104EB000B0ECCB2EB3E0DB2EE12CF12C20E0809186
:104EC0004B0690E00E2C02C0959587950A94E2F768
:104ED00080FD08C2BFEFEB1AFB0AE2E0CE0ED11C48
:104EE000F5E0EF16F10459F78AE00E94B9510C94ED
:104EF000A03080918A0A882339F08091890A88231A
:104F000019F0E5E4F3E003C0E7E5F3E028C084919D
:104F10008F010F5F1F4F882321F00E94B951F801C4
:104F2000F6CF6091030D7091040D8091050D909165
:104F3000060D4AE00E94DB548FE20E94B951609155
:104F4000FF0C7091000D8091010D9091020D4AE0CF
:104F50000E94DB548AE00E94B9510C94A0308491E5
:104F60008F010F5F1F4F882311F40C94A0300E9413
:104F7000B951F801F4CF40E060E08091321890918F
:104F800033180E946AC50C94A0308091890A81115F
:104F90000E94087180918A0A882311F40C94A03031
:104FA00080E50E949D51882319F00E940E5103C094
:104FB00080E50E945451182F482F61E080913218EB
:104FC000909133180E946AC583E50E949D51882301
:104FD00081F00E94ED50AB01BC014093030D509352
:104FE000040D6093050D7093060D82E59CE00E9410
:104FF000CAA180918A0A882319F081E08093890AE6
:1050000011110C94A030F6CE809132189091331883
:1050100021E02093880A40E060E00E946AC50C9479
:10502000A0300E94DD9A7B018C0120E831E541E04F
:1050300050E00E947BD9C9016DE671E00E948CDCD2
:105040004B015C01C801B70120E13EE040E050E0C7
:105050000E947BD9CA01B90128E130E040E050E06C
:105060000E947BD9762E672EC62ED72E8CE3282E53
:10507000312C412C512CC801B701A20191010E9491
:105080007BD9F62EE72ECA01B901A20191010E9437
:105090007BD9CB018E010F5F1F4F81149104D1F09A
:1050A000EF92FF927F936F936F927F92BF92AF9236
:1050B0009F928F928FE993E09F938F931F930F930B
:1050C0000E945FD50FB6F894DEBF0FBECDBFEFE6EE
:1050D000FEE145C0A114B10489F0EF92FF927F93E5
:1050E0006F936F927F92BF92AF928FE893E09F93FE
:1050F0008F931F930F930E945FD5E4CFCD2879F053
:10510000EF92FF927F936F936F927F9283E893E089
:105110009F938F931F930F930E945FD5D3CF892BBB
:1051200069F0EF92FF927F936F938BE793E09F93E9
:105130008F931F930F930E945FD5C4CFEF92FF927E
:1051400087E793E09F938F931F930F930E945FD500
:105150000F900F900F900F900F900F90B8CF8491F9
:105160007F019FEFE91AF90A882321F00E94B951C3
:10517000F701F5CFB80183EB93E00E9453B78AE0C3
:105180000E94B951DDC783E50E949D51882309F42F
:10519000D7C70E94FD50E82E80E50E949D518823CC
:1051A00031F00E94FD50182F87FF02C0C9C71DE0D3
:1051B00089E40E949D51882341F00E940E51811183
:1051C0000C94E530E5EBF5E00AC089E40E94545107
:1051D000F6CF3196A5E0E53EFA0709F4F6C78491CB
:1051E0001813F7CFC8C70E942C9BAAC7809139100B
:1051F000813009F0A5C782E0809339100E9402C572
:105200006093351070933610809337109093381058
:1052100097C70E944E9B94C788E690E00E948C82BC
:1052200081118EC780914B0683FD8AC783E50E945A
:105230009D51882399F00E941D510E94FBDACB01F9
:105240000E9445910E941D5120E030E044EB52E461
:105250000E948DD5181614F00E944E9B0E947DB9B5
:105260006FC78EE40E949D51882309F469C70E948C
:10527000ED5060931018709311188093121890934A
:1052800013185EC783E50E945451882359F083E5C3
:105290000E949D51882319F00E94FD5001C080E0BA
:1052A00080934B06EFE6FEE184918F010F5F1F4F65
:1052B000811103C0EEECF3E004C00E94B951F80183
:1052C000F3CF84918F010F5F1F4F882321F00E943D
:1052D000B951F801F6CF80914B068111E9CDEAEC86
:1052E000F3E018C0BB24B394B20E222319F08CE271
:1052F0000E94B951F60185919491FC0184918F012E
:105300000F5F1F4F882321F00E94B951F801F6CF9B
:105310002B2DE0CD84918F010F5F1F4F882309F45F
:10532000E3CD0E94B951F801F5CF1092340208C7BD
:1053300085ED93E00E940D580E94227501C783E518
:105340000E949D51811103C0EFE6FEE10BC00E9457
:10535000FD508D3318F480932202F2C68CE38093C3
:105360002202EEC684918F010F5F1F4F882321F028
:105370000E94B951F801F6CF4091220250E060E05E
:1053800070E08EED93E00E9400B78AE00E94B95170
:10539000D7C689E690E00E948C82811111C0E5EEAB
:1053A000F3E084918F010F5F1F4F882321F00E944B
:1053B000B951F801F6CF0E9465988AE00E94B95170
:1053C0001092C50517C783E50E949D51882309F4F3
:1053D000B7C60E94FD50182F8D3308F01CE31093C0
:1053E000D2050E9402C56B017C01212F30E0A8EE9E
:1053F000B3E00E94A7D9C60ED71EE81EF91EC092C0
:10540000CE05D092CF05E092D005F092D10598C696
:105410000E94CE8295C680914B0683FD91C683E59E
:105420000E949D51882309F48BC60E941D510E9441
:10543000FBDA6E36710514F06EE670E070933C0492
:1054400060933B040E941F997BC60E948D7D78C6A5
:1054500080E50E949D51811106C083E50E949D5107
:10546000882359F005C00E94FD50811169C6F5CF0F
:105470000E94ED506F3F710510F06FEF70E0709378
:105480003A04609339045CC680E50E949D51811105
:1054900005C010923A041092390452C60E94ED5091
:1054A000672B09F04DC6F5CF62E370E080E090E035
:1054B0000E94CAC40E94239E0F5F1F4F0331110533
:1054C00099F762E370E080E090E00E94CAC40E9415
:1054D000239EAAD635C610921D0432C681E0809361
:1054E0001D042EC60E942D7D2BC683E50E945451BB
:1054F000882309F425C60E941D5120E030E04AE7C8
:1055000054E40E94F2D50E9400DB6093CA057093B8
:10551000CB058093CC059093CD0512C6D6018D9115
:105520006D010E945451882309F46DC0133009F0B5
:1055300063C00E941D514B015C0120E030E040EA55
:1055400051E40E948DD587FF4EC0A5019401609162
:105550006A1170916B1180916C1190916D110E9484
:1055600093DA2B013C019B01AC0160911A0670910A
:105570001B0680911C0690911D060E94F2D5609337
:105580001A0670931B0680931C0690931D06A301B8
:10559000920160913A0670913B0680913C06909191
:1055A0003D060E94F2D560933A0670933B068093C5
:1055B0003C0690933D0660913A1170913B118091A9
:1055C0003C1190913D110E9491D5A30192010E943E
:1055D000F2D50E9400DB60933A1170933B118093E7
:1055E0003C1190933D1180926A1190926B11A092A0
:1055F0006C11B0926D1107C00E941D51F7016083BC
:105600007183828393831F5FF4E0EF0EF11C1430EB
:1056100009F084CF0E941EBB93C50E94087183E5E8
:105620000E949D51882309F453C80E94ED506230B6
:10563000710509F04DC80E94155C8BE50E94B951B7
:105640006091B8057091B9058091BA059091BB053C
:1056500042E00E9460554091BC055091BD056091AB
:10566000BE057091BF058BEE93E00E941DB740917F
:10567000C0055091C1056091C2057091C30588EEC7
:1056800093E00E941DB78DE50E94B9518AE00E9407
:10569000B95156C584918F010F5F1F4F882321F0A8
:1056A0000E94B951F801F6CF60E08DEB94E00E94C2
:1056B0002C7C61E086EB94E00E942C7C61E08BEA1C
:1056C00094E00E942C7C61E08BE994E00E942C7CA9
:1056D00060E082E994E00E942C7C61E088E894E03C
:1056E0000E942C7C60E08EE794E00E942C7C60E0BD
:1056F00086E794E00E942C7C61E088E694E00E94BA
:105700002C7C60E08AE594E00E942C7C60E08BE4D5
:1057100094E00E942C7C60E08DE394E00E942C7C5D
:1057200060E087E294E00E942C7C60E086E194E0F7
:105730000E942C7C60E081E094E00E942C7C61E07F
:105740008EEE93E00E942C7CFBC4009132181091E5
:10575000331883E0D12C40E08150E9F0D8019C91CE
:10576000292F2B7F2134C1F711962C912133A1F7DA
:10577000913421F0953421F441E002C0DD24D3942A
:1057800098012E5F3F4F89012F5F3F4FF8019081B5
:105790009032C9F3E1CF442369F0EFE6FEE1849152
:1057A0007F012FEFE21AF20A882321F00E94B951FB
:1057B000F701F5CFDD2069F0E3E9F5E084917F01A1
:1057C0003FEFE31AF30A882321F00E94B951F70151
:1057D000F5CFD8018D918D01882309F485CB0E94E6
:1057E000B951F7CF0E9437B0ABC481E0809368060F
:1057F00080936706A5C488EC90E00E948C8281119A
:105800009FC484E40E945451882309F441C00E943B
:105810001D516B017C0111E020E030E0A9010E94E4
:105820008DD5811101C010E01093191120E030E0F6
:10583000A901C701B6010E948DD5882349F10E94B4
:105840001D51E0915C10B4E0EB9FF0011124E25E89
:10585000FE4E608371838283938320E030E0A90150
:1058600060911E1170911F11809120119091211152
:105870000E948DD581110CC080E090E0A0EEBFE3C6
:1058800080931E1190931F11A0932011B0932111AA
:105890000E94D2A955C4F70181917F010E94545101
:1058A000882351F00E941D510E9400DBD8016D93A6
:1058B0007D938D939C9313970C5F1F4FC016D10659
:1058C00051F70E94ADB93CC46FE4E62E62E0F62EBB
:1058D0000EE216E0F70181917F010E945451882366
:1058E00041F00E941D51D8016D937D938D939C933F
:1058F00013970C5F1F4FB6E00E331B0759F720C4F8
:1059000083E50E949D518823A1F00E941D51609360
:1059100026067093270680932806909329066093A5
:10592000220670932306809324069093250610E0A8
:1059300001C011E080E50E949D51882359F00E942A
:105940001D51609326067093270680932806909336
:10595000290610E082E50E949D51882359F00E949B
:105960001D5160932A0670932B0680932C0690930A
:105970002D0610E084E50E949D51882359F00E9475
:105980001D51609322067093230680932406909302
:105990002506D6C3112309F4D3C34091260650919E
:1059A000270660912806709129068DE995E00E94EE
:1059B0001DB740912A0650912B0660912C067091DC
:1059C0002D068AE995E00E941DB74091220650916C
:1059D0002306609124067091250687E995E00E94D0
:1059E0001DB78AE00E94B951ABC30E949D7BA8C33A
:1059F0004FE4C42E42E0D42E59E6E52E56E0F52EB3
:105A000010E0F60181916F010E945451882359F0F2
:105A10000E941D51D7016D937D938D939C93139795
:105A2000812F0E944C821F5FB4E0EB0EF11C1330FB
:105A300041F70C9468230E94187182C383E50E9489
:105A40009D51882309F47CC30E94ED50709303029A
:105A50006093020275C38DED90E00E948C828111EB
:105A60006FC383E50E949D51811103C0EFE6FEE103
:105A700039C000915C1010E00E94ED50000F111F22
:105A8000F801E35CFD4F7183608380915C1090E0CE
:105A90007C01EE0CFF1CEE0CFF1C8701095D1D4F05
:105AA000880F991FFC01E35CFD4F60817181072E17
:105AB000000C880B990B0E9493D52AE037ED43E246
:105AC0005CE30E94F2D5F701E65EFE4E2081318153
:105AD000428153810E94F2D5F801608371838283F1
:105AE00093832EC384918F010F5F1F4F882321F072
:105AF0000E94B951F801F6CF85E40E94B951809116
:105B00005C10805D0E94B951E0915C10F0E0EE0FF6
:105B1000FF1FE35CFD4F608171818DEA95E00E947B
:105B20003AB785E20E94B9518AE00E94B95108C390
:105B300080E50E945451882309F402C30E94ED506D
:105B40006B017C0183E50E949D51882321F00E9416
:105B5000ED508B0102C00FEF1FEFC80101960397B4
:105B600008F0EEC2D7FCECC22C2DE5EBF5E085EE9B
:105B700095E03491231709F4FEC231968E179F07E2
:105B8000C1F7FCC283E50E949D51882319F00E9451
:105B9000ED5002C064E071E079A368A380E50E9443
:105BA0009D51882339F00E94ED506938F3E17F0759
:105BB00030F402C068EE73E07A83698304C088E839
:105BC00093E19A838983BE01605E7F4FCE01019687
:105BD0000E9420C3B5C285E40E949D51811110C06E
:105BE00080E50E945451882391F00E941D516093DA
:105BF0004A1070934B1080934C1090934D1007C037
:105C00000E94FD50882361F3EAE5FEE171C089E45A
:105C10000E945451882381F00E941D512CEA35ECDA
:105C200047E25EE30E94F2D56093461070934710FE
:105C3000809348109093491084E40E945451882323
:105C400081F00E941D512CEA35EC47E25EE30E9490
:105C500093DA60934E1070934F108093501090938E
:105C60005110EFE6FEE184918F010F5F1F4F8823F3
:105C700021F00E94B951F801F6CF40914A1050919D
:105C80004B1060914C1070914D108DEE95E00E947C
:105C90001DB72CEA35EC47E25EE360914610709147
:105CA000471080914810909149100E9493DAAB01FF
:105CB000BC0189EE95E00E941DB72CEA35EC47E265
:105CC0005EE360914E1070914F1080915010909152
:105CD00051100E94F2D5AB01BC0185EE95E00E9407
:105CE0001DB78AE00E94B9512BC20E94B951F80138
:105CF00084918F010F5F1F4F8111F7CFE1EFF5E026
:105D000084918F010F5F1F4F882309F419C20E94ED
:105D1000B951F801F5CF83E50E945451182F88231B
:105D200071F00E941D510E94FBDA70932C02609367
:105D30002B0221E0672B09F020E020934A0680E542
:105D40000E945451882359F020912B0230912C024B
:105D5000232B11F00E940E5180934A06F1C11111BC
:105D6000EFC1EFE6FEE184918F010F5F1F4F8823A3
:105D700021F00E94B951F801F6CF80914A0688239C
:105D800019F063E173E002C066E173E088E196E038
:105D90000E9453B760912B0270912C0287E096E02D
:105DA0000E943AB7E3E0F6E084918F010F5F1F4F46
:105DB000882309F4C5C10E94B951F801F5CF0E94AA
:105DC0005E75BEC180E50E945451882351F00E9447
:105DD0001D51609342107093431080934410909330
:105DE000451089E40E945451882381F00E941D517E
:105DF0002CEA35EC47E25EE30E94F2D560933E1058
:105E000070933F10809340109093411084E40E945F
:105E10005451882381F00E941D512CEA35EC47E251
:105E20005EE30E9493DA60933A1070933B10809384
:105E30003C1090933D10EFE6FEE184918F010F5FDF
:105E40001F4F882321F00E94B951F801F6CF4091ED
:105E5000421050914310609144107091451083E3BB
:105E600096E00E941DB72CEA35EC47E25EE36091B4
:105E70003E1070913F1080914010909141100E940F
:105E800093DAAB01BC018FE296E00E941DB72CEAC9
:105E900035EC47E25EE360913A1070913B108091DF
:105EA0003C1090913D100E94F2D5AB01BC018BE2F9
:105EB00096E00E941DB78AE00E94B95141C10E943C
:105EC000B951F80184918F010F5F1F4F8111F7CFF6
:105ED000E7E3F6E084918F010F5F1F4F882309F4F9
:105EE0002FC10E94B951F801F5CF0E94717228C1EB
:105EF0000E949C8B25C10E94DBB422C183E50E94D5
:105F00005451882321F00E940E5191E089270E946C
:105F10006CB016C181E0809358060E949285109261
:105F20005806882309F40CC1EFE6FEE184918F0145
:105F30000F5F1F4F811103C0E6E4F6E004C00E942A
:105F4000B951F801F3CF84918F010F5F1F4F882360
:105F500009F4F6C00E94B951F801F5CF8091890A81
:105F6000882309F4EDC081E080938C0AE9C08AE5BA
:105F70000E949D51811103C0E4E5F6E00BC00E9430
:105F80001D516093261170932711809328119093CF
:105F90002911D6C084918F010F5F1F4F882321F0F4
:105FA0000E94B951F801F6CF409126115091271166
:105FB000609128117091291181E596E00E941DB72A
:105FC0008AE00E94B951BCC08BE40E949D518111AE
:105FD00003C0EFE6FEE136C08BE40E949D518823AA
:105FE000C1F00E941D516B017C0120E030E0A9014D
:105FF0000E94DDDB87FD0AC020E030E040E251E492
:10600000C701B6010E948DD5181634F4E3E7F6E017
:106010000EC0C12CD12C76010E940871C0921E06C0
:10602000D0921F06E0922006F092210689C084914A
:106030008F010F5F1F4F882309F482C00E94B9515E
:10604000F801F5CF84918F010F5F1F4F882321F056
:106050000E94B951F801F6CF40911E0650911F06DB
:10606000609120067091210682E996E00E941DB79A
:106070008AE00E94B95164C081E08093350283E5D3
:106080000E949D51882339F00E940E51811158C001
:106090000E94BD6055C083E50E945451F7CF0E9415
:1060A00054C34EC0F09034180E9408711091FD172F
:1060B00080E00E94E880FF2029F1EFE6FEE1849174
:1060C0008F010F5F1F4F882321F00E94B951F80103
:1060D000F6CF84E50E94B9516F2D70E080E090E02A
:1060E0004AE00E94DB5480E20E94B951EFEAF6E0F8
:1060F00084918F010F5F1F4F882311F10E94B951C6
:10610000F801F6CF1092C405812F0E94E880EFE6D7
:10611000FEE184918F010F5F1F4F882321F00E94C1
:10612000B951F801F6CF6091C40570E08DE996E0B1
:106130000E943AB78AE00E94B95102C00E9454C33B
:106140001092C5050E94A06055C00E94687F0E9401
:10615000C85CF6CF0E94ED50AB01BC014093030D2B
:106160005093040D6093050D7093060D82E59CE03D
:106170000E94CAA1E5CF0E9413CAE2CF0E94087113
:10618000BC2C60E08C2D0E94C7C30F3F2FEF12077D
:1061900059F48C2D0E9471C331E020E0892B09F065
:1061A00030E0032F122F05C00130110559F401E032
:1061B00010E08B2D0E9471C38017910709F20E9495
:1061C0005258F7CF00E010E0F4CF61E0812F0E9439
:1061D000C7C36E2D812F0E9499C3F12CB701812F67
:1061E0000E9403C4193009F0ABCFF0923A04E09258
:1061F0003904A6CFCC55DF4F0FB6F894DEBF0FBEE3
:10620000CDBFDF91CF911F910F91FF90EF90DF9065
:10621000CF90BF90AF909F908F907F906F905F9046
:106220004F903F902F9008952F923F924F925F9200
:106230006F927F928F929F92AF92BF92CF92DF9296
:10624000EF92FF920F931F93CF93DF93CDB7DEB7FB
:106250006F970FB6F894DEBF0FBECDBFC09043045A
:10626000D0904404E0904504F090460420E030E0F3
:1062700040EA50E4C701B6010E948DD587FD19C1DF
:1062800020E030E041E953E4C701B6010E94DDDBC4
:1062900018160CF40EC11092A60E1092A50E809145
:1062A00009014091A40E042E000C550B817021E0D1
:1062B000822790E04817590709F433C080910901FB
:1062C000817028272093A40E81111BC00E94AC92DC
:1062D000EFEBFCE084918F01882351F0082E000C35
:1062E000990B0E94A7920F5F1F4FF8018491F4CF82
:1062F0008DE090E00E94A7928AE090E00E94A79231
:1063000010C0E3ECFCE084918F01882389F3082E10
:10631000000C990B0E94A7920F5F1F4FF801849108
:10632000F4CF8091970E833009F44CC02CF488236D
:1063300051F08130D9F072C0843009F43EC085300C
:1063400009F44DC06BC08091890A882309F466C0A6
:1063500081E08093970E0E9402C560939B0E70931C
:106360009C0E80939D0E90939E0E58C08091890A3A
:10637000811154C08091550C882321F082E08093D4
:10638000970E4CC01092970EEBEBFCE084918F01BE
:10639000882351F0082E000C990B0E94A7920F5FE2
:1063A0001F4FF8018491F4CF8DE090E00E94A792F6
:1063B0008AE090E00E94A79231C08091E40E882389
:1063C000E9F22CC08091890A811128C080910B0AC2
:1063D00090910C0A891B8F7009F496C01FC08091A0
:1063E000890A81111BC080910B0A90910C0A891BAC
:1063F0008F7009F4ABC012C08DE090E00E94A792AC
:106400008AE090E00E94A7921092970E8BE99CE0A0
:106410009093FC078093FB070E94E55180918C0EBE
:1064200090918D0E03974CF57FEC272E78E0372E58
:10643000E0E68E2EEAEE9E2EA12CB12C82EF9FE09C
:106440000E94C64C18161906C4F480918C0E9091C7
:106450008D0E049794F482EF9FE00E948A4C809303
:10646000920EE091930EF091940E8A3019F08D30D7
:1064700009F07DC0309709F083C080918C0E909117
:106480008D0E009711F40C94A040019790938D0EFF
:1064900080938C0E80918E0E90918F0E019664E009
:1064A00070E00E94A0DC90938F0E80938E0E0C946F
:1064B000A0408091A50E9091A60E8136FAEE9F071E
:1064C000E8F01092A60E1092A50EE7ECFCE0849185
:1064D0008F01882351F0082E000C990B0E94A7927F
:1064E0000F5F1F4FF8018491F4CF8DE090E00E9480
:1064F000A7928AE090E00E94A792D1CE0196909355
:10650000A60E8093A50ECBCE87EA9CE09093FC0765
:106510008093FB070E94E5518091E40E882311F0DF
:1065200082E001C084E08093970EE3EAFCE084916E
:106530008F01882309F438CF082E000C990B0E9494
:10654000A7920F5F1F4FF8018491F3CFEFE9FCE0B2
:1065500084918F01882309F44FCF082E000C990BEA
:106560000E94A7920F5F1F4FF8018491F3CF8A33E7
:1065700009F480CFEF35F10514F40C94343E7ACF52
:106580008091900E9091910E20E6289F7001299F96
:10659000F00C11248701045F124FE00FF11F1082ED
:1065A00061E470E0C8010E9423DD009711F40C94AF
:1065B000183E9093960E8093950E801B910B8E0D36
:1065C0009F1D60E070E0835F924F0E948ED10E9419
:1065D000FBDACB01770FAA0BBB0B8232910510F0CF
:1065E0000C94183EFC018827EE58FF4F8F4F0C94F7
:1065F000CFDCE6E9FCE084918F01882351F0082E7E
:10660000000C990B0E94A7920F5F1F4FF801849115
:10661000F4CF20E030E040E05FE36091430470910C
:10662000440480914504909146041EC0E1E9FCE0D9
:1066300084918F01882351F0082E000C990B0E9441
:10664000A7920F5F1F4FF8018491F4CF609141042E
:1066500070914204072E000C880B990B0E9493D571
:1066600020E030E040E05FE30E94B7D90E94FBDA0F
:10667000CB010E94FB550E94A2C78DE090E00E94D2
:10668000A7928AE090E00E94A7920C94183EECE852
:10669000FCE084918F01882351F0082E000C990BA7
:1066A0000E94A7920F5F1F4FF8018491F4CF20E062
:1066B00030E040E05FE360913D0470913E048091E2
:1066C0003F0490914004D0CFE7E8FCE084918F0133
:1066D000882351F0082E000C990B0E94A7920F5F9F
:1066E0001F4FF8018491F4CF60913B0470913C04FA
:1066F000B1CF2091390430913A0444E6429FC00161
:10670000439F900D11246FEF70E00E94A0DC8B017D
:106710006536710510F004E610E0E2E8FCE08491D3
:106720007F01882359F0082E000C990B0E94A79234
:10673000FFEFEF1AFF0AF7018491F3CFB80180E071
:1067400090E041C7EEE7FCE084918F01882351F08F
:10675000082E000C990B0E94A7920F5F1F4FF801A3
:106760008491F4CF80E290E00E94A792EAE7FCE0F7
:1067700084918F01882351F0082E000C990B0E9400
:10678000A7920F5F1F4FF8018491F4CF6091290405
:1067900070912A0480912B0490912C040E94A3C72D
:1067A00080E290E00E94A792E6E7FCE084918F01EE
:1067B000882351F0082E000C990B0E94A7920F5FBE
:1067C0001F4FF8018491F4CF60912D0470912E0435
:1067D00080912F04909130040E94A3C780E290E042
:1067E0000E94A792E2E7FCE084918F01882351F098
:1067F000082E000C990B0E94A7920F5F1F4FF80103
:106800008491F4CF6091310470913204809133040B
:10681000909134040E94A3C780E290E0A0C58091CB
:10682000890A882309F450C0EDE6FCE084918F01C9
:10683000882351F0082E000C990B0E94A7920F5F3D
:106840001F4FF8018491F4CF80918A0A882359F16F
:106850008091550C882329F18091FF0C9091000DB7
:10686000A091010DB091020D0097A105B105C1F0F5
:10687000BC01CD016D597F4F8F4F9F4F24E630E013
:1068800040E050E00E947BD96091030D7091040DAF
:106890008091050D9091060D0E947BD9822F01C039
:1068A00080E090E0E6CEE9E6FCE084918F01882369
:1068B00009F4E3CE082E000C990B0E94A7920F5FFB
:1068C0001F4FF8018491F3CFE1E6FCE084918F0142
:1068D000882309F4D2CE082E000C990B0E94A792AF
:1068E0000F5F1F4FF8018491F3CFECE5FCE084913A
:1068F0008F01882351F0082E000C990B0E94A7925B
:106900000F5F1F4FF8018491F4CF80919B0E9091FF
:106910009C0EA0919D0EB0919E0E892B8A2B8B2BE5
:1069200009F477C00E9402C5A50194010E947BD999
:1069300069017A0160919B0E70919C0E80919D0E71
:1069400090919E0EA50194010E947BD98601021BA5
:10695000130BC8016CE370E00E948CDCCB0199271B
:10696000EAE0F0E0BF010E94A0DC282FCB01BF01CC
:106970000E94A0DC805D80932004205D2093210490
:106980001092220480E294E00E94A2C780E290E08C
:106990000E94A792EAE5FCE084917F01882359F0E8
:1069A000082E000C990B0E94A792FFEFEF1AFF0A26
:1069B000F7018491F3CF80E290E00E94A792C80192
:1069C0006CE370E00E948CDC6AE070E00E94A0DC66
:1069D000605D60932004805D809321041092220406
:1069E00080E294E00E94A2C780E290E00E94A79219
:1069F000E8E5FCE084918F01882309F43ECE082E5F
:106A0000000C990B0E94A7920F5F1F4FF801849111
:106A1000F3CF80E290E00E94A792E0E5FCE0849151
:106A20008F01882309F429CE082E000C990B0E94AF
:106A3000A7920F5F1F4FF8018491F3CF1092C50EFC
:106A40008091090180FF11C0ECE4FCE084918F018A
:106A5000882309F412CE082E000C990B0E94A792ED
:106A60000F5F1F4FF8018491F3CF83E50E943EC76B
:106A7000882341F00E9459C70E9400DB70939A0E50
:106A80006093990EE8E4FCE084918F01882351F033
:106A9000082E000C990B0E94A7920F5F1F4FF80160
:106AA0008491F4CF8DE090E00E94A7928AE090E07C
:106AB0000E94A7928091E30E882309F442C280913C
:106AC000990E90919A0E8430910509F4C8C08830CF
:106AD000910509F47DC1892B09F0E7C3ECE6FAE0E2
:106AE00084918F01882351F0082E000C990B0E948D
:106AF000A7920F5F1F4FF8018491F4CF8DE090E0D3
:106B00000E94A7928AE090E00E94A792E1E6FAE054
:106B100084918F01882351F0082E000C990B0E945C
:106B2000A7920F5F1F4FF8018491F4CF8DE090E0A2
:106B30000E94A7928AE090E00E94A792E5E5FAE021
:106B400084918F01882351F0082E000C990B0E942C
:106B5000A7920F5F1F4FF8018491F4CF8DE090E072
:106B60000E94A7928AE090E00E94A792E9E4FAE0EE
:106B700084918F01882351F0082E000C990B0E94FC
:106B8000A7920F5F1F4FF8018491F4CF8DE090E042
:106B90000E94A7928AE090E00E94A792EBE3FAE0BD
:106BA00084918F01882351F0082E000C990B0E94CC
:106BB000A7920F5F1F4FF8018491F4CF8DE090E012
:106BC0000E94A7928AE090E00E94A792EDE2FAE08C
:106BD00084918F01882351F0082E000C990B0E949C
:106BE000A7920F5F1F4FF8018491F4CF8DE090E0E2
:106BF0000E94A7928AE090E00E94A792E0E2FAE069
:106C000084918F01882351F0082E000C990B0E946B
:106C1000A7920F5F1F4FF8018491F4CF8DE090E0B1
:106C20000E94A7928AE090E00E94A792E3E1FAE036
:106C300084918F01882351F0082E000C990B0E943B
:106C4000A7920F5F1F4FF8018491F4CF8DE090E081
:106C50000E94A7928AE090E00E94A79226C3E5E0F6
:106C6000FAE084918F01882351F0082E000C990BD3
:106C70000E94A7920F5F1F4FF8018491F4CF8DE01F
:106C800090E00E94A7928AE090E00E94A792E7EF2E
:106C9000F9E084918F01882351F0082E000C990BA4
:106CA0000E94A7920F5F1F4FF8018491F4CF8DE0EF
:106CB00090E00E94A7928AE090E00E94A792E1EE05
:106CC000F9E084918F01882351F0082E000C990B74
:106CD0000E94A7920F5F1F4FF8018491F4CF8DE0BF
:106CE00090E00E94A7928AE090E00E94A792EBECCD
:106CF000F9E084918F01882351F0082E000C990B44
:106D00000E94A7920F5F1F4FF8018491F4CF8DE08E
:106D100090E00E94A7928AE090E00E94A792E9EB9F
:106D2000F9E084918F01882351F0082E000C990B13
:106D30000E94A7920F5F1F4FF8018491F4CF8DE05E
:106D400090E00E94A7928AE090E00E94A792E7EA72
:106D5000F9E084918F01882351F0082E000C990BE3
:106D60000E94A7920F5F1F4FF8018491F4CF8DE02E
:106D700090E00E94A7928AE090E00E94A792E9E941
:106D8000F9E084918F01882351F0082E000C990BB3
:106D90000E94A7920F5F1F4FF8018491F4CF8DE0FE
:106DA00090E00E94A7928AE090E00E94A792EBE810
:106DB000F9E084918F01882309F448CF082E000C54
:106DC000990B0E94A7920F5F1F4FF8018491F3CF98
:106DD000E4E8F9E084918F01882351F0082E000C3B
:106DE000990B0E94A7920F5F1F4FF8018491F4CF77
:106DF0008DE090E00E94A7928AE090E00E94A79226
:106E0000EDE7F9E084918F01882351F0082E000C02
:106E1000990B0E94A7920F5F1F4FF8018491F4CF46
:106E20008DE090E00E94A7928AE090E00E94A792F5
:106E3000E6E6F9E084918F01882351F0082E000CDA
:106E4000990B0E94A7920F5F1F4FF8018491F4CF16
:106E50008DE090E00E94A7928AE090E00E94A792C5
:106E6000EFE4F9E084918F01882351F0082E000CA3
:106E7000990B0E94A7920F5F1F4FF8018491F4CFE6
:106E80008DE090E00E94A7928AE090E00E94A79295
:106E9000E8E3F9E084918F01882351F0082E000C7B
:106EA000990B0E94A7920F5F1F4FF8018491F4CFB6
:106EB0008DE090E00E94A7928AE090E00E94A79265
:106EC000E1E2F9E084918F01882351F0082E000C53
:106ED000990B0E94A7920F5F1F4FF8018491F4CF86
:106EE0008DE090E00E94A7928AE090E00E94A79235
:106EF000E3E1F9E084918F01882351F0082E000C22
:106F0000990B0E94A7920F5F1F4FF8018491F4CF55
:106F10008DE090E00E94A7928AE090E00E94A79204
:106F2000E5E0F9E084918F01882309F48FCE082EE3
:106F3000000C990B0E94A7920F5F1F4FF8018491DC
:106F4000F3CF80918A0A882309F486C181E0809377
:106F5000070D1092090D1092080D89ED9AE00E941C
:106F600011A48BE1E9EDFAE0DE01159601900D9296
:106F70008A95E1F78091D70A9091D80A9C838B83F8
:106F800085EE92E09A83898340E050E0BE016F5F16
:106F90007F4F80E090E00E94DD94CE0101960E9438
:106FA000EB57C090080DD090090D0091990E1091EB
:106FB0009A0EC601801B910B049720F06801F3E044
:106FC000CF0ED11C56EF452E58E0552E67EE662E9B
:106FD00068E0762EC016D10608F467C101151105C8
:106FE00009F0A1C06DE87AE089ED9AE00E94D9A28B
:106FF0006AE173E08DE89AE00E942EDD892B09F0AA
:107000004AC0F201849146EFE42E48E0F42E882332
:1070100059F0082E000C990B0E94A792FFEFEF1A6F
:10702000FF0AF7018491F3CF8DE090E00E94A792D0
:107030008AE090E00E94A792F301849137EEE32E5C
:1070400038E0F32E882359F0082E000C990B0E948B
:10705000A792FFEFEF1AFF0AF7018491F3CF8DE0BB
:1070600090E00E94A7928AE090E00E94A7924AE0F6
:1070700060E070E0CB010E94DB54E7EDF8E0849122
:107080007F012FEFE21AF20A882309F4E2C00E947E
:10709000B951F701F4CFE3EDF8E084917F01882343
:1070A00059F0082E000C990B0E94A792FFEFEF1ADF
:1070B000FF0AF7018491F3CF8DE090E00E94A79240
:1070C0008AE090E00E94A792F10184912FECE22ED9
:1070D00028E0F22E882359F0082E000C990B0E940C
:1070E000A792FFEFEF1AFF0AF7018491F3CF8DE02B
:1070F00090E00E94A7928AE090E00E94A7924AE066
:1071000060E070E0CB010E94DB54EAECF8E084918F
:107110007F012FEFE21AF20A882309F49AC00E9435
:10712000B951F701F4CF60E070E0C80101970E9407
:10713000A39680918B0A882309F45FC0E8ECF8E0FD
:1071400084917F01882359F0082E000C990B0E942E
:10715000A792FFEFEF1AFF0AF7018491F3CF8DE8B2
:107160009AE00E94A2C78DE090E00E94A7928AE078
:1071700090E00E94A792E6ECF8E084917F018823DA
:1071800059F0082E000C990B0E94A792FFEFEF1AFE
:10719000FF0AF7018491F3CF8AE99AE00E94A2C71F
:1071A0008DE090E00E94A7928AE090E00E94A79272
:1071B000C801A0E0B0E04AE0BC01CD010E94DB5470
:1071C000E4ECF8E084917F012FEFE21AF20A8823C1
:1071D00021F00E94B951F701F5CF9AE9E92E9AE022
:1071E000F92EF70181917F01882319F00E94B9518E
:1071F000F8CF8AE00E94B9512CC08DE89AE00E9435
:10720000A2C78DE090E00E94A7928AE090E00E94E1
:10721000A7928AE99AE00E94A2C78DE090E00E94BE
:10722000A7928AE090E00E94A792C801A0E0B0E097
:107230004AE0BC01CD010E94DB548AE9E82E8AE0D5
:10724000F82EF70181917F01882399F20E94B951AC
:10725000F8CF0F5F1F4FBECEE5EBF8E084918F01B2
:10726000882351F0082E000C990B0E94A7920F5F03
:107270001F4FF8018491F4CF8DE090E00E94A79217
:107280008AE090E00E94A792E6EAF8E084918F01FC
:10729000882309F4DBCC082E000C990B0E94A792DE
:1072A0000F5F1F4FF8018491F3CFE4E4FCE0849179
:1072B0008F01882309F4E1C9082E000C990B0E9464
:1072C000A7920F5F1F4FF8018491F3CF8091890A35
:1072D000882339F00E940F94ABC48091890A8823D7
:1072E000E9F00E9487C1A4C48091970E823019F002
:1072F000833609F09DC40E94EE93E0E4FCE08491A3
:107300008F01882309F4B9C9082E000C990B0E943B
:10731000A7920F5F1F4FF8018491F3CF8091970ED2
:10732000833609F085C4DDCF87E39CE00E940D58C9
:1073300080910B0A90910C0A891B8F7009F078C418
:107340008091970E823009F473C4833609F0A4C487
:107350006FC48DE090E00E94A7928AE090E00E94C6
:10736000A7928BC980910B0A90910C0A891B8F7090
:1073700009F05EC48091970E823009F459C48336B7
:1073800009F456C48091550C8111DAC451C483E5C7
:107390000E943EC7811126C083E40E943EC7882315
:1073A00009F446C480910B0A90910C0A891B8F70D6
:1073B00009F03EC420E030E040E251E46091310445
:1073C0007091320480913304909134040E948DD5E1
:1073D00087FF08C084E29CE09093FC078093FB0742
:1073E0000E94E5510E9459C720E030E0A9010E94A7
:1073F0008DD587FD10C00E9459C720E030E849E8CC
:1074000053E40E94DDDB18164CF00E9459C70E941D
:1074100000DBCB0105C080E090E002C083E191E099
:107420000E94459105C483E50E943EC7882309F464
:10743000FFC30E9459C720E030E0A9010E948DD50A
:1074400087FD11C00E9459C720E030E046E153E4B7
:107450000E94DDDB18164CF00E9459C70E9400DB29
:10746000362F272F04C030E001C036E920E0832FFB
:10747000922F8E36910514F08EE690E090933C04A6
:1074800080933B040E941F99D3C383E50E943EC7AB
:107490008823D9F00E9459C720E030E04FE753E439
:1074A0000E94F2D520E030E048EC52E40E9493DAEA
:1074B0000E9400DB6F3F710519F010F06FEF70E074
:1074C00070933A0460933904D8C88FEF90E090939A
:1074D0003A0480933904D1C880910B0A90910C0A28
:1074E000891B8F7009F0C9C88091890A8111C5C8AC
:1074F0000E9422755F9A809128048E7F80932804D1
:107500008A9A479A809128048D7F809328048091DD
:1075100008018095817080930601479A8091280424
:107520008B7F80932804129AA8C883E50E943EC7E7
:10753000882319F10E9459C720E030E040E252E46C
:107540000E948DD587FD0FC00E9459C720E030EC06
:1075500049E754E40E94DDDB181644F00E9459C745
:107560000E94FBDA05C068E270E002C067EE73E0DB
:1075700070930302609302025BC3EEE1FCE084912E
:107580008F01882351F0082E000C990B0E94A792BE
:107590000F5F1F4FF8018491F4CFC0900202D0908A
:1075A00003020D2C000CEE08FF08F7FE0EC06DE282
:1075B00082EF9FE00E943D4C66277727CB016C1934
:1075C0007D098E099F094AE003C04AE0C701B60160
:1075D0000E9462C752C880910B0A90910C0A891BC5
:1075E0008F7009F025C38091970E823009F420C373
:1075F000833609F0EBC21CC380910B0A90910C0AF0
:10760000891B8F7009F039C88091970E823009F478
:1076100034C8833609F0B6C330C880910B0A909104
:107620000C0A891B8F7009F003C38091970E82307A
:1076300009F4FEC2833609F0FBC4FAC280910B0A3A
:1076400090910C0A891B8F7009F0F2C28091970EFD
:10765000823009F4EDC2833609F020C5E9C2809179
:107660000B0A90910C0A891B8F7009F0E1C280917E
:10767000970E823009F4DCC2833609F045C5D8C2C2
:107680008091C50E811103C00E94AC92C4C18E329C
:1076900071F58091C60E8E3209F046C180912A0C98
:1076A000882309F4B8C1815080932A0C882361F0A3
:1076B00090E001974FE1489F9001499F300D1124C0
:1076C000C9018C50954F02C086EB9AE02BE1FC017A
:1076D0003496A9EDBAE001900D922A95E1F7FC01EC
:1076E000828193819093D80A8093D70A94C18C3376
:1076F00009F01AC16CE173E085EC9EE00E942EDD7A
:10770000892B21F481E08093E30E85C16BE273E065
:1077100085EC9EE00E942EDD892B79F4E2E8F8E00A
:1077200084918F010F5F1F4F882321F00E94B95170
:10773000F801F6CF8FE698E0E4C062E473E085ECF0
:107740009EE00E942EDD892B79F4EBE4F8E0849131
:107750008F010F5F1F4F882321F00E94B951F8015C
:10776000F6CF88E398E0CDC069E573E085EC9EE054
:107770000E942EDD892B79F4EDE1F8E084918F01F0
:107780000F5F1F4F882321F00E94B951F801F6CFF7
:1077900088E198E0B6C067E673E085EC9EE00E9461
:1077A0002EDD892B79F4EDEFF7E084918F010F5FE7
:1077B0001F4F882321F00E94B951F801F6CF88EFBE
:1077C00097E09FC065E773E085EC9EE00E942EDDA8
:1077D000892B79F4EDEDF7E084918F010F5F1F4F56
:1077E000882321F00E94B951F801F6CF84ED97E08B
:1077F00088C063E873E085EC9EE00E942EDD892B53
:1078000071F401EB17E0F8018491882329F00F5FF0
:107810001F4F0E94B951F7CF8AEA97E072C069E919
:1078200073E085EC9EE00E942EDD892B79F4EBE875
:10783000F7E084918F010F5F1F4F882321F00E9492
:10784000B951F801F6CF84E897E05BC06BEA73E0CA
:1078500085EC9EE00E942EDD892B79F4ECE6F7E0C2
:1078600084918F010F5F1F4F882321F00E94B9512F
:10787000F801F6CF8BE597E044C066EB73E085EC4A
:107880009EE00E942EDD892B79F4E2E4F7E08491FA
:107890008F010F5F1F4F882321F00E94B951F8011B
:1078A000F6CF80E397E02DC062EC73E085EC9EE0BC
:1078B0000E942EDD892B79F4E5E1F7E084918F01B8
:1078C0000F5F1F4F882321F00E94B951F801F6CFB6
:1078D00083E097E016C060ED73E085EC9EE00E94C7
:1078E0002EDD892BA9F4E9EEF6E084918F010F5F7C
:1078F0001F4F882321F00E94B951F801F6CF87ED80
:1079000096E09093FC078093FB070E94E55183C0AB
:107910006DED73E085EC9EE00E942EDD892B09F071
:107920007AC01092E30E77C01D8218861C821B82DB
:1079300085EE92E09A8389838091DC0A811103C0ED
:1079400066EB7AE002C065ED7AE06115710519F029
:107950006C5F7F4F02C060E070E021E045EC5EE0CC
:10796000CE0105960E9447A8882361F18BE1FE01B4
:107970003596A9EDBAE001900D928A95E1F72B8139
:107980003C813093D80A2093D70A80912A0C8A3000
:1079900008F03DC091E0980F90932A0CFFE18F9F73
:1079A000C0011124DC01A850B54F4BE1E9EDFAE02C
:1079B00001900D924A95E1F7FC01EC50F54F3383AD
:1079C000228325C0EFE6FEE184918F010F5F1F4FF8
:1079D000882321F00E94B951F801F6CFE1ECF6E0DE
:1079E00084918F010F5F1F4F882321F00E94B951AE
:1079F000F801F6CF05EC1EE0F80181918F01882394
:107A000019F00E94B951F8CF8AE00E94B951CE0115
:107A100001960E94EB571092C50E8091090180FFDC
:107A200007C1E2E6FBE084918F01882311F40C94F6
:107A30003D33082E000C990B0E94A7920F5F1F4F39
:107A4000F8018491F2CF8FE40E943EC781110C941B
:107A50003D3383E40E943EC70C943D3383E50E948E
:107A60003EC7811159C08FE40E943EC7882319F098
:107A70008AE29BE007C084E50E943EC7882349F064
:107A800082E09BE09093FC078093FB070E94E55106
:107A900043C083E40E943EC7882319F089ED9AE031
:107AA000F1CF81E50E943EC7882319F081EB9AE06F
:107AB000E9CF88E40E943EC78823C9F0EDEAFAE0E6
:107AC00084918F01882351F0082E000C990B0E949D
:107AD000A7920F5F1F4FF8018491F4CF8DE090E0E3
:107AE0000E94A7928AE090E00E94A79215C08CE4C1
:107AF0000E943EC7882381F0E9EAFAE084918F0171
:107B0000882361F3082E000C990B0E94A7920F5F47
:107B10001F4FF8018491F4CFE1E7FBE084918F01DE
:107B2000882311F40C943D33082E000C990B0E940D
:107B3000A7920F5F1F4FF8018491F2CF80910B0A3B
:107B400080910C0A0C943D3383E50E943EC7882344
:107B500009F46EC081E89AE09093FC078093FB07DC
:107B60000E94E551E1E7FBE084918F01882311F445
:107B70000C943D33082E000C990B0E94A7920F5FC6
:107B80001F4FF8018491F2CFECE7FAE084918F0166
:107B9000882351F0082E000C990B0E94A7920F5FCA
:107BA0001F4FF8018491F4CFE7E7FAE084918F0149
:107BB000882311F40C943D33082E000C990B0E947D
:107BC000A7920F5F1F4FF8018491F2CF88E50E94C2
:107BD0003EC7811106C089E50E943EC7882309F48B
:107BE000C3C088E50E943EC7882341F088E19CE03D
:107BF0009093FC078093FB070E94E55189E50E9462
:107C00003EC7882341F082E19CE09093FC0780937B
:107C1000FB070E94E5518AE50E943EC7882341F098
:107C20008CE09CE09093FC078093FB070E94E55159
:107C30008091900E9091910E019664E070E00E9408
:107C4000A0DC9093910E8093900E80918C0E909179
:107C50008D0E019690938D0E80938C0E1092940E43
:107C60001092930E0C941E324091900E5091910EF2
:107C70009F012F5F3F4F3093940E2093930E90E619
:107C8000949F9001959F300D1124245F324FE20F95
:107C9000F31F80830C941E320091950E1091960E66
:107CA000780124E0E20EF11C6AE270E0C7010E9454
:107CB00023DDF80124812F3221F4B8016B5F7F4F5F
:107CC00003C02C3339F4B70185EC9EE00E9437DD08
:107CD0000C943D331092C50E009719F0FC013197BA
:107CE00010828091950E9091960E40E061E004968E
:107CF0000E946AC58091550C882389F0E3E3FCE07B
:107D000084918F01882309F424CB082E000C990B51
:107D10000E94A7920F5F1F4FF8018491F3CFEFE20B
:107D2000FCE084918F01882309F413CB082E000C0A
:107D3000990B0E94A7920F5F1F4FF8018491F3CF18
:107D40000E94EE93EBE2FCE084918F01882311F412
:107D50000C943D33082E000C990B0E94A7920F5FE4
:107D60001F4FF8018491F2CF8AE50E943EC781112E
:107D700038CF83E40E943EC7882309F459CF88E0B6
:107D80009CE050CF86E40E943EC7882309F44DC191
:107D90000E9459C70E9400DB8B0184E09CE0909315
:107DA000FC078093FB070E94E55188E50E943EC7CF
:107DB000882309F451C00E9459C72B013C012DECC6
:107DC0003CEC4CE45EE30E948DD59E012F5F3F4F5B
:107DD0007901181674F020E030E0A901C301B20166
:107DE0000E94DDDB18162CF41F930F9389EF9BE0A4
:107DF00005C12DEC3CEC4CEC5DEBC301B2010E94E3
:107E00008DD518167CF020E030E040E85FEBC30130
:107E1000B2010E94DDDB18162CF41F930F938DEE38
:107E20009BE0ECC01F930F93C301B2010E94FBDAE9
:107E30007F936F9383EE9BE09F938F93FF92EF92DC
:107E40000E945FD50FB6F894DEBF0FBECDBFCE0146
:107E500001960E94C051DFC089E50E943EC7882379
:107E600009F441C00E9459C72B013C012DEC3CECA8
:107E70004CE45EE30E948DD5FE0131967F01181619
:107E800074F020E030E0A901C301B2010E94DDDB03
:107E900018162CF41F930F9388ED9BE0AFC02DECC8
:107EA0003CEC4CEC5DEBC301B2010E948DD5181681
:107EB0007CF020E030E040E85FEBC301B2010E94BB
:107EC000DDDB18162CF41F930F938CEC9BE096C00F
:107ED0001F930F93C301B2010E94FBDA7F936F934C
:107EE00082EC9BE0A9CF8AE50E943EC7882309F473
:107EF00041C00E9459C72B013C012DEC3CEC4CE4E5
:107F00005EE30E948DD5FE0131967F01181674F054
:107F100020E030E0A901C301B2010E94DDDB1816A8
:107F20002CF41F930F9387EB9BE068C02DEC3CEC87
:107F30004CEC5DEBC301B2010E948DD518167CF0AC
:107F400020E030E040E85FEBC301B2010E94DDDBDE
:107F500018162CF41F930F938BEA9BE04FC01F93CE
:107F60000F93C301B2010E94FBDA7F936F9381EA02
:107F70009BE062CF85E40E943EC7882309F44BC092
:107F80000E9459C72B013C012DEC3CEC4CE45EE314
:107F90000E948DD5FE0131967F01181674F020E005
:107FA00030E0A901C301B2010E94DDDB18162CF4F8
:107FB0001F930F9386E99BE021C02DEC3CEC4CEC29
:107FC0005DEBC301B2010E948DD518167CF020E054
:107FD00030E040E85FEBC301B2010E94DDDB181620
:107FE0002CF41F930F938AE89BE008C0C301B201F1
:107FF0000E94FBDA7F936F938FE79BE09F938F93B1
:10800000FF92EF920E945FD50F900F900F900F900C
:108010000F900F901CCF8BE79BE09093FC07809311
:10802000FB070E94E5510C943D3300E010E0B5CE13
:1080300020E030E040E251E460913104709132047C
:1080400080913304909134040E948DD587FF08C03D
:1080500084E79BE09093FC078093FB070E94E55127
:1080600082E390E090933C0480933B040E941F992C
:1080700088EC90E00E944591E1E7FBE084918F015C
:10808000882311F40C943D33082E000C990B0E94A8
:10809000A7920F5F1F4FF8018491F2CF20E030E0EC
:1080A00040E251E4609131047091320480913304D4
:1080B000909134040E948DD587FF08C08AE69BE02A
:1080C0009093FC078093FB070E94E55180E590E0C8
:1080D00090933C0480933B040E941F9980EF90E0B2
:1080E0000E944591E1E7FBE084918F01882311F420
:1080F0000C943D33082E000C990B0E94A7920F5F41
:108100001F4FF8018491F2CF80E090E00E944591EA
:1081100010923C0410923B040E941F99E6E6FBE09B
:1081200084918F01882311F40C943D33082E000CA8
:10813000990B0E94A7920F5F1F4FF8018491F2CF15
:108140006F960FB6F894DEBF0FBECDBFDF91CF9113
:108150001F910F91FF90EF90DF90CF90BF90AF9065
:108160009F908F907F906F905F904F903F902F9057
:1081700008952F923F924F925F926F927F928F92CB
:108180009F92AF92BF92CF92DF92EF92FF920F93A6
:108190001F93CF93DF93CDB7DEB762970FB6F894F6
:1081A000DEBF0FBECDBFF8948FEF9FEF9093890095
:1081B000809388002AE02A8B212C312C789480919E
:1081C000990490919A04A0919B04B0919C04892BEE
:1081D0008A2B8B2B09F00FC2809118108823E1F0B5
:1081E000109218108091161090911710892B09F495
:1081F00002C2109251041092171010921610909112
:108200000B0A80910C0A981709F4F5C180910C0AA9
:108210008F5F8F7080930C0A8091161090911710C9
:10822000892B09F4E8C1409195045091960460911E
:108230009704709198048091910490919204A09178
:108240009304B09194040091880410E020E030E0A1
:10825000841B950BA60BB70B081719072A073B07BA
:1082600010F4D901C801E82F840F951FA61FB71F6E
:108270008093950490939604A0939704B0939804E8
:108280002091840030918500245E3F4F40916D0421
:1082900050916E0460916F047091700480915D0440
:1082A00090915E04A0915F04B0916004840F951FCB
:1082B000A61FB71F80936D0490936E04A0936F0464
:1082C000B0937004B7FD1CC0889A809125109091DE
:1082D0002610A0912710B091281040910402042E7E
:1082E000000C550B660B770B840F951FA61FB71F4D
:1082F0008093251090932610A0932710B0932810F8
:1083000040917104509172046091730470917404EF
:108310008091610490916204A0916304B09164041F
:10832000840F951FA61FB71F80937104909372044A
:10833000A0937304B0937404B7FD1CC08E9A80910F
:10834000291090912A10A0912B10B0912C104091DF
:108350000502042E000C550B660B770B840F951F3E
:10836000A61FB71F8093291090932A10A0932B105B
:10837000B0932C104091750450917604609177046D
:10838000709178048091650490916604A0916704CF
:10839000B0916804840F951FA61FB71F80937504C2
:1083A00090937604A0937704B0937804B7FD3FC010
:1083B00080914B04F09106028823C9F08091490412
:1083C00082FF02C0F7FD06C080914804882311F4A3
:1083D0000C94634A8091490490914A0493FF02C02F
:1083E000F7FD0CC080914704811108C006C0809140
:1083F0000B018095887080930901419A40912D105E
:1084000050912E1060912F10709130108F2FFF0F10
:10841000990BAA0BBB0B840F951FA61FB71F809348
:108420002D1090932E10A0932F10B09330104091E8
:10843000790450917A0460917B0470917C0480915E
:10844000690490916A04A0916B04B0916C04840F4C
:10845000951FA61FB71F8093790490937A04A09369
:108460007B04B0937C04B7FD3AC040913110509129
:1084700032106091331070913410C09007020C2CB0
:10848000000CDD08EE08FF084C0D5D1D6E1D7F1D04
:108490004093311050933210609333107093341026
:1084A0004091590450915A0460915B0470915C04AE
:1084B000841B950BA60BB70B8093790490937A04D9
:1084C000A0937B04B0937C0490914C04809186042B
:1084D00093FF02C0815001C08F5F8093860480911A
:1084E0006D0490916E04A0916F04B0917004B7FD7B
:1084F00015C04091590450915A0460915B047091E9
:108500005C04841B950BA60BB70B80936D049093B2
:108510006E04A0936F04B0937004889880917104E6
:1085200090917204A0917304B0917404B7FD15C0CA
:108530004091590450915A0460915B0470915C041D
:10854000841B950BA60BB70B809371049093720458
:10855000A0937304B09374048E98809175049091E5
:108560007604A0917704B0917804B7FD3AC04091A9
:10857000590450915A0460915B0470915C04841B0F
:10858000950BA60BB70B8093750490937604A0937C
:108590007704B093780480914B048823E1F08091B4
:1085A000490482FF04C08091060287FD05C08091C6
:1085B0004804882309F48FC78091490490914A04A4
:1085C00093FF04C08091060287FD0BC08091470491
:1085D000811107C005C080910B018870809309014B
:1085E0004198E15041F0809184009091850082177C
:1085F0009307C8F34BCE8091110290911202A09183
:108600001302B0911402892B8A2B8B2B09F08AC09C
:1086100080918704882309F453C08090950490903A
:108620009604A0909704B0909804C0908204D090D3
:108630008304E0908404F090850440918604C8147B
:10864000D904EA04FB0480F480915204909153040D
:1086500020915604309157042817390728F44150C7
:1086600040938604019714C08C149D04AE04BF048B
:10867000E0F480915204909153042091540430917D
:1086800055048217930788F44F5F40938604019640
:10869000909353048093520440910D0250910E0226
:1086A00060910F02709110020EC08FEF9FEFDC01FE
:1086B00080930D0290930E02A0930F02B0931002CC
:1086C0004FEF5FEFBA018091860487FD02C0169AD2
:1086D00001C0169880918400909185004C9620915D
:1086E00086042223B9F0149A2091860427FF02C041
:1086F0002F5F01C021502093860414982091860496
:10870000222369F3209184003091850028173907CE
:10871000C8F3E5CF40931102509312026093130205
:10872000709314028091990490919A04A0919B04F3
:10873000B0919C04892B8A2B8B2B09F049C6A09100
:108740001610B0911710109711F40C940D4C8090E6
:10875000950490909604A0909704B090980440914E
:108760009104509192046091930470919404841642
:108770009506A606B706D8F010925104109217106D
:108780001092161090910B0A80910C0A981711F410
:108790000C940D4C80910C0A8F5F8F7080930C0AA3
:1087A00040EDC42E47E0D42EE12CF12C1AC44091A8
:1087B0008D0450918E0460918F047091900448153F
:1087C00059056A057B0508F4AAC1409189045091B6
:1087D0008A0460918B0470918C04D6960D911D9142
:1087E0002D913C91D997401751076207730708F004
:1087F00077C1411551056105710549F480904D041B
:1088000090904E04A0904F04B090500464C1E12CAD
:10881000F980842E952F862F0A811B81FD81EE81A0
:108820003F8128859C80E091EE17E89D912CFF27E1
:108830003091EF17389D900CF11D1090F017189C97
:10884000F00DE99F900CF11D399FF00DE89FF00DA0
:10885000092D1F2F099DE12D332722270F9FE00DA2
:10886000311D2E1D199DE00D311D2E1D1F9F300D38
:10887000211D032F122F099DF12C332722270F9F33
:10888000F00C311D2E1D199DF00C311D2E1D1F9F4A
:10889000300D211D032F122FEE2780904D04909153
:1088A0004E0480914F040090A9040E2809F483C05F
:1088B0003091A504309FE1198E089E098E09209100
:1088C000A604209FE01981089E098E09F090A70454
:1088D000F09E801891098E09319FE01981089E0948
:1088E0008E09219F801891098E09F19E90198109A6
:1088F000099DF12C332722270F9FF00C311D2E1DCF
:10890000199DF00C311D2E1D1F9F300D211D032FB1
:10891000122F3091A104309FE10D8E1C9E1D8E1DE3
:108920002091A204209FE00D811C9E1D8E1DF090C1
:10893000A304F09E800C911D8E1D319FE00D811CC3
:108940009E1D8E1D219F800C911D8E1DF19E900DF0
:10895000811D099DF12C332722270F9FF00C311D1B
:108960002E1D199DF00C311D2E1D1F9F300D211D38
:10897000032F122F30919D04309FE1198E089E091C
:108980008E0920919E04209FE01981089E098E097E
:10899000F0909F04F09E801891098E09319FE01994
:1089A00081089E098E09219F801891098E09F19EE8
:1089B0009019810982C03091A504309FE10D8E1C71
:1089C0009E1D8E1D2091A604209FE00D811C9E1DE2
:1089D0008E1DF090A704F09E800C911D8E1D319F7E
:1089E000E00D811C9E1D8E1D219F800C911D8E1DF2
:1089F000F19E900D811D099DF12C332722270F9F99
:108A0000F00C311D2E1D199DF00C311D2E1D1F9FC8
:108A1000300D211D032F122F3091A104309FE11939
:108A20008E089E098E092091A204209FE0198108DA
:108A30009E098E09F090A304F09E801891098E097A
:108A4000319FE01981089E098E09219F80189109A4
:108A50008E09F19E90198109099DF12C3327222757
:108A60000F9FF00C311D2E1D199DF00C311D2E1D78
:108A70001F9F300D211D032F122F30919D04309F19
:108A8000E10D8E1C9E1D8E1D20919E04209FE00DE9
:108A9000811C9E1D8E1DF0909F04F09E800C911DE8
:108AA0008E1D319FE00D811C9E1D8E1D219F800C0F
:108AB000911D8E1DF19E900D811D11249C82F982C5
:108AC0000A831B83FD83EE833F832887912C992A99
:108AD000A12CB12CA82A8BEC94E121E0298B14C0A5
:108AE000D2968D909D90AD90BC90D597F4CFB694D2
:108AF000A79497948794D988DD0CD98A049624E1A9
:108B0000873E920709F4EDC4FC010591159125916A
:108B10003491081519052A053B0548F3E2C4409035
:108B200082045090830460908404709085044814FB
:108B300059046A047B0408F0C3C180918104811147
:108B400021C0FD01EE5BFF4FE080F18002811381C7
:108B500078962081318142815381D2966D917D91A9
:108B60008D919C91D5970E944CB6DD24D394D092E0
:108B70008104E0911610F091171082A993A9A4A97D
:108B8000B5A98EC140917D0450917E0460917F040F
:108B900070918004DA960D911D912D913C91DD9795
:108BA000401751076207730708F073C1411551055B
:108BB0006105710549F480914D0490914E04A09196
:108BC0004F04B09150046CC1F0E0E985842F352F3B
:108BD000262FAA857B856C855D85BE854F85988906
:108BE000B091EE17B89F612D55274091EF17489F20
:108BF000600D511D1090F017189E500DB39F600D21
:108C0000511D439F500DB29F500DA62F752FA69F4B
:108C1000B12D44279927A59FB00D411D9F1F769F19
:108C2000B00D411D9F1F759F400D911DA42F792FE1
:108C3000A69FE12D44279927A59FE00D411D9F1F69
:108C4000769FE00D411D9F1F759F400D911DA42F24
:108C5000792FBB2780914D0430914E0420914F0411
:108C60000090A9040F2A09F483C04091A5044A9FEB
:108C7000B1198F0B3F0B2F0B9091A6049A9FB0193F
:108C800081093F0B2F0BE091A704EA9F801931095E
:108C90002F0B479FB01981093F0B2F0B979F80190E
:108CA00031092F0BE79F30192109A69FE12D442799
:108CB0009927A59FE00D411D9F1F769FE00D411D47
:108CC0009F1F759F400D911DA42F792F4091A104E6
:108CD0004A9FB10D8F1F3F1F2F1F9091A2049A9F93
:108CE000B00D811D3F1F2F1FE091A304EA9F800D4F
:108CF000311D2F1F479FB00D811D3F1F2F1F979FB5
:108D0000800D311D2F1FE79F300D211DA69FE12DE6
:108D100044279927A59FE00D411D9F1F769FE00DD9
:108D2000411D9F1F759F400D911DA42F792F4091CC
:108D30009D044A9FB1198F0B3F0B2F0B90919E04FE
:108D40009A9FB01981093F0B2F0BE0919F04EA9F76
:108D5000801931092F0B479FB01981093F0B2F0B49
:108D6000979F801931092F0BE79F3019210982C085
:108D70004091A5044A9FB10D8F1F3F1F2F1F909157
:108D8000A6049A9FB00D811D3F1F2F1FE091A704DD
:108D9000EA9F800D311D2F1F479FB00D811D3F1F82
:108DA0002F1F979F800D311D2F1FE79F300D211D15
:108DB000A69FE12D44279927A59FE00D411D9F1FE8
:108DC000769FE00D411D9F1F759F400D911DA42FA3
:108DD000792F4091A1044A9FB1198F0B3F0B2F0BA4
:108DE0009091A2049A9FB01981093F0B2F0BE0913B
:108DF000A304EA9F801931092F0B479FB0198109FD
:108E00003F0B2F0B979F801931092F0BE79F3019CC
:108E10002109A69FE12D44279927A59FE00D411D1B
:108E20009F1F769FE00D411D9F1F759F400D911D57
:108E3000A42F792F40919D044A9FB10D8F1F3F1F92
:108E40002F1F90919E049A9FB00D811D3F1F2F1FD1
:108E5000E0919F04EA9F800D311D2F1F479FB00DA9
:108E6000811D3F1F2F1F979F800D311D2F1FE79FD3
:108E7000300D211D1124E987AA877B876C875D87C8
:108E8000BE874F87988B90E0932BA0E0B0E0A22B99
:108E900007C0A65ABF4F8D919D910D90BC91A02DFA
:108EA0002BEC34E141E0498BF901459155916591F5
:108EB0007491481759076A077B0708F49CC3AAC333
:108EC000809186048823E1F0FD01E85BFF4F40813B
:108ED000518160E070E000910D0210910E0220912E
:108EE0000F0230911002401751076207730741F0DB
:108EF0001092110210921202109213021092140298
:108F00004091090250910A0260910B0270910C028B
:108F100077FF5FC0AE5ABF4FCD90DD90ED90FC90D3
:108F20008BEC94E121E0FC014591559165917491A0
:108F30004C155D056E057F0550F4F694E794D794C3
:108F4000C794220F049674E1873E970761F7209338
:108F5000880480E2C816D104E104F10428F470E228
:108F6000C72ED12CE12CF12C90E2C91AD108E108CE
:108F7000F108C114A8E0DA06E104F10408F406C41B
:108F8000B4E0DB9EC001112485539F4EFC01329654
:108F900025913491EC2D6627E39FA001E29F410DBE
:108FA000561F0694461F561F112460E070E0FC0116
:108FB00025913491C901A0E0B0E0841B950BA60B6C
:108FC000B70B8093090290930A02A0930B02B0930F
:108FD0000C02C0900902D0900A02E0900B02F090BF
:108FE0000C028091161090911710892B09F0E8C19E
:108FF0000E94CBB69093171080931610892B09F41A
:10900000DFC1E0911610F0911710808183FF3EC000
:1090100085899689A789B08D809325109093261015
:10902000A0932710B0932810818D928DA38DB48DBD
:109030008093291090932A10A0932B10B0932C109A
:10904000858D968DA78DB0A180932D1090932E10B5
:10905000A0932F10B093301081A192A1A3A1B4A12D
:109060008093311090933210A0933310B09334104A
:1090700090910B0A80910C0A981709F4B9CF80914E
:109080000C0A8F5F8F7080930C0AB2CFC588D68888
:10909000E788F08C81E0C114D104E104F10409F403
:1090A00080E0018D128D238D348D01151105210570
:1090B000310509F08260458D568D678D70A141158F
:1090C00051056105710509F0846080935104109287
:1090D0007D0410927E0410927F04109280041092FE
:1090E000890410928A0410928B0410928C0485A13A
:1090F00096A1A7A1B0A58093910490939204A09308
:109100009304B0939404882499245401881A990AEA
:10911000AA0ABB0A8092790490927A04A0927B04F6
:10912000B0927C048092750490927604A0927704A9
:10913000B09278048092710490927204A0927304A9
:10914000B092740480926D0490926E04A0926F04A9
:10915000B0927004CC0CDD1CEE1CFF1CC0925D04B0
:10916000D0925E04E0925F04F0926004000F111F41
:10917000221F331F00936104109362042093630441
:1091800030936404440F551F661F771F4093650496
:1091900050936604609367047093680441A152A1E0
:1091A00063A174A1440F551F661F771F4093690484
:1091B00050936A0460936B0470936C04880F991F3A
:1091C000AA1FBB1F8093590490935A04A0935B0479
:1091D000B0935C0410929504109296041092970438
:1091E0001092980482A593A5A4A5B5A580938D049B
:1091F00090938E04A0938F04B093900486A597A5B6
:10920000A0A9B1A98093820490938304A0938404BD
:10921000B093850481A580935804DF01A95BBF4FFB
:109220009C9190938704992339F115962D913C9147
:109230001197309357042093560412972D913C9127
:1092400011973093550420935404109211021092F8
:109250001202109213021092140212972D913C9157
:10926000A90160E070E040930D0250930E026093FC
:109270000F02709310020CC088248A94982C540119
:1092800080920D0290920E02A0920F02B0921002F4
:10929000EA5BFF4F908120914C0492130AC0209109
:1092A000080230E0482F082E000C550B42175307D8
:1092B00031F090934C04809308020E949EB68091F6
:1092C000680681110E94AFAF2FEF3FEFA9012093F5
:1092D000090230930A0240930B0250930C02E09172
:1092E0001610F0911710DF01DE96ED90FD900D91B4
:1092F0001C9122A933A944A955A9EA5AFF4F6081BC
:109300007181828193810E944CB610928104E09118
:109310001610F0911710EA5AFF4F80809180A280BA
:10932000B3808BEC94E121E0FC014591559165916E
:109330007491481559056A057B0558F4B694A794AD
:1093400097948794220F0496A7EEB4E1A817B90763
:1093500059F720938804B0E28B169104A104B1045C
:1093600028F4B0E28B2E912CA12CB12C30E2831A80
:109370009108A108B108811448E09406A104B10441
:1093800008F428C254E0959EC001112485539F4ED5
:10939000FC01329625913491782D6627739FA001A8
:1093A000729F410D561F0694461F561F1124FC0143
:1093B000C590D490E12CF12CC41AD50AE108F1082B
:1093C000C0929904D0929A04E0929B04F0929C047B
:1093D0000091990410919A0420919B0430919C046F
:1093E0004091110250911202609113027091140287
:1093F000F02E198BF22FE32F4017510762077307E6
:1094000020F4F42E598BF62FE72F8F2D9989AF2F4B
:10941000BE2F0097E1E0AE07B10520F08FEF9FEF80
:10942000A0E0B0E0081B190B2A0B3B0B009399043A
:1094300010939A0420939B0430939C044F3FFFEFBA
:109440005F076F077F0761F0481B590B6A0B7B0BA7
:10945000409311025093120260931302709314020E
:10946000F8942091840030918500205F3F4F4A8915
:1094700041504A8B442341F0280E391E22163306F0
:1094800010F40C94DE4001C0190130928900209242
:109490008800789462960FB6F894DEBF0FBECDBFF9
:1094A000DF91CF911F910F91FF90EF90DF90CF90C0
:1094B000BF90AF909F908F907F906F905F904F90F4
:1094C0003F902F90089580910B0180958870809334
:1094D00009010C94EA4180910B0188708093090185
:1094E0006BC839893093880480E288169104A104FE
:1094F000B10428F430E2832E912CA12CB12C30E25F
:10950000831A9108A108B108811488E09806A10483
:10951000B10420F1E4E09E9EC001112485539F4ECA
:10952000FC01329625913491F82DEE27F39F7001BE
:10953000F29FE10CFE1E0694EE1EFE1E1124FC019D
:10954000C590D490860120E030E0480159018E1882
:109550009F08A108B1087501640122C0950184012A
:109560003695279517950795F801EC7FCF01855320
:10957000934FFC01C590D490FC0132962591349113
:10958000E82DE770E29FC001E39F900D112423E0D6
:10959000969587952A95E1F7C81AD90AE12CF12CFE
:1095A0004C0D5D1D6E1D7F1D4093890450938A04F0
:1095B00060938B0470938C0490918704809186044F
:1095C000992309F474C0882309F40BCDA85BBF4F1D
:1095D0008D919C91A0E0B0E040910D0250910E025F
:1095E00060910F027091100284179507A607B707C4
:1095F00009F060C0F6CCB695A79597958795D98860
:10960000DD0CD98A2C5F3F4F47EE54E142175307D8
:1096100009F04ACC59895093880480329105A105FC
:10962000B10520F480E290E0A0E0B0E08097A109CD
:10963000B109811558E09507A105B10508F443C0AB
:1096400074E0979F9001112425533F4EF901329603
:1096500045915491EE27859FB001849F610D7E1F37
:1096600006946E1F7E1F1124F901C590D490E12C41
:10967000F12CC61AD70AE108F10880917D04909177
:109680007E04A0917F04B09180048C0D9D1DAE1DC1
:10969000BF1D80937D0490937E04A0937F04B093BC
:1096A000800480918704811130C0809186048823D2
:1096B00009F497CC10921102109212021092130228
:1096C000109214028ECCAC01BD017695679557952A
:1096D0004795FA01EC7F9F012553334FF901C5905F
:1096E000D490F9013296459154918770849F9001EE
:1096F000859F300D1124F3E036952795FA95E1F713
:10970000C21AD30AE12CF12CB8CF8989480E511C1A
:10971000611C711C80911610909117104814590407
:109720006A047B04D8F420918604222309F459CCDE
:10973000FC01E85BFF4F20813181A90160E070E00E
:1097400000910D0210910E0220910F023091100233
:10975000401751076207730709F443CC10921102B6
:10976000109212021092130210921402FC01E85B94
:10977000FF4F80819181A0E0B0E080930D02909333
:109780000E02A0930F02B09310022BCCD701C6019A
:10979000B695A79597958795FC01EC7FCF018553EA
:1097A000934FFC0125913491FC01329645915491DF
:1097B0006C2D6770649FC001659F900D112463E05C
:1097C000969587956A95E1F7281B390BC901A0E0AA
:1097D000B0E0F7CBD501C401B695A79597958795CD
:1097E000FC01EC7FCF018553934FFC01C590D490D1
:1097F000FC01329625913491482D4770429FC0015B
:10980000439F900D1124A3E096958795AA95E1F7C3
:10981000C81AD90AE12CF12CD3CD80EDC82E87E0EF
:10982000D82EE12CF12CE4CB90910318E92FF0E035
:10983000EB58F94F80839F5F943018F4909303188E
:1098400002C010920318809104188F5F809304184F
:1098500008958091AA059091AB05981759F0E92FCA
:10986000F0E0E65DFA4F80819F5F9F779093AB05B4
:1098700090E008958FEF9FEF08950F931F93CF937C
:10988000DF93FC01A685B7858D0100581F4FE801C5
:109890008881998101968F779927AD014E575F4F47
:1098A000EA012881398128173907D1F3E801288195
:1098B0003981A20FB31F6C93A685B785A058BF4FFF
:1098C00011969C938E93A689B7892C9181E090E0A4
:1098D000078C02C0880F991F0A94E2F7822B8C93A1
:1098E00081E081A30488F589E02D808180648083F4
:1098F00081E090E0DF91CF911F910F910895FC01DD
:1099000081A1882329F0A489B5898C9186FFFBCF9A
:1099100011A20895FC01A485B585FD01E058FF4F13
:10992000208131813296808191812817390779F021
:1099300080819181A80FB91F8C91208131812F5F87
:109940003F4F2F7733273183208390E008958FEFA7
:109950009FEF0895DC011C96ED91FC911D97DF01AE
:10996000A058BF4F2D913C91119712968D919C91CB
:1099700011972817390739F08D919C91E80FF91F3D
:10998000808190E008958FEF9FEF0895FC0124857A
:109990003585F901E058FF4F808191813296208111
:1099A000318180589F4F821B930B60E870E00C94CC
:1099B000A0DC0895089580E090E00895CF93FC0125
:1099C00020812B33A1F020910418243080F4C62F7D
:1099D000BC0180910318F0E68F9FC00111248658C6
:1099E000994F0E9437DD8C2F1FDF81E001C080E09E
:1099F000CF9108952F923F924F925F926F927F92F4
:109A00008F929F92AF92BF92CF92DF92EF92FF928E
:109A10000F931F93CF93DF9300D000D0CDB7DEB765
:109A20009A8389830E9402C5E981FA81C680D78022
:109A3000E084F184C114D104E104F10409F0ACC262
:109A40002485222309F469C332852150248721E02B
:109A5000230F22874585241301C01286E981FA81EC
:109A600024E0329FE00DF11D1124C684D784E088E4
:109A7000F188E981FA81C282D382E482F582DC0135
:109A8000CB018C0D9D1DA11DB11D86839783A087E1
:109A9000B18784819581892B09F43FC3FFB7FD838A
:109AA000F894E981FA81228033802101612C712CA4
:109AB0000481158180912D028F3121F08F3F09F0B3
:109AC00068C205C0EFE8FCE124912E83DAC08FE183
:109AD00080932D02EFE8FCE184918E838F3F09F49F
:109AE00058C2823009F469C030F5882309F44CC0AB
:109AF000813009F0C6C010928000109281008091E0
:109B000081008860809381008091810081608093D2
:109B10008100E6EAF7E2E491F0E0EE0FFF1FED5A74
:109B2000F84D85919491ECEEF7E2E491E093AD0469
:109B3000E1E0EE8330C19E81943009F482C008F4E4
:109B400060C0953009F09DC0109220011092210153
:109B500080912101886080932101809121018160A1
:109B600080932101E6EAF7E2E491F0E0EE0FFF1FB7
:109B7000ED5AF84D85919491ECEEF7E2E491E09383
:109B8000AA0495E09E8307C114BC15BC84B582600D
:109B900084BD85B5816085BDE6EAF7E2E491F0E039
:109BA000EE0FFF1FED5AF84D85919491ECEEF7E220
:109BB000E491E093AE041E82ABC21092B00010920A
:109BC000B1008091B00082608093B0008091B100BC
:109BD00081608093B100E6EAF7E2E491F0E0EE0FF5
:109BE000FF1FED5AF84D8591949190935A068093FA
:109BF0005906ECEEF7E2E491E0935B06F2E0FE83B7
:109C000087C210929000109291008091910088601C
:109C10008093910080919100816080939100E6EAA9
:109C2000F7E2E491F0E0EE0FFF1FED5AF84D859159
:109C30009491ECEEF7E2E491E093AC0423E02E8300
:109C4000AAC01092A0001092A1008091A10088608B
:109C50008093A1008091A10081608093A100E6EA39
:109C6000F7E2E491F0E0EE0FFF1FED5AF84D859119
:109C70009491ECEEF7E2E491E093AB0484E08E8300
:109C80008AC0EE81E7FD85C161E08FE10E94C7C314
:109C90008E818D7F09F083C04801A12CB12C60E03A
:109CA00072E18AE790E0A50194010E94B3DC298368
:109CB0003A834B835C8369017A01F1E0CF1AD108C2
:109CC000E108F1082FEFC216D104E104F10409F014
:109CD00008F44EC060E472E48FE090E0A5019401C6
:109CE0000E94B3DC69017A0181E0C81AD108E10859
:109CF000F1089E81923009F5EFEFCE16D104E10410
:109D0000F10409F008F4CBC160E970ED83E090E064
:109D1000A50194010E94B3DC69017A01F1E0CF1A38
:109D2000D108E108F1082FEFC216D104E104F104D3
:109D300011F008F041C183E027C08FEFC816D104AD
:109D4000E104F104B9F0B0F068E478EE81E090E06D
:109D5000A50194010E94B3DC69017A0191E0C91A5E
:109D6000D108E108F108EE81EE2309F49AC163C13C
:109D700081E001C082E09E81911106C095B5987F77
:109D8000892B85BD7AC085E09091B100987F892BA1
:109D90008093B10072C061E08FE10E94C7C34801A7
:109DA000A12CB12C60E072E18AE790E0A50194015A
:109DB0000E94B3DC69017A01E1E0CE1AD108E10822
:109DC000F108C114D104F1E0EF06F10488F068E471
:109DD00078EE81E090E0A50194010E94B3DC690176
:109DE0007A0181E0C81AD108E108F10883E001C0D6
:109DF00081E09E81913071F490918100987F892B50
:109E000080938100452846284728D9F52FEF3FEF5A
:109E1000A90168C0EE81E33071F490919100987FC0
:109E2000892B8093910045284628472851F52FEF2C
:109E30003FEFA90179C0FE81F43071F49091A10047
:109E4000987F892B8093A100452846284728C9F48C
:109E50002FEF3FEFA9017AC02E81253071F4909148
:109E60002101987F892B8093210145284628472886
:109E700041F42FEF3FEFA9017BC045284628472832
:109E800069F0D801AA0FBB1F91010E94A7D928EE43
:109E900033E040E050E00E947BD903C02FEF3FEF5A
:109EA000A9018E81823081F12CF4882361F0813008
:109EB000C9F06FC09E81943009F448C0ACF1953070
:109EC00009F456C066C0C7BC2093BF043093C004D9
:109ED0004093C1045093C20480916E0082608093CD
:109EE0006E0057C0D0928900C09288002093BB04B6
:109EF0003093BC044093BD045093BE0480916F0026
:109F0000826080936F0045C0C092B30020935C06CE
:109F100030935D0640935E0650935F06809170001B
:109F200082608093700035C0D0929900C0929800F2
:109F30002093B7043093B8044093B9045093BA0403
:109F40008091710082608093710023C0D092A9003B
:109F5000C092A8002093B3043093B4044093B50496
:109F60005093B6048091720082608093720011C099
:109F7000D0922901C09228012093AF043093B004FD
:109F80004093B1045093B204809173008260809337
:109F90007300ED81EFBFC1C0DC01CB018C199D09BD
:109FA000AE09BF09B7FDB9C04698E981FA811682AA
:109FB000178210861186B1C068E478EE81E090E0E7
:109FC000A50194010E94B3DC69017A01F1E0CF1A86
:109FD000D108E108F1082FEFC216D104E104F10421
:109FE00041F138F164E274EF80E090E0A501940162
:109FF0000E94B3DC69017A01F1E0CF1AD108E108CF
:10A00000F1082FEFC216D104E104F10409F008F4BD
:10A01000BACE62E17AE780E090E0A50194010E9467
:10A02000B3DC69017A0181E0C81AD108E108F108BE
:10A0300019C084E0A9CE2FEFC216D104E104F104C7
:10A0400009F008F463C062E17AE780E090E0A501DE
:10A0500094010E94B3DC69017A01F1E0CF1AD108C2
:10A06000E108F1082FEFC216D104E104F104A9F0D0
:10A07000A0F089819A81AB81BC812AE0B595A79532
:10A08000979587952A95D1F76C017D01F1E0CF1A5C
:10A09000D108E108F10887E077CE86E075CE82E04E
:10A0A00073CEEFEFCE16D104E104F10469F160F153
:10A0B00062E17AE780E090E0A50194010E94B3DCC0
:10A0C00069017A0181E0C81AD108E108F1089FEF1F
:10A0D000C916D104E104F104A9F0A0F089819A81A4
:10A0E000AB81BC813AE0B595A795979587953A9550
:10A0F000D1F76C017D01E1E0CE1AD108E108F10849
:10A1000085E03CCE84E03ACE83E038CE84E033CEA6
:10A1100061E08FE10E94C7C3BFCD26960FB6F894C9
:10A12000DEBF0FBECDBFDF91CF911F910F91FF908A
:10A13000EF90DF90CF90BF90AF909F908F907F90E7
:10A140006F905F904F903F902F9008950F931F93C3
:10A15000CF93DF93CDB7DEB72C970FB6F894DEBF61
:10A160000FBECDBFE9E2F4E080859185A285B3857D
:10A1700044815581668177810081118122813381FB
:10A1800009831A832B833C834D835E836F83788797
:10A1900089879A87AB87BC87AE01475F5F4FBE0157
:10A1A0006B5F7F4FCE0101960E94B2AE25E334E093
:10A1B000AE01475F5F4FBE016B5F7F4FCE010196DF
:10A1C0000E9408BA2C960FB6F894DEBF0FBECDBF22
:10A1D000DF91CF911F910F91089580910C04909180
:10A1E0000D04009731F04AE050E060E070E00C941C
:10A1F000E1D260E070E0CB010895EFDF97FD0AC087
:10A20000ECDF6F3F71058105910509F02CF4E5DF66
:10A21000862F089580E008958FEF089580910C04B3
:10A2200090910D04892B31F0E8DF91E0811103C09A
:10A2300090E001C091E0892F08950F931F93CF9371
:10A2400080910C0490910D04009711F1FC018F0195
:10A25000C1912C2F2F7DA9F0C53411F0C536B9F767
:10A26000F801108260E070E080910C0490910D0480
:10A270000E948ED1F801C083562F472F382F292FE7
:10A280000BC060E070E0CF911F910F910C948ED1C4
:10A2900050E040E030E020E0652F742F832F922FB4
:10A2A000CF911F910F91089581548A3108F042C0D7
:10A2B000E82FF0E040912E1850912F18609130183F
:10A2C0007091311804C076956795579547958A9592
:10A2D000D2F7842F817040FF2FC0EC5EF74E908143
:10A2E000992309F1E091F317F091F417E90FF11DAB
:10A2F000908120ED290F2A3098F09E3211F491813F
:10A300000CC09D3211F09B3271F4918120ED290F28
:10A310002A3030F09E3239F4928190539A3018F4FA
:10A320002E2F9F2F02C020E090E020930C049093EA
:10A330000D04089580E008950895B6DF882341F064
:10A3400081E020910C0430910D04232B09F480E06E
:10A350000895FC01238121110C94B4A2089580E199
:10A36000E9E2F4E0A0EEB5E001900D928A95E1F704
:10A3700008959091C00095FFFCCF8093C60008958A
:10A38000EF92FF921F93CF93DF937C0160E016DB87
:10A39000182F882399F0EFE6FEE18491EF012196D2
:10A3A000882319F0E6DFFE01F8CFB7018BEE94E1C8
:10A3B0000E9453B782E2DDDF8AE0DBDF812FDF918D
:10A3C000CF911F91FF90EF900895DF92EF92FF924F
:10A3D0000F931F93CF93DF93CDB7DEB76E970FB672
:10A3E000F894DEBF0FBECDBF6091FB077091FC07F4
:10A3F0006115710541F14DE150E0CE0101967C01FE
:10A400000E9436D51E8EF7018F010E191F09D190BB
:10A41000DD2019F09AE0D912F7CFF701E00FF11F14
:10A420001082C701ADDF882371F0DD20A9F00F5F36
:10A430001F4F8091FB079091FC07080F191F109385
:10A44000FC070093FB0781E02091FB073091FC079C
:10A45000232B29F480E003C000E010E0F0CF6E96DB
:10A460000FB6F894DEBF0FBECDBFDF91CF911F9125
:10A470000F91FF90EF90DF9008953F924F925F927F
:10A480006F927F928F929F92AF92BF92CF92DF9204
:10A49000EF92FF920F931F93CF93DF931F92CDB74D
:10A4A000DEB793DF811174C280910418843008F004
:10A4B00047C0CFD9AC0197FF7CC142C08E3409F0B0
:10A4C000D9C10115110509F4D5C16EE176E1C801C4
:10A4D0000E9445D57C01892B09F48EC16EE470E0A1
:10A4E000C80104960E9423DD009709F485C14AE063
:10A4F00050E060E070E001960E94E1D26093C304F6
:10A500007093C4048093C5049093C604809010187F
:10A5100090901118A0901218B09013182FEF821A73
:10A52000920AA20AB20A681579058A059B0509F400
:10A5300065C1EF2809F062C18BEE95E10E940CC75E
:10A540008091890A882309F423C28091041881111B
:10A5500002C010922905EE24E3944091030D50911E
:10A56000040D6091050D7091060D8091FF0C909186
:10A57000000DA091010DB091020D481759076A070F
:10A580007B0708F4E12C00E010E09924939480E626
:10A59000882E93E2A92E96E1B92E2DE8322E8091D5
:10A5A0000418843008F0F4C1E110F2C1809129054B
:10A5B0008111EEC180915A0C90915B0CA0915C0CC2
:10A5C000B0915D0C8093030D9093040DA093050D45
:10A5D000B093060D41E050E0BE016F5F7F4F82E512
:10A5E0009CE00E943BA5019719F4898190E002C08C
:10A5F0008FEF9FEFF82E4090030D5090040D609068
:10A60000050D7090060D4091FF0C5091000D60916A
:10A61000010D7091020DEE24E39444165506660672
:10A62000770608F4E12C4416550666067706B0F462
:10A63000019609F46AC08AE0F81609F489C09DE021
:10A64000F91609F485C023E2F21619F08AE3F8122C
:10A6500096C080912805811192C06FC00E94087138
:10A6600082E59CE00E94B4A280916D0C882359F190
:10A67000815080936D0C389EC001112441E061E04F
:10A680008E58934F0E946AC5E0916D0C94E0E99F4B
:10A69000F0011124E259F34F4081518162817381AD
:10A6A0004093030D5093040D6093050D7093060DB8
:10A6B00082E59CE00E94CAA180918A0A8823A9F0C1
:10A6C0009092890A12C01092890A0E9494A90E944D
:10A6D0004E9B0E94DD9A6D3371058105910528F02E
:10A6E000B092FC07A092FB0770DE8091890A81116D
:10A6F00028C0E6E3F6E184916F012FEFC21AD20A77
:10A700008823D9F036DEF601F6CFEAE5FEE1849142
:10A710006F019FEFC91AD90A882319F02ADEF601C2
:10A72000F6CFE7E2F6E184916F012FEFC21AD20A69
:10A73000882319F01EDEF601F6CF83E2F81208C076
:10A7400005C023E2F21221C100E010E09092290539
:10A75000109228050115110519F40E94239E0CC0C2
:10A7600080910318889E000D111D1124F801E658F0
:10A77000F94F108280E058D800E010E010CF0F357C
:10A78000110508F00CCF9BE3F91202C09092280546
:10A7900080912805811103CF80910318F801889ECC
:10A7A000E00DF11D1124E658F94FF0820F5F1F4FA5
:10A7B000F6CE982F20910E1830910F188A3019F08C
:10A7C0009D3009F0B0C0109227052115310519F40C
:10A7D0000E94239E69CEF901E953FB4F108210922B
:10A7E0000F1810920E1807EC14E0F80181918032D6
:10A7F00009F064CE8F01F9CFC80179CE6AE270E02A
:10A80000C8010E945BDD9C01009701F1982F901B0D
:10A81000F12C992339F09150F801E90FF11D808155
:10A82000F826F7CF4AE050E060E070E0C9010196F9
:10A830000E94E1D2CF2CD12CE12CF12C6C157D059E
:10A840008E059F0531F08CEC95E178CE82EA95E19A
:10A8500075CE8091C3049091C404A091C504B091B9
:10A86000C6048093101890931118A0931218B093F7
:10A8700013180EC08091870A882351F064EE73E0AC
:10A88000C8010E942EDD892B19F088E795E156CE8C
:10A8900080913502811126C067E470E0C8010E94F2
:10A8A00023DD0097F9F04AE050E060E070E00196A7
:10A8B0000E94E1D297FD16C06430710581059105B3
:10A8C0002CF0653071058105910561F4E1E0F5E159
:10A8D00084917F019FEFE91AF90A882319F049DD75
:10A8E000F701F6CF68EE73E0C8010E942EDD892BD8
:10A8F00011F4109234026DEE73E0C8010E942EDD57
:10A90000892B19F488EF94E188D362EF73E0C801D2
:10A910000E942EDD892B11F40E94227561E087ECE4
:10A9200094E04CD8C1CD2F3531050CF0BDCD9C3510
:10A93000C1F40E94294C97FDB7CD20912705211124
:10A94000B3CD20910E1830910F18A9014F5F5F4FC2
:10A9500050930F1840930E18F901E953FB4F808371
:10A96000A3CD9B3319F481E08093270580912705BF
:10A9700081119ACDC901019690930F1880930E18FA
:10A98000F901E953FB4F40838FCD10922805E5CEA6
:10A990000F90DF91CF911F910F91FF90EF90DF907B
:10A9A000CF90BF90AF909F908F907F906F905F906F
:10A9B0004F903F9008958F929F92AF92BF92EF92E7
:10A9C000FF920F931F93CF93DF93CDB7DEB7A0977E
:10A9D0000FB6F894DEBF0FBECDBF611571058105BE
:10A9E000910589F100E0842E912CA12CB12C102F1F
:10A9F000EE24E394F12CEC0EFD1EE00EF11C07FD9D
:10AA0000FA94A50194010E947BD9F7016083B901F2
:10AA1000CA010F5F611571058105910541F71F3F5F
:10AA200021F1E1E0F0E0EC0FFD1FE10FF11D17FD5A
:10AA3000FA9580818A3010F097E301C090E3890F86
:10AA400098DC1150ECCF80E3A0960FB6F894DEBFEF
:10AA50000FBECDBFDF91CF911F910F91FF90EF906F
:10AA6000BF90AF909F908F9084CCA0960FB6F89433
:10AA7000DEBF0FBECDBFDF91CF911F910F91FF9031
:10AA8000EF90BF90AF909F908F900895CF92DF92FC
:10AA9000EF92FF926B017C0197FF0AC08DE269DCA7
:10AAA000F094E094D094C094C11CD11CE11CF11C22
:10AAB0004AE0C701B601FF90EF90DF90CF907BCFC7
:10AAC0008F929F92AF92BF92CF92DF92EF92FF92BE
:10AAD000CF936B017C01B42E20E030E0A9010E94ED
:10AAE0008DD587FF06C08DE244DCF7FAF094F7F8C5
:10AAF000F094C0E060E070E080E09FE3CB1541F0AF
:10AB00002DEC3CEC4CEC5DE30E94F2D5CF5FF6CF30
:10AB10009B01AC01C701B6010E94B7D96B017C0152
:10AB20000E9400DB4B015C014AE045DFCC2379F158
:10AB3000C501B4010E9491D59B01AC01C701B601CA
:10AB40000E94B6D96B017C018EE213DC20E030E07C
:10AB500040E251E4C701B6010E94F2D54B015C010D
:10AB60000E94FBDA6B01770FEE08FF08C701B60100
:10AB70008DDFC701B6010E9493D59B01AC01C501D1
:10AB8000B4010E94B6D96B017C01C150F9F6CF9196
:10AB9000FF90EF90DF90CF90BF90AF909F908F90FD
:10ABA00008951F920F920FB60F9211240BB60F92B9
:10ABB0002F938F939F93EF93FF932091AB05E09199
:10ABC000AA0581E08E0F8F779091C600281729F093
:10ABD000F0E0E65DFA4F9083E82FE093AA05FF913D
:10ABE000EF919F918F912F910F900BBE0F900FBE01
:10ABF0000F901F9018959C0197FD0EC0843691050B
:10AC000084F064E670E00E94A0DCCB016AE070E0B2
:10AC10000E94A0DC805D06C03195219531098DE24E
:10AC200001C080E2809324042A30310564F0EAE018
:10AC3000F0E0C901BF010E94A0DCCB01BF010E946E
:10AC4000A0DC805D01C080E280932504C9016AE038
:10AC500070E00E94A0DC805D8093260484E294E092
:10AC600008951F920F920FB60F9211240BB60F92F8
:10AC70002F933F938F939F93EF93FF9320916A0FAE
:10AC800030916B0F80916C0F90916D0F28173907E1
:10AC900031F4809131018F7D8093310114C0E091B6
:10ACA0006C0FF0916D0FE651F14F208180916C0F88
:10ACB00090916D0F01968F77992790936D0F8093E8
:10ACC0006C0F20933601FF91EF919F918F913F91EF
:10ACD0002F910F900BBE0F900FBE0F901F901895E5
:10ACE0001F920F920FB60F9211240BB60F922F9353
:10ACF0004F935F938F939F93EF93FF9380913001D6
:10AD000082FD1CC0209136018091EE0F9091EF0FD3
:10AD10004091F00F5091F10F01968F7799274817C6
:10AD2000590771F0E091EE0FF091EF0FE259F04FFB
:10AD300020839093EF0F8093EE0F02C08091360135
:10AD4000FF91EF919F918F915F914F912F910F9074
:10AD50000BBE0F900FBE0F901F9018958FEF8EBDFA
:10AD60000DB407FEFDCF8EB508954F925F926F929E
:10AD70007F928F929F92AF92BF92CF92DF92EF928B
:10AD8000FF920F931F93CF93DF93D82EC82FD0E05D
:10AD9000FE01E255F84EC49082E0D81203C081E073
:10ADA00080934B047E01EE0CFF1CEE0CFF1CF701A0
:10ADB000EE55F84E45905590659074906C2D0C2C86
:10ADC000000C770B880B990B0E9493D54B015C010B
:10ADD00020E030E040EC5FE3C301B2010E94F2D515
:10ADE000A50194010E94F2D5AB01BC0100E010E086
:10ADF00098018D2D0E94EC7FF701EA56F84E2591BF
:10AE0000359145915491C501B4010E94F2D54B0191
:10AE10005C0120E030E0A9010E948DD5882309F46F
:10AE200046C000E010E09801B501A40170588D2DD6
:10AE30000E94EC7FFE01ED56F84EC491C11115C081
:10AE4000EFE6FEE18491EF012196882319F091DA73
:10AE5000FE01F8CFE1E7F7E18491EF012196882325
:10AE600019F087DAFE01F8CFCAE0F701E459F74D8F
:10AE700045905590659074906C2F70E080E090E064
:10AE80000E9493D59B01AC01C301B2010E9493DAE9
:10AE90002B013C01A5019401C501B4010E94B7D961
:10AEA000AB01BC01930182018D2D0E94EC7F82E0F9
:10AEB000D81249C040902611509027116090281157
:10AEC0007090291120E030E0A901C301B2010E9475
:10AED000DDDB5301420187FF04C0B7FAB094B7F835
:10AEE000B09420E030E0A901C501B4010E948DD5E5
:10AEF000882349F120E030E0A901C301B2011C140C
:10AF00002CF40E94DDDB18162CF008C00E948DD5B1
:10AF100087FF04C081E08093480403C081E08093F0
:10AF200047041C1424F4B7FAB094B7F8B09400E0C6
:10AF300010E09801B501A40182E00E94EC7F10921C
:10AF400048041092470410924B0481E090E00D2CCD
:10AF500001C0880F0A94EAF790912804982B9093E7
:10AF600028049091DF05892B8093DF05F701ED52CE
:10AF7000FA4F10821182128213828D2D0E944C8210
:10AF8000F701EB59F84E85919591A591B491E701A0
:10AF9000C75DDB4F88839983AA83BB83D7D8F7012A
:10AFA000E052FA4F88819981AA81BB818083918385
:10AFB000A283B383DF91CF911F910F91FF90EF9008
:10AFC000DF90CF90BF90AF909F908F907F906F90C9
:10AFD0005F904F90089525EE32E0FC01318320838D
:10AFE0000496B7C95F9A809128048E7F80932804C5
:10AFF0008A9A479A809128048D7F809328048091B3
:10B0000008018095817080930601479A80912804F9
:10B010008B7F80932804129A0895EAE5FEE18491DB
:10B02000EF012196882319F0A4D9FE01F8CFE5E4B9
:10B03000F7E18491EF012196882319F09AD9FE0156
:10B04000F8CF0E94639BCEDFE1E4F7E18491EF014A
:10B05000882349F0082E000C990B0E94A792219694
:10B06000FE018491F5CF8DE090E00E94A7928AE0E6
:10B0700090E00E94A792FFEF2BE48DE1F150204079
:10B080008040E1F700C00000F8949FEFE4E3FCE0AB
:10B090009150E040F040E1F700C000000E94639B47
:10B0A000A895FECF2F923F924F925F926F927F9220
:10B0B0008F929F92AF92BF92CF92DF92EF92FF92C8
:10B0C0000F931F93CF93DF9300D01F92CDB7DEB7BE
:10B0D0000E9414310E9402C56B017C011091220272
:10B0E000112309F475C08091C505882309F470C047
:10B0F0004091FC055091FD056091FE057091FF05A2
:10B1000046015701841A950AA60AB70AB7FC72C00D
:10B11000833041F134F481300CF45AC0EFE6FEE1A3
:10B1200006C0843009F054C0EFE6FEE137C08491D8
:10B130009F012F5F3F4F3B832A83882321F019D93A
:10B14000EA81FB81F4CFEFEBF6E184919F012F5F61
:10B150003F4F3B832A83882309F43AC00AD9EA8106
:10B16000FB81F3CFEFE6FEE184919F012F5F3F4F1C
:10B170003B832A83882321F0FCD8EA81FB81F4CF2A
:10B18000E8EAF6E184919F012F5F3F4F3B832A83DA
:10B190008823F1F0EED8EA81FB81F4CF84919F01FE
:10B1A0002F5F3F4F3B832A83882321F0E2D8EA8137
:10B1B000FB81F4CFE0E9F6E184919F012F5F3F4FDF
:10B1C0003B832A83882321F0D4D8EA81FB81F4CF02
:10B1D000212F30E0A8EEB3E00E94A7D9C60ED71EFB
:10B1E000E81EF91EC092FC05D092FD05E092FE0516
:10B1F000F092FF0589B182FB882780F98093E40EE5
:10B200009091E50E98170CF049C08091E60E909150
:10B21000E70EA091E80EB091E90E0196A11DB11DB7
:10B22000883B3DE39307A105B1054CF48093E60EFE
:10B230009093E70EA093E80EB093E90E3BC01092F6
:10B24000E60E1092E70E1092E80E1092E90E809131
:10B25000890A882319F00E940F941DC0E1EDF6E1E0
:10B260008491FB83EA83882371F0082E000C990BEC
:10B270000E94A7922A813B812F5F3F4F3B832A8305
:10B28000F9018491F0CF8DE090E00E94A7928AE0CE
:10B2900090E00E94A7928091E40E0AC0891751F0B5
:10B2A0001092E60E1092E70E1092E80E1092E90E40
:10B2B0008093E50E80910418843008F4DED80E9453
:10B2C00002C5C090CA05D090CB05E090CC05F090A7
:10B2D000CD05C114D104E104F10479F10091C60552
:10B2E0001091C7052091C8053091C9050C0D1D1D91
:10B2F0002E1D3F1D4B015C01801A910AA20AB30A60
:10B30000B7FC1BC0EAE5FEE184919F012F5F3F4F30
:10B310003B832A83882321F02CD8EA81FB81F4CF58
:10B320006091F3177091F41787E097E10E9453B78B
:10B330008AE01FD88EEF96E181C0C0902302D090A2
:10B340002402E0902502F0902602C114D104E10409
:10B35000F104E9F130910B0A20910C0A321749F0FF
:10B360006093C6057093C7058093C8059093C9057F
:10B370002EC00091C6051091C7052091C8053091D7
:10B38000C9050C0D1D1D2E1D3F1DDC01CB01801BB1
:10B39000910BA20BB30BB7FD1AC05F9A80912804E2
:10B3A0008E7F809328048A9A479A809128048D7F03
:10B3B0008093280480910801809581708093060114
:10B3C000479A809128048B7F80932804129A809159
:10B3D0000C0690910D06909902C0019604C01816B3
:10B3E00019062CF4019790930D0680930C0680911A
:10B3F0000C0690910D068E3E92400CF1EAE5FEE1BE
:10B4000084919F012F5F3F4F3B832A83882329F03C
:10B410000E94B951EA81FB81F3CFEEEDF6E1849110
:10B420009F012F5F3F4F3B832A83882329F00E948F
:10B43000B951EA81FB81F3CF85ED96E1EEDD0E9403
:10B4400002C5009108061091090620910A06309164
:10B450000B064B015C01801A910AA20AB30AB7FCE1
:10B460004EC08B019C010C53164F2F4F3F4F009342
:10B4700008061093090620930A0630930B064F9B8B
:10B48000A9C17A9BA7C12091060120FFA3C12091E9
:10B490005B1021119FC1379B9DC1379B9BC1029BB4
:10B4A00099C100910406109105062091060630917D
:10B4B0000706011511052105310599F0DC01CB01C5
:10B4C000801B910BA20BB30B80569A4EA109B109B8
:10B4D0008827B7FD83959927AA27BB27682F6195F1
:10B4E00001C060E0262F30E080910201611180955B
:10B4F000807180930001B90187E00E9403C490919C
:10B500000B0A80910C0A981791F0E0910C0A28E63A
:10B51000E29FF0011124E053FE4E608180910C0AFD
:10B5200090910B0A981729F08F5F8F70F9CF609177
:10B53000390470E089E00E9403C48091561088238A
:10B5400009F4F8C000914302109144028090450232
:10B550008C82909046029A826091410470914204DC
:10B560006E5F7F4F072E000C880B990B0E9493D5BE
:10B570009801A4010E948DD587FDDCC0F0900C0AD3
:10B58000212C312CE12C198280910B0A8F1509F4A2
:10B5900062C08F2D90E038E6A32EA89EF001A99EF0
:10B5A000F00D1124E259FE4E458956896789708D48
:10B5B000452B462B472B81F4418D528D638D748D25
:10B5C000452B462B472B41F4458D568D678D70A139
:10B5D000452B462B472BD1F128E6B22EB89E900181
:10B5E000B99E300D1124C90182599E4E6C01FC0197
:10B5F00061817281838194810E9422DC4B015C0114
:10B60000F60161A172A183A194A10E9491D52B01A1
:10B610003C01F60165A176A187A190A50E9491D574
:10B620009B01AC01C301B2010E9493DAA501940110
:10B630000E94F2D55B016C0191014E2D59810E944F
:10B64000DDDB18161CF41501EC2CD98281E08F0D7E
:10B650008F70F82E99CF2091470230914802409187
:10B66000490250914A02B1018E2D99810E94F2D572
:10B6700098014C815A810E94B7D96B017C019B01D2
:10B68000AC01B8018C819A810E94DDDB1816ACF008
:10B6900000913F0210914002809041028C82909074
:10B6A00042029A829801A401B601C7010E94DDDB23
:10B6B00018161CF08601EC82FA82C0900006D09029
:10B6C0000106E0900206F090030698014C815A8131
:10B6D000C701B6010E94DDDB1816D4F420E037ED77
:10B6E00043EA5CE3B8018C819A810E94F2D54B0158
:10B6F0005C0128E431EE4AE75FE3C701B6010E942E
:10B70000F2D5A50194010E94B7D98B018C839A834D
:10B71000C801AC81BA818093000690930106A09382
:10B720000206B0930306B801CD010E94FBDACB01FB
:10B730000E9445910E94239E89E69AE00E94FA4C5D
:10B74000A090D205A982AA2009F44DC00E9402C58A
:10B750000091CE051091CF052091D0053091D105F3
:10B76000DC01CB01801B910BA20BB30BB7FD3BC0DF
:10B770000E9402C56B017C01B9802B2D30E0A8EE40
:10B78000B3E00E94A7D9C60ED71EE81EF91EC092CC
:10B79000CE05D092CF05E092D005F092D1050E945F
:10B7A00065988AE00F900F900F900F90DF91CF91E6
:10B7B0001F910F91FF90EF90DF90CF90BF90AF90CF
:10B7C0009F908F907F906F905F904F903F902F90C1
:10B7D0000C94B95160930406709305068093060695
:10B7E000909307065ECE0F900F900F900F90DF9111
:10B7F000CF911F910F91FF90EF90DF90CF90BF906E
:10B80000AF909F908F907F906F905F904F903F9000
:10B810002F9008955F988A984798809108018170C9
:10B8200080930601479812980895CF93DF9380E0A4
:10B830000E9467A9C8EBD5E0688379838A839B83DC
:10B8400081E00E9467A96C837D838E839F8382E061
:10B850000E9467A9688779878A879B87DF91CF9144
:10B860000895CF92DF92EF92FF92CF93DF932091D2
:10B870002102222309F485C0EC01C090AC05D090D0
:10B88000AD05E090AE05F090AF05A7019601688187
:10B8900079818A819B810E948DD587FF04C0C882EF
:10B8A000D982EA82FB82C090B005D090B105E090C9
:10B8B000B205F090B305A70196016C817D818E8160
:10B8C0009F810E948DD587FF04C0CC82DD82EE82ED
:10B8D000FF82C0901502D0901602E0901702F090FF
:10B8E0001802A7019601688179818A819B810E9453
:10B8F000DDDB181624F4C882D982EA82FB82C0906C
:10B900001902D0901A02E0901B02F0901C02A701CD
:10B9100096016C817D818E819F810E94DDDB1816EE
:10B9200024F4CC82DD82EE82FF82C090B405D090F8
:10B93000B505E090B605F090B705A70196016885BA
:10B9400079858A859B850E948DD587FF04C0C8862E
:10B95000D986EA86FB86C0901D02D0901E02E09038
:10B960001F02F0902002A7019601688579858A85DB
:10B970009B850E94DDDB181624F4C886D986EA86EA
:10B98000FB86DF91CF91FF90EF90DF90CF900895ED
:10B990002F923F924F925F926F927F928F929F92DF
:10B9A000AF92BF92CF92DF92EF92FF920F931F93CD
:10B9B000CF93DF93CDB7DEB7CC54D1090FB6F8944F
:10B9C000DEBF0FBECDBF80EE95E04BDF80914B0612
:10B9D00083FDA9C0C090EC05D090ED05E090EE0588
:10B9E000F090EF05209135043091360440913704F2
:10B9F00050913804C701B6010E948DD5882309F4FF
:10BA000092C080914A06811133C0609143047091C5
:10BA1000440480914504909146040E94FBDA2091F1
:10BA20002B0230912C026217730714F5C092350473
:10BA3000D0923604E0923704F0923804EFE6FEE14B
:10BA400084917F019FEFE91AF90A882321F00E946F
:10BA5000B951F701F5CFE5E7F6E184917F01AFEF4A
:10BA6000EA1AFA0A882321F00E94B951F701F5CFAA
:10BA70008090EC059090ED05A090EE05B090EF055C
:10BA800020913504309136044091370450913804A8
:10BA9000C501B4010E94B6D96B017C0120E030E001
:10BAA000A9010E94DDDB87FF04C0F7FAF094F7F8E4
:10BAB000F094E091C405B4E0EB9FF0011124E95D3E
:10BAC000FD4F2081318142815381C701B6010E941F
:10BAD000F2D520E030E048E453E40E94DDDB1816A4
:10BAE00014F58092350490923604A0923704B092F7
:10BAF0003804EFE6FEE184917F019FEFE91AF90A2D
:10BB0000882321F00E94B951F701F5CFE6E5F6E16F
:10BB100084917F01AFEFEA1AFA0A882321F00E948C
:10BB2000B951F701F5CF8091FD1760900202709036
:10BB30000302C090E005D090E105E090E205F090AE
:10BB4000E3058090E4059090E505A090E605B090AF
:10BB5000E705882309F481C22090FE173090FF1773
:10BB6000409000185090011820E030E0A901C20177
:10BB7000B1010E948DD5882379F02091E80530919C
:10BB8000E9054091EA055091EB05C201B1010E941F
:10BB9000DDDB18160CF061C2B301770C880B990B32
:10BBA0000E9493D520914B0230914C0240914D025E
:10BBB00050914E020E94F2D52AE037ED43E25CE359
:10BBC0000E94F2D56DA77EA78FA798AB209129047C
:10BBD00030912A0440912B0450912C04C701B601E6
:10BBE0000E94B6D92B013C0120912D0430912E04E6
:10BBF00040912F0450913004C501B4010E94B6D980
:10BC000025966CAF7DAF8EAF9FAF259720E030E0DB
:10BC1000A901C301B2010E948DD5811141C020E06C
:10BC200030E0A90125966CAD7DAD8EAD9FAD259719
:10BC30000E948DD5811134C07090C40519AA1AAA2A
:10BC40001BAA1CAAC982DA82EB82FC828D829E82A8
:10BC5000AF82B8868091E8059091E905A091EA0548
:10BC6000B091EB0589879A87AB87BC87AE01475FA8
:10BC70005F4FBE016B5F7F4FCE0101960E94B2AE57
:10BC8000FE01F1966F01E72C8E01035D1F4F2CEE34
:10BC900035E0AE01475F5F4FBE016B5F7F4F2AC249
:10BCA0002091310430913204409133045091340496
:10BCB0006091E8057091E9058091EA059091EB05A6
:10BCC0000E94B6D929966CAF7DAF8EAF9FAF2997F2
:10BCD0002091350430913604409137045091380456
:10BCE0006091EC057091ED058091EE059091EF0566
:10BCF0000E94B6D921966CAF7DAF8EAF9FAF2197D2
:10BD0000A3019201C301B2010E94F2D56B017C0133
:10BD100025962CAD3DAD4EAD5FAD2597CA01B9015D
:10BD20000E94F2D59B01AC01C701B6010E94B7D9B0
:10BD30006B017C0129962CAD3DAD4EAD5FAD2997D1
:10BD4000CA01B9010E94F2D59B01AC01C701B6013D
:10BD50000E94B7D90E9422DC6B017C012DEB37E3F6
:10BD600046E855E30E948DD587FF17C020E030E0FC
:10BD7000A90121966CAD7DAD8EAD9FAD21970E943E
:10BD8000DDDB2196CCACDDACEEACFFAC219787FFC0
:10BD900004C0F7FAF094F7F8F0942DEB37E346E897
:10BDA00055E3C701B6010E948DD587FDA6C120E0ED
:10BDB00030E040EA50E4C701B6010E9493DA0E94E5
:10BDC00000DB1B01672B19F422242394312CB101D1
:10BDD00080E090E00E9491D59B01AC0160E070E0B2
:10BDE00080E89FE30E9493DA4B015C019B01AC0168
:10BDF000C701B6010E94F2D52D966CAF7DAF8EAF14
:10BE00009FAF2D97A5019401C301B2010E94F2D505
:10BE1000698B7A8B8B8B9C8BA501940125966CADDD
:10BE20007DAD8EAD9FAD25970E94F2D56D8B7E8B3B
:10BE30008F8B988FA501940129966CAD7DAD8EAD49
:10BE40009FAD29970E94F2D5698F7A8F8B8F9C8F37
:10BE5000A501940121966CAD7DAD8EAD9FAD21976E
:10BE60000E94F2D56D8F7E8F8F8F98A380E1E9E2DB
:10BE7000F4E0DE01119601900D928A95E1F7992484
:10BE80009394F1E02F1A310809F04BC0E090C405FB
:10BE90002D968CAD9DADAEADBFAD2D9789AF9AAF50
:10BEA000ABAFBCAF8091E0059091E105A091E205B8
:10BEB000B091E30589A39AA3ABA3BCA38091E40549
:10BEC0009091E505A091E605B091E7058DA39EA3AD
:10BED000AFA3B8A78091E8059091E905A091EA0584
:10BEE000B091EB0589A79AA7ABA7BCA7AE01475DA8
:10BEF0005F4FBE016B5D7F4FCE0181960E94B2AE57
:10BF0000DE01D9966D018E01035D1F4F2CEE35E0E9
:10BF1000AE01475D5F4FBE016B5D7F4FCE018196E5
:10BF2000EBC08091F405811112C00E9402C5DC01B2
:10BF3000CB0188539F4FAF4FBF4F8093F005909335
:10BF4000F105A093F205B093F3059092F4050E94D9
:10BF5000239E0E9402C5C090F005D090F105E090AC
:10BF6000F205F090F305DC01CB018C199D09AE09B7
:10BF7000BF09B7FD11C00E9402C5DC01CB01885387
:10BF80009F4FAF4FBF4F8093F0059093F105A09363
:10BF9000F205B093F30586D86E01B1E1CB0ED11C4A
:10BFA000FE0131967F015601D6012D913D914D91B3
:10BFB0005D916D01F70160817181828193810E94A1
:10BFC000B7D9D7016D937D938D939D937D01AA166B
:10BFD000BB0651F7E090C4052D968CAD9DADAEAD7E
:10BFE000BFAD2D978DAB9EABAFABB8AF89819A81BA
:10BFF000AB81BC8189A39AA3ABA3BCA38D819E8195
:10C00000AF81B8858DA39EA3AFA3B8A789859A8574
:10C01000AB85BC8589A79AA7ABA7BCA7AE01475D36
:10C020005F4FBE016B5D7F4FCE0181960E94B2AE25
:10C03000DE01D5966D018E01035D1F4F9E01235FCA
:10C040003F4FAE01475D5F4FBE016B5D7F4FCE013D
:10C050008196BAD0811115CF19CFB301770C880B17
:10C06000990B0E9493D520914B0230914C02409144
:10C070004D0250914E020E94F2D52AE037ED43E284
:10C080005CE30E94F2D569AB7AAB8BAB9CAB709052
:10C09000C4058091E8059091E905A091EA05B09169
:10C0A000EB05C982DA82EB82FC82898A9A8AAB8AA2
:10C0B000BC8A89A39AA3ABA3BCA31DA61EA61FA6D8
:10C0C00018AAAE014F5D5F4FBE016F5E7F4FCE017C
:10C0D00001960E94B2AEFE01BD966F01E72C8E0163
:10C0E0000F5C1F4F2CEE35E0AE014F5D5F4FBE0180
:10C0F0006F5E7F4FCE01019667D080E1E0EEF5E004
:10C10000A9E2B4E001900D928A95E1F7C45BDF4F9C
:10C110000FB6F894DEBF0FBECDBFDF91CF911F9158
:10C120000F91FF90EF90DF90CF90BF90AF909F90D6
:10C130008F907F906F905F904F903F902F900895D9
:10C14000CF93DF93E0910218F0E0EB58F94F808134
:10C15000882381F0E3E5F6E18491EF0121968823BD
:10C1600021F00E94B951FE01F7CF8AE0DF91CF9113
:10C170000C94B951DF91CF910895CF93DF938091C3
:10C18000AA058093AB05EAE4F6E18491EF012196DC
:10C19000882321F00E94B951FE01F7CF8091101839
:10C1A00090911118A0911218B0911318BC01CD01F3
:10C1B0006F5F7F4F8F4F9F4F0E9446558AE00E94CE
:10C1C000B951DF91CF91BCCF2F923F924F925F92A6
:10C1D0006F927F928F929F92AF92BF92CF92DF9297
:10C1E000EF92FF920F931F93CF93DF93CDB7DEB7FC
:10C1F000C857D1090FB6F894DEBF0FBECDBFE0918E
:10C200005810F0915910EF2B11F00C94A469289656
:10C21000DFAECEAE28976E2C79016A015B01FC017E
:10C2200020813181428153816C962CAF3DAF4EAF5E
:10C230005FAF6C9720915E1130915F11409160115A
:10C24000509161116C966CAD7DAD8EAD9FAD6C97CC
:10C250000E94F2D50E94E8DBE0966CAF7DAF8EAF16
:10C260009FAFE097D5018D919D910D90BC91A02D30
:10C27000A0968CAF9DAFAEAFBFAFA09720916211DB
:10C28000309163114091641150916511BC01CD0151
:10C290000E94F2D50E94E8DBE4966CAF7DAF8EAFD2
:10C2A0009FAFE497D6012D913D914D915C91A4965D
:10C2B0002CAF3DAF4EAF5FAFA49720916611309188
:10C2C00067114091681150916911A4966CAD7DADD4
:10C2D0008EAD9FADA4970E94F2D50E94E8DBE89650
:10C2E0006CAF7DAF8EAF9FAFE897D7012D913D9199
:10C2F0004D915C9122962CAF3DAF4EAF5FAF229730
:10C3000020916A1130916B1140916C1150916D1117
:10C3100022966CAD7DAD8EAD9FAD22970E94F2D579
:10C320000E94E8DB60966CAF7DAF8EAF9FAF6097E9
:10C3300080914B0683FF1CC060962CAD3DAD4EAD89
:10C340005FAD609720933D0A30933E0A40933F0AC9
:10C350005093400A22968CAD9DADAEADBFAD2297F5
:10C3600080932D0A90932E0AA0932F0AB093300A3F
:10C37000D801BC91B9A7F801F181F9ABD8011296A7
:10C38000BC91BEABF801F381FAAF80910B0A90919A
:10C390000C0A891B8F708F3019F40E945258F5CF08
:10C3A00000910B0AE9960FAFE99780910B0A082FCD
:10C3B00010E01CA30BA38091310A9091320AA09146
:10C3C000330AB091340AE0968CAC9DACAEACBFACF5
:10C3D000E097881A990AAA0ABB0A8091350A9091B7
:10C3E000360AA091370AB091380AE4962CAC3DACDD
:10C3F0004EAC5FACE497281A390A4A0A5B0A80916E
:10C40000390A90913A0AA0913B0AB0913C0AE89609
:10C410002CAD3DAD4EAD5FADE897281B390B4A0BF7
:10C420005B0B2DA33EA34FA358A780913D0A90918B
:10C430003E0AA0913F0AB091400A60960CAD1DAD36
:10C440002EAD3FAD6097081B190B2A0B3B0B0DA7B8
:10C450001EA72FA738AB012B022B032B09F4BCC05E
:10C4600080914A0681114BC060914304709144044D
:10C4700080914504909146040E94FBDA20912B02A2
:10C4800030912C02621773070CF039C060962CAD06
:10C490003DAD4EAD5FAD609720933D0A30933E0AAF
:10C4A00040933F0A5093400A22968CAD9DADAEADAD
:10C4B000BFAD229780932D0A90932E0AA0932F0A46
:10C4C000B093300AEFE6FEE184918F010F5F1F4FBA
:10C4D000811103C0E0EDF7E104C00E94B951F801F9
:10C4E000F3CF84918F010F5F1F4F882321F00E94AB
:10C4F000B951F801F6CF1DA61EA61FA618AA94E0F2
:10C50000699E80011124095D1D4F6DA57EA58FA533
:10C5100098A90E9493D5D8012D913D914D915C91A0
:10C520000E94F2D56B017C0120E030E0A9010E945D
:10C53000DDDB87FF04C0F7FAF094F7F8F094609120
:10C540006A1170916B1180916C1190916D110E9424
:10C55000FBDA9B01AC01A8ECB0E00E949DD90E94DF
:10C5600093D5A70196010E948DD587FF39C06096AB
:10C570000CAD1DAD2EAD3FAD609700933D0A1093FD
:10C580003E0A20933F0A3093400A22962CAD3DADDF
:10C590004EAD5FAD229720932D0A30932E0A409323
:10C5A0002F0A5093300AEFE6FEE184918F010F5F6E
:10C5B0001F4F811103C0E1EBF7E104C00E94B951A4
:10C5C000F801F3CF84918F010F5F1F4F882321F073
:10C5D0000E94B951F801F6CF1DA61EA61FA618AAE3
:10C5E000D501C4018827B7FD83959927AA27BB27C2
:10C5F000782E57FE03C0382F3260732E8DA19EA176
:10C60000AFA1B8A5B7FF03C0972D9460792E0DA5F3
:10C610001EA52FA538A937FF03C0172D1860712E4E
:10C6200024E0629E80011124095D1D4F6DA57EA549
:10C630008FA598A90E9493D5D8012D913D914D9138
:10C640005C910E94F2D56B017C0120E030E0A901F1
:10C650000E94DDDB87FF04C0C701B601905802C00D
:10C66000C701B60120E030E040E05FE30E94B7D9A7
:10C670000E9400DB6AAB7BAB8CAB9DAB88E60BA169
:10C680001CA1809FF001819FF00D1124E259FE4E04
:10C690001082EA5BFF4F7082B501A401B7FE07C0AC
:10C6A00044275527BA01481959096A097B0988E6C0
:10C6B0000BA11CA1809FF001819FF00D1124E25974
:10C6C000FE4E458B568B678B708F2C962CAE3DAEF5
:10C6D0004EAE5FAE2C9757FE0DC088279927DC0120
:10C6E00082199309A409B5092C968CAF9DAFAEAF02
:10C6F000BFAF2C9728E60BA11CA1209FF001219F22
:10C70000F00D1124E259FE4E2C968CAD9DADAEADD0
:10C71000BFAD2C97818F928FA38FB48F0DA11EA1D7
:10C720002FA138A537FF07C03095209510950195AA
:10C730001F4F2F4F3F4FE8E67E2EABA1BCA17A9E44
:10C74000F0017B9EF00D1124E259FE4E058F168FED
:10C75000278F30A38AA99BA9ACA9BDA981A392A3C5
:10C76000A3A3B4A323964FAF2397752EF62FE72FDD
:10C770002C968CAD9DADAEADBFAD2C97481759072B
:10C780006A077B0778F429969FAD299723969FAF78
:10C7900023972A967FAC2A972B96FFAD2B972C9642
:10C7A000EFAD2C9723968FAD2397972DAF2FBE2FEC
:10C7B00080179107A207B30710F4D901C8010AA98D
:10C7C0001BA92CA93DA980179107A207B30710F454
:10C7D000D901C80128E60BA11CA1209FF001219FCF
:10C7E000F00D1124E259FE4E85A396A3A7A3B0A78E
:10C7F0000697A105B10508F4A0C5DF01AE59BF4FEA
:10C800008091390490913A048D939C9361A6452BB5
:10C81000462B472B09F05F9888E60BA11CA1809F4F
:10C82000F001819FF00D1124E259FE4E818D928D11
:10C83000A38DB48D892B8A2B8B2B11F08A98479866
:10C8400088E60BA11CA1809FF001819FF00D1124AF
:10C85000E259FE4E858D968DA78DB0A1892B8A2B2E
:10C860008B2B31F0809108018170809306014798ED
:10C870002AA93BA94CA95DA9232B242B252B09F41C
:10C8800065C580915006882319F081508093500629
:10C89000611004C0129880E28093500660904606B2
:10C8A0007090470600914806109149069301A8012F
:10C8B00069A579A98EA99AAD0E948DD587FF04C07C
:10C8C00069A679AA0EAB1AAFC501B4010E9493D52F
:10C8D00020914E1130914F114091501150915111B2
:10C8E0000E94F2D526966CAF7DAF8EAF9FAF269794
:10C8F000698B7A8B8B8B9C8BC201B1010E9493D583
:10C900002091521130915311409154115091551171
:10C910000E94F2D52B013C016D8B7E8B8F8B988F03
:10C920006DA17EA18FA198A50E9493D5209156114B
:10C930003091571140915811509159110E94F2D5E0
:10C940004B015C01698F7A8F8B8F9C8F20915A11DC
:10C9500030915B1140915C1150915D11C701B6019E
:10C960000E94F2D56B017C016D8F7E8F8F8F98A313
:10C9700088E60BA11CA1809FF001819FF00D11247E
:10C98000E259FE4E258936894789508D2DA33EA355
:10C990004FA358A7263031054105510508F4DFC4DF
:10C9A0002896AEADBFAD2897CD90DD90ED90FC9070
:10C9B00020E030E0A901C701B6010E948DD58111A8
:10C9C000EDC426962CAD3DAD4EAD5FAD2697CA01A8
:10C9D000B9010E94F2D56B017C01A3019201C30150
:10C9E000B2010E94F2D59B01AC01C701B6010E94C1
:10C9F000B7D96B017C01A5019401C501B4010E9466
:10CA0000F2D59B01AC01C701B6010E94B7D90E94C3
:10CA100022DC28E60BA11CA1209FF001219FF00D34
:10CA20001124E259FE4E658776878787908B88E6CA
:10CA30000BA11CA1809FF001819FF00D1124E259F0
:10CA4000FE4E4584568467847088A301920160E09D
:10CA500070E080E89FE30E9493DA64966CAF7DAF4C
:10CA60008EAF9FAF649729A539A94EA95AAD0E94F0
:10CA7000F2D54B015C0180910B0A9091090A891B48
:10CA80008F7027968FAF2797A501940160E074E21D
:10CA900084E799E40E9493DA0E94E8DB6B017C0151
:10CAA00027968FAD27978250863008F486C4A5015B
:10CAB0009401C301B2010E94F2D59B01AC010E9416
:10CAC000F2D568966CAF7DAF8EAF9FAF689788E662
:10CAD000ABA1BCA18A9F80018B9F100D112402592C
:10CAE0001E4E68962CAD3DAD4EAD5FAD6897D8013A
:10CAF00011962D933D934D935C93149795962D919C
:10CB00003D914D915C9198972EAB3FAB48AF59AF9B
:10CB1000CA01B9010E9491D56AAF7BAF8CAF9DAFBE
:10CB20009B01AC01C501B4010E94F2D50E947DDADF
:10CB30000E9400DBA8966CAF7DAF8EAF9FAFA89729
:10CB4000F801EE5AFF4F60837183828393838E01D5
:10CB50000F5E1F4F2A961FAF0EAF2A970051110983
:10CB600024961FAF0EAF24970EE216E0AC961FAFCF
:10CB70000EAFAC978E010F5D1F4F1AA309A3249629
:10CB80000EAD1FAD2497AA961FAF0EAFAA97312CFA
:10CB9000212C10E819A70FE309AB2A96AEADBFAD63
:10CBA0002A972D913D914D915D912A96BFAFAEAFE1
:10CBB0002A97C501B4010E94F2D56B017C01AA96A7
:10CBC000EEADFFADAA976193719381939193AA966D
:10CBD000FFAFEEAFAA9720E030E0A9010E94DDDBB5
:10CBE00087FF04C0F7FAF094F7F8F094AC96AEAD76
:10CBF000BFADAC974D905D906D907D90AC96BFAF02
:10CC0000AEAFAC97A7019601C301B2010E948DD5CA
:10CC100087FD0DC409A11AA12A962EAD3FAD2A9712
:10CC20000217130709F0B9CF20E030E040E85FE3D6
:10CC3000632D722D89A599A90E948DD587FF58C0B3
:10CC40007E0131E1E30EF11C24960EAD1FAD249759
:10CC5000232D322D49A559A9D8016D917D918D9132
:10CC60009C910E94F2D5F801619371938193919305
:10CC70008F01EE16FF0661F728E60BA11CA1209F8D
:10CC8000C001219F900D11249C0122593E4E790133
:10CC900089010E5A1F4FA8966CAD7DAD8EAD9FAD2C
:10CCA000A8970E9491D5232D322D49A559A90E94FC
:10CCB000F2D50E9400DBD8016D937D938D939C93F8
:10CCC0001397232D322D49A559A9632D722D89A5BE
:10CCD00099A90E94F2D568962CAD3DAD4EAD5FADE1
:10CCE00068970E94F2D5F7016183728383839483EE
:10CCF0002AAD3BAD4CAD5DAD64966CAD7DAD8EADFA
:10CD00009FAD64970E94F2D569A77AA78BA79CA7CD
:10CD10000DA11EA12FA138A5012B022B032B09F079
:10CD20009EC388E62BA13CA1829F8001839F100DAA
:10CD3000112402591E4EF801818D928DA38DB48D60
:10CD4000892B8A2B8B2B09F08AC3858D968DA78D15
:10CD5000B0A1892B8A2B8B2B09F081C320912A0645
:10CD600030912B0640912C0650912D0669A57AA58D
:10CD70008BA59CA50E94F2D50E947DDA0E9400DB63
:10CD80002B013C01F801E95BFF4F108288E62BA1E3
:10CD90003CA1829F8001839F100D112402591E4ED9
:10CDA000F801E25AFF4F4082518262827382C301CE
:10CDB000B2010E9491D529A53AA54BA55CA50E9478
:10CDC00093DA6AAF7BAF8CAF9DAFD80151966D936C
:10CDD0007D938D939C935497F801E95BFF4F80817D
:10CDE000882381F17801B8E4EB0EF11C379620918D
:10CDF0001E0630911F064091200650912106608149
:10CE00007181828193810E94F2D52AAD3BAD4CADF8
:10CE10005DAD0E94F2D520916A1130916B11409165
:10CE20006C1150916D110E94F2D59B01AC0160E034
:10CE300074E284EF99E40E9493DA0E9400DBF70128
:10CE40007183608388E60BA11CA1809FF001819F04
:10CE5000F00D1124E259FE4E21813281438154812B
:10CE60002C962CAF3DAF4EAF5FAF2C97CA01B901E6
:10CE70000E9422DC362E272E8C014EE056E0629670
:10CE80005FAF4EAF62973E0151E1650E711C8EE0BF
:10CE900096E09FAB8EAB24964EAC5FAC24973DA63C
:10CEA0002DA209A719AB1AAAD201CD90DD90ED9061
:10CEB000FD902D0120E030E0A901C701B6010E94DC
:10CEC000DDDB87FF04C0F7FAF094F7F8F094EEA9E1
:10CED000FFA981909190A190B190FFABEEABA7011B
:10CEE0009601C501B4010E948DD587FDD8C5641493
:10CEF0007504D1F627965FAD2797552309F448C6E8
:10CF0000C0900D0AD0900E0AE0900F0AF090100A1F
:10CF10002DEB37E346E855E3C701B6010E948DD5F6
:10CF200087FD36C6C701B6010E9422DC6B017C0179
:10CF30009B01AC01632D722DC8010E948DD587FD28
:10CF400003C03C2C2D2C87019601A701632D722D67
:10CF5000C8010E9493DA68966CAF7DAF8EAF9FAF29
:10CF6000689781E19AE028969FAF8EAF289720E0DE
:10CF700030E040E85FE32AAB3BAB4CAB5DAB1EAAB5
:10CF80002896AEADBFAD28972D913D914D915D9105
:10CF90002896BFAFAEAF289768966CAD7DAD8EADCD
:10CFA0009FAD68970E94F2D54B015C012496EEADCF
:10CFB000FFAD2497C190D190E190F1902496FFAFFE
:10CFC000EEAF2497FEA9FF2391F02AA93BA94CA913
:10CFD0005DA90E94F2D54B015C012AA93BA94CA98D
:10CFE0005DA9C701B6010E94F2D56B017C01A701C2
:10CFF0009601C501B4010E94DDDB20E030E0A9010B
:10D0000018160CF092C5C701B6010E94DDDB181698
:10D010000CF486C520E030E0A901C501B4010E94EE
:10D020008DD587FD7DC52601370177FA709477F895
:10D030007094A3019201C501B4010E94DDDB1816B2
:10D0400014F4240135016296AEADBFAD6297CD9068
:10D05000DD90ED90FD906296BFAFAEAF6297A301F9
:10D060009201C701B6010E948DD587FF15C0A301AB
:10D070009201C701B6010E9493DA9B01AC016AA933
:10D080007BA98CA99DA90E94F2D56AAB7BAB8CAB26
:10D090009DABBEA9BF5FBEABE1E2FAE028962EAD24
:10D0A0003FAD2897E217F30709F06ACF3EA9332373
:10D0B00061F02AA93BA94CA95DA9632D722DC80175
:10D0C0000E94F2D5362E272E8C0124EA30E74DE758
:10D0D0005FE3632D722DC8010E94F2D56B017C01C4
:10D0E00020914C0630914D0640914E0650914F06CE
:10D0F0000E948DD587FD42C58DA59DA1A9A5B9A981
:10D1000080934C0690934D06A0934E06B0934F0625
:10D1100028E64BA15CA1249FC001259F900D1124FE
:10D12000DC01A259BE4E7D01232D322DA801632DB5
:10D13000722DC8010E94F2D5F7016187728783873B
:10D1400094876AAD7BAD8CAD9DAD90589B01AC01D1
:10D150000E94B7D9D7011D962D913D914D915C91BB
:10D1600050970E94F2D59B01AC016BE077ED83E212
:10D170009BE30E94B6D99B01AC018BE097EDA3E243
:10D18000BBE3F70185839683A783B08710812C9634
:10D190006CAD7DAD8EAD9FAD2C970E948DD51816D0
:10D1A0000CF4FBC483E0182B88E62BA13CA1829FE2
:10D1B000F001839FF00D1124E259FE4E108380E1AF
:10D1C000FE013196A1E1BAE001900D928A95E1F756
:10D1D0002C968CAD9DADAEADBFAD2C9780930D0A56
:10D1E00090930E0AA0930F0AB093100AE0960CAD2C
:10D1F0001DAD2EAD3FADE0970093310A1093320A7A
:10D200002093330A3093340AE4962CAD3DAD4EADF5
:10D210005FADE4972093350A3093360A4093370A7E
:10D220005093380AE8968CAD9DADAEADBFADE89792
:10D230008093390A90933A0AA0933B0AB0933C0A30
:10D2400060960CAD1DAD2EAD3FAD609700933D0ACD
:10D2500010933E0A20933F0A3093400A6C962CADFF
:10D260003DAD4EAD5FAD6C972093210A3093220AFD
:10D270004093230A5093240AA0968CAD9DADAEAD89
:10D28000BFADA0978093250A9093260AA093270A02
:10D29000B093280AA4960CAD1DAD2EAD3FADA4975A
:10D2A0000093290A10932A0A20932B0A30932C0A00
:10D2B00022962CAD3DAD4EAD5FAD229720932D0A49
:10D2C00030932E0A40932F0A5093300A90910B0A04
:10D2D00080910C0A981303C084E68093080AE996AB
:10D2E0008FADE9978F5F8F7080930B0A80910B0A47
:10D2F00090910A0A81508F70891351C410910C0AC1
:10D300001BA300910B0A0DA728E61BA10DA5101366
:10D31000D1C4812C912CA12CB12C1DA219A619AA23
:10D320001EAE212C312C00E010E02DA53BA12313D3
:10D33000CEC42114310409F07FC580916F00826052
:10D3400080936F0081E0ECC680E0EAC66090420600
:10D35000709043060091440610914506A7CA818D3E
:10D36000928DA38DB48D0697A105B10508F018CB59
:10D37000858D968DA78DB0A10697A105B10508F002
:10D380000FCB20E030E0A901C701B6010E94DDDB30
:10D3900087FF04C0F7FAF094F7F8F09488E60BA141
:10D3A0001CA1809FF001819FF00D1124E259FE4ED7
:10D3B000C586D686E786F08A3ACB80913E06909164
:10D3C0003F06A0914006B0914106C816D906EA066C
:10D3D000FB0608F06CCB8C199D09AE09BF09BC0196
:10D3E000CD01660F771F881F991F27964FAD27978E
:10D3F000042F10E020E030E0A90198010E947BD9C1
:10D40000CA01B9010E9491D50E94E8DB6C0D7D1D17
:10D410008E1D9F1D0E9491D59B01AC0160E074E2BE
:10D4200084E799E40E9493DA4B015C0140CBA701A9
:10D430009601C301B2010E9493DA7B018C019B012A
:10D44000AC01632D722D89A599A90E94DDDB181608
:10D450000CF0E0CB3E2C2F2C09A719ABDBCB0AA993
:10D460001BA92CA93DA9012B022B032B49F02091CC
:10D47000260630912706409128065091290608C0BB
:10D4800020912206309123064091240650912506D2
:10D4900069A57AA58BA59CA50E94F2D50E947DDA8C
:10D4A0000E9400DB2B013C012AA93BA94CA95DA9E4
:10D4B000232B242B252BC9F020E030E0A90160911B
:10D4C0001E0670911F0680912006909121060E94F1
:10D4D0008DD5882351F081E00DA51EA52FA538A973
:10D4E00010161106120613060CF080E098E62BA128
:10D4F0003CA1929F8001939F100D112402591E4E52
:10D50000180137E4230E311CD1018C93882309F4D0
:10D51000B3C02091210A3091220A4091230A5091F0
:10D52000240A6C966CAD7DAD8EAD9FAD6C970E945C
:10D53000B6D96DA77EA78FA798AB2091250A309109
:10D54000260A4091270A5091280AA0966CAD7DAD1D
:10D550008EAD9FADA0970E94B6D94B015C01209182
:10D56000290A30912A0A40912B0A50912C0AA4963C
:10D570006CAD7DAD8EAD9FADA4970E94B6D96B0109
:10D580007C012DA53EA54FA558A9CA01B9010E944D
:10D59000F2D56DA77EA78FA798ABA5019401C50111
:10D5A000B4010E94F2D59B01AC016DA57EA58FA5AB
:10D5B00098A90E94B7D94B015C01A7019601C70148
:10D5C000B6010E94F2D59B01AC01C501B4010E94D5
:10D5D000B7D90E9422DC6B017C0120912D0A309189
:10D5E0002E0A40912F0A5091300A22966CAD7DADE3
:10D5F0008EAD9FAD22970E94B6D9A70196010E94D9
:10D6000093DA6B017C01F801E25BFF4F6083718369
:10D610008283938320E030E040E450E40E94DDDB2D
:10D6200018161CF4F101108227C020911E063091BB
:10D630001F064091200650912106C701B6010E94A5
:10D64000F2D59B01AC0160911A0670911B06809186
:10D650001C0690911D060E9493DA29A53AA54BA5B8
:10D660005CA50E94F2D50E9400DB64157505860555
:10D67000970510F42B013C0180912A1190912B11F8
:10D68000A0912C11B0912D110EA91FA928AD39AD73
:10D6900080179107A207B30708F4DFC02DA13EA1B0
:10D6A0004FA158A5232B242B252B41F160912E113E
:10D6B00070912F1180913011909131116415750581
:10D6C00086059705D8F42EA93FA948AD59AD0E940B
:10D6D0006CD96B017C012DA13EA14FA158A5C301BE
:10D6E000B2010E946CD9C616D706E806F90630F4D6
:10D6F000C701B6010E947BD929013A0188E60BA136
:10D700001CA1809FF001819FF00D1124E259FE4E73
:10D71000C18CD28CE38CF48CC114D104E104F104EB
:10D7200031F16091321170913311809134119091E7
:10D7300035116415750586059705C8F42EA93FA90E
:10D7400048AD59AD0E946CD94B015C01A70196010F
:10D75000C301B2010E946CD986169706A806B906C5
:10D7600030F4C501B4010E947BD929013A0188E651
:10D770000BA11CA1809FF001819FF00D1124E259A3
:10D78000FE4EC58CD68CE78CF0A0C114D104E10408
:10D79000F10431F160913611709137118091381197
:10D7A000909139116415750586059705C8F42EA961
:10D7B0003FA948AD59AD0E946CD94B015C01A7014E
:10D7C0009601C301B2010E946CD986169706A8067D
:10D7D000B90630F4C501B4010E947BD929013A0190
:10D7E00088E60BA11CA1809FF001819FF00D112400
:10D7F000E259FE4EC1A0D2A0E3A0F4A0C114D1040E
:10D80000E104F10409F4C2CA60913A1170913B112C
:10D8100080913C1190913D11641575058605970521
:10D8200008F0B4CA2EA93FA948AD59AD0E946CD9E1
:10D830004B015C01A7019601C301B2010E946CD9A2
:10D8400086169706A806B90608F0A0CAC501B40155
:10D850000E947BD929013A0199CA2DA13EA14FA16D
:10D8600058A5232B242B252BC9F160912E117091E3
:10D870002F11809130119091311164157505860535
:10D88000970560F50E9491D52AAD3BAD4CAD5DADDD
:10D890000E94F2D56B017C016DA17EA18FA198A59C
:10D8A0000E9491D54B015C01C301B2010E9491D548
:10D8B000A50194010E94F2D59B01AC01C701B601FC
:10D8C0000E948DD587FF0AC0A5019401C701B6014A
:10D8D0000E9493DA0E9400DB2B013C0188E60BA139
:10D8E0001CA1809FF001819FF00D1124E259FE4E92
:10D8F000818C928CA38CB48C81149104A104B1040A
:10D90000B9F160913211709133118091341190917D
:10D910003511641575058605970550F50E9491D55A
:10D920002AAD3BAD4CAD5DAD0E94F2D56B017C01E3
:10D93000C501B4010E9491D54B015C01C301B20144
:10D940000E9491D5A50194010E94F2D59B01AC01E2
:10D95000C701B6010E948DD587FF0AC0A5019401B9
:10D96000C701B6010E9493DA0E9400DB2B013C0143
:10D9700088E60BA11CA1809FF001819FF00D11246E
:10D98000E259FE4E858C968CA78CB0A08114910430
:10D99000A104B104B9F160913611709137118091F1
:10D9A000381190913911641575058605970550F564
:10D9B0000E9491D52AAD3BAD4CAD5DAD0E94F2D534
:10D9C0006B017C01C501B4010E9491D54B015C0142
:10D9D000C301B2010E9491D5A50194010E94F2D524
:10D9E0009B01AC01C701B6010E948DD587FF0AC01B
:10D9F000A5019401C701B6010E9493DA0E9400DBE1
:10DA00002B013C0188E60BA11CA1809FF001819FA6
:10DA1000F00D1124E259FE4EC1A0D2A0E3A0F4A063
:10DA2000C114D104E104F10409F4B0C960913A11C0
:10DA300070913B1180913C1190913D1164157505D9
:10DA40008605970508F0A2C90E9491D52AAD3BAD85
:10DA50004CAD5DAD0E94F2D54B015C01C701B60132
:10DA60000E9491D56B017C01C301B2010E9491D546
:10DA7000A70196010E94F2D59B01AC01C501B4013A
:10DA80000E948DD587FF82C9A7019601C501B40107
:10DA90000E9493DA0E9400DB2B013C0177C9FAA9AE
:10DAA000FF2331F1A5019401632D722DC8010E945D
:10DAB000F2D54B015C012DA53DA149A559A9C7018E
:10DAC000B6010E94F2D59B01AC01C501B4010E94D0
:10DAD0008DD587FF22C0A7019601C501B4010E9420
:10DAE00093DA6DA77DA389A799AB21E02AABFFC983
:10DAF000A7019601C501B4010E9493DA9B01AC0114
:10DB00006DA57DA189A599A90E94F2D56DA77DA3D8
:10DB100089A799AB31E03AABEAC941E04AABE7C922
:10DB2000A7019601C501B40113C0C701B6010E9447
:10DB30008DD587FD09C020E030E0A901C501B40101
:10DB40000E94DDDB18164CF4A5019401C701B60153
:10DB50000E94B6D92B013C0176CA2401350177FA1F
:10DB6000709477F87094A3019201C701B6010E94E6
:10DB70008DD587FD68CA2601370165CA2DA53DA14F
:10DB800049A559A9C701B6010E948DD587FFB4CA1E
:10DB90003DA42DA009A519A9AFCA81E004CBF0903E
:10DBA0000B0A8FEF8F0D8F708BA3B0900A0A8091B4
:10DBB0000B0AB81609F454C0C12CD12C0BA10B15BB
:10DBC00009F44EC0602E712C28E6269D8001279D09
:10DBD000100D112402591E4ED8018C9183FD2BC0CB
:10DBE0000EAF1AAB0115110541F11996BC91BDA7F5
:10DBF000F801F285FDA3D8011B96BC91B9A7F801E5
:10DC0000F485F9ABD80115962D903D904D905C9020
:10DC10001897A20191016DA57DA189A59F2F0E9452
:10DC20008DD5811186C1C114D10439F0F6018081EE
:10DC300080FD7FC102C0CEAEDAAA8BA181508F7069
:10DC40008BA380910A0A8B1103C0CEACDAA8B6CFA1
:10DC50000BA10B1529F081E08B0D8F70B82EF1CF41
:10DC600010910A0A1BA3C12CD12C80910B0A0BA185
:10DC7000801709F443CB802E912C28E6289D800143
:10DC8000299D100D112402591E4ED8018C9183FD3F
:10DC90000AC05801C114D10439F0C6010E949BA1E9
:10DCA000811102C0C5C156018BA18F5F8F708BA3FC
:10DCB0006501DBCF802F81508F70289FF0011124E8
:10DCC000E259FE4E908193FF24CB8DA71ECB48E6F0
:10DCD000439FC0011124DC01A259BE4E1D018C914D
:10DCE00083FD19C015966D917D918D919C9118972A
:10DCF0000E9422DCF62EE72ED82EC92E0115110522
:10DD000009F48CC0F801808180FD0AC0D1018C919A
:10DD100080FD06C083C0FDA0E9A4D9A8CEAC83C015
:10DD2000F801808181608083C8010E949BA18111DC
:10DD300071C0F80161817281838194810E9422DC2B
:10DD40002B013C019B01AC0160E070E080E89FE3A7
:10DD50000E9493DA4B015C019B01AC016F2D7E2D7B
:10DD60008D2D9C2D0E94F2D569837A838B839C83B1
:10DD70002DA139A549A95EADC501B4010E94F2D516
:10DD8000698B7A8B8B8B9C8BAE014F5F5F4FBE0193
:10DD90006F5E7F4FC8010E9437AAF801E95BFF4F11
:10DDA00080818823B9F120911E0630911F06409191
:10DDB000200650912106379660817181828193817E
:10DDC0000E94F2D520916A1130916B1140916C1133
:10DDD00050916D110E94F2D54B015C019B01AC0189
:10DDE000C301B2010E94F2D50E9400DBF801E65B9C
:10DDF000FF4F71836083A50194016F2D7E2D8D2DC2
:10DE00009C2D0E94F2D50E9400DBF801E45BFF4FDD
:10DE100071836083D8018C918E7F8C938F2C9E2C84
:10DE2000AD2CBC2C81018BA18F5F8F708BA3FDA2C9
:10DE3000E9A6D9AACEAE79CAF1018081816080833A
:10DE4000C8010E949BA181116FC0D10111966D91F3
:10DE50007D918D919C9114970E9422DC6B017C0135
:10DE60009B01AC0160E070E080E89FE30E9493DAE0
:10DE70002B013C012DEC3CEC4CE45DE30E94F2D51F
:10DE800069837A838B839C839401A501C301B201CA
:10DE90000E94F2D5698B7A8B8B8B9C8BAE014F5F86
:10DEA0005F4FBE016F5E7F4FC1010E9437AAF10133
:10DEB000E95BFF4F80818823B9F120911E063091E4
:10DEC0001F0640912006509121063796608171818E
:10DED000828193810E94F2D520916A1130916B1159
:10DEE00040916C1150916D110E94F2D54B015C0173
:10DEF0009B01AC01C701B6010E94F2D50E9400DB74
:10DF0000F101E65BFF4F718360832DEC3CEC4CE448
:10DF10005DE3C501B4010E94F2D50E9400DBF1016E
:10DF2000E45BFF4F71836083F10180818E7F80838A
:10DF300004CA28E6269DF001279DF00D1124E25920
:10DF4000FE4E808181FD43C0C114D10441F0D60151
:10DF50001596CD90DD90ED90FC90189708C08BE061
:10DF6000C82E87EDD82E83E2E82E8BE3F82EB8E694
:10DF7000B69DF001B79DF00D1124E259FE4E818946
:10DF80009289A389B489BC01CD0190589B01AC0151
:10DF90000E94B7D9F80125853685478550890E94AA
:10DFA000F2D59B01AC01C701B6010E94B6D9E62E9D
:10DFB000872E982EA92E262F372F482F592F6DA543
:10DFC0007DA189A599A90E948DD587FF04C0EDA4E4
:10DFD0008DA099A4A9A82E2D382D492D5A2DC20106
:10DFE000B1010E948DD5882309F427CEF8E6F69D6D
:10DFF000C001F79D900D11249C0122593E4E6901EC
:10E00000D9018C9181608C93C8010E949BA18823C7
:10E0100029F0F60180818E7F80830FCE8E2D982D82
:10E02000A92DBA2DF60185839683A783B08705CEE7
:10E03000D6018C9181FD52C0D60115962D913D914E
:10E040004D915C9118972DA73EA74FA758AB15018E
:10E05000B5E02B0E311CF801458056806780708436
:10E06000A30192016DA57EA58FA598A90E948DD5CB
:10E0700087FF34C0F60181899289A389B489BC01E4
:10E08000CD0190589B01AC010E94B7D9D6011D96D5
:10E090002D913D914D915C9150970E94F2D59B013D
:10E0A000AC016DA57EA58FA598A90E94B6D96B017C
:10E0B0007C019B01AC01C301B2010E94DDDB18169B
:10E0C0006CF4D8018C9181608C93C5010E949BA156
:10E0D0008823E1F0F80180818E7F808318E6189D07
:10E0E000F001199DF00D1124E259FE4E2185328573
:10E0F0004385548565817681878190850E948DD581
:10E100008111D2CD0BA100930A0ACECDD101CD92BF
:10E11000DD92ED92FC9213970BA100930A0ADECFD9
:10E12000C858DF4F0FB6F894DEBF0FBECDBFDF91EA
:10E13000CF911F910F91FF90EF90DF90CF90BF9004
:10E14000AF909F908F907F906F905F904F903F9097
:10E150002F90089580910B0A90910C0A891B8F7063
:10E160008F3019F40E945258F5CF80910B0A8F5FBF
:10E170008F70E0910B0A98E69E9FF0011124E259FE
:10E18000FE4EDF011D929A95E9F798E09083409149
:10E19000310A5091320A6091330A7091340A458BEA
:10E1A000568B678B708F4091350A5091360A60917B
:10E1B000370A7091380A418F528F638F748F409164
:10E1C000390A50913A0A60913B0A70913C0A458F96
:10E1D000568F678F70A340913D0A50913E0A60911F
:10E1E0003F0A7091400A41A352A363A374A32091F4
:10E1F0000B0A90910C0A291303C094E69093080A25
:10E2000080930B0A80916F00826080936F00089565
:10E2100090910B0A80910C0A981306C080915810B7
:10E2200090915910892B19F00E945258F1CF0895FE
:10E230002F923F924F925F926F927F928F929F9216
:10E24000AF92BF92CF92DF92EF92FF920F931F9304
:10E25000CF93DF93CDB7DEB762970FB6F894DEBFEA
:10E260000FBECDBF8091DF05982F9270E92EE82F69
:10E27000E470FE2EF82FF170DF2E80FF04C099238A
:10E2800011F0E11152C0EFE6FEE184918F010F5FC2
:10E290001F4F811103C0E5EDFAE104C00E94B9519E
:10E2A000F801F3CF84918F010F5F1F4F882321F076
:10E2B0000E94B951F801F6CFD1100CC0E3EDFAE19C
:10E2C00084918F010F5F1F4F882321F00E94B95165
:10E2D000F801F6CFE1100CC0E1EDFAE184918F0175
:10E2E0000F5F1F4F882321F00E94B951F801F6CF2C
:10E2F000F11003C0EFECFAE103C0E7ECFAE10AC069
:10E3000084918F010F5F1F4F8823B9F30E94B95189
:10E31000F801F6CF84918F010F5F1F4F882309F416
:10E32000C7C00E94B951F801F5CF05E617E189E2AF
:10E3300094E09A8B898BFE0131965F019EEA892ECB
:10E3400097E1992E1F01F80165917591859194913E
:10E35000E989FA89C190D190E190F190FA8BE98B2B
:10E36000A70196010E94B6D92B013C01F1016083FF
:10E3700071838283938320E030E040EA51EC0E9475
:10E38000DDDB87FD0AC020E030E040EA51E4C30154
:10E39000B2010E948DD518162CF4F4018491181640
:10E3A0000CF47CC0F101C190D190E190F1901F017B
:10E3B00020E030E040EA51ECC701B6010E94DDDB0D
:10E3C00087FD0AC020E030E040EA51E4C701B60111
:10E3D0000E948DD5181614F5EAE5FEE184918F01AF
:10E3E0000F5F1F4F811103C0EBEDFAE104C00E94E3
:10E3F000B951F801F3CF84918F010F5F1F4F88232C
:10E4000021F00E94B951F801F6CF88E290E0988B94
:10E410008F8788EC90E09E878D8738C00C5F1F4FF8
:10E42000FFEF8F1A9F0A87E10137180709F08BCF9A
:10E4300089E6E82E86E0F82E10E0F50181919191B1
:10E44000A191B1915F01F70181939193A193B19350
:10E450007F01812F0E944C821F5F133071F70E9451
:10E46000637C83E992E0988B8F8704E610E01E8737
:10E470000D87BE01615F7F4FCE010D960E9420C3C4
:10E480008AEB92E0988B8F871E870D87BE01615FB4
:10E490007F4FCE010D960E9420C30AC0F7FAF09478
:10E4A000F7F8F094F101C082D182E282F3827ACF50
:10E4B00062960FB6F894DEBF0FBECDBFDF91CF914D
:10E4C0001F910F91FF90EF90DF90CF90BF90AF9092
:10E4D0009F908F907F906F905F904F903F902F9084
:10E4E0000895CF92DF92EF92FF920F931F93CF93F5
:10E4F000DF9388E50E945451D82E89E40E9454513C
:10E50000C82E882319F00E94ED501CC0DD20C1F0F8
:10E510000E941D5120E030E040E251E40E94B6D953
:10E5200020E030E04CEB51E40E94B7D921E43CE418
:10E530004EEA5CE30E94F2D50E94FBDA653010F0EF
:10E540001FEF01C0162F89E50E945451082F8AE45D
:10E550000E945451C82F882319F00E94ED501CC00E
:10E560000023C1F00E941D5120E030E040E251E460
:10E570000E94B6D920E030E04CEB51E40E94B7D9BC
:10E5800021E43CE44EEA5CE30E94F2D50E94FBDA0F
:10E59000653010F0DFEF01C0D62F8AE50E9454519C
:10E5A000E82E811105C081E50E945451F82E01C06A
:10E5B000F12CC11001C0C0E02C2F30E0D11001C0FF
:10E5C00000E0200F311D2130310521F4E1101AC087
:10E5D000F11018C0EAE5FEE18491EF012196811166
:10E5E00003C0E7EAFAE104C00E94B951FE01F4CF8A
:10E5F0008491EF012196882309F455C00E94B951F6
:10E60000FE01F6CF17FD02C0D7FF17C0EAE5FEE115
:10E610008491EF012196811103C0E8E8FAE104C07A
:10E620000E94B951FE01F4CF8491EF012196882315
:10E63000D1F10E94B951FE01F7CF0E941D519B01FB
:10E64000AC01012F110F110BAD2FDD0FBB0BFF2004
:10E6500099F085E0809FF001819FF00D1124EA0F71
:10E66000FB1FEE0FFF1FEE0FFF1FEB54FF4E6081ED
:10E6700071818281938103C060E070E0CB01E5E0AD
:10E68000E09FE001E19FD00D1124CA0FDB1FCC0FEA
:10E69000DD1FCC0FDD1FCB54DF4E0E94B7D968833E
:10E6A00079838A839B83DF91CF911F910F91FF9094
:10E6B000EF90DF90CF9008952F923F924F925F920C
:10E6C0006F927F928F929F92AF92BF92CF92DF9282
:10E6D000EF92FF920F931F93CF93DF93CDB7DEB7E7
:10E6E00061970FB6F894DEBF0FBECDBF83E50E94E1
:10E6F0005451882349F00E940E51182F811106C0F1
:10E7000080E00E94E88002C01091FD1780912904EA
:10E7100090912A04A0912B04B0912C0489839A83B0
:10E72000AB83BC8380912D0490912E04A0912F0483
:10E73000B09130048D839E83AF83B887809131047C
:10E7400090913204A0913304B091340489879A8760
:10E75000AB87BC870E94BB80882309F49AC083E4FE
:10E760000E945451882309F494C00E941D511B013A
:10E770002C0105E0612C712C38EC388B82EC898BF4
:10E78000A12CB12C98EC9E87E2E4EF87015080F138
:10E7900025E02D87209F400111243D8531503D8784
:10E7A0003F3FA1F3F401E30FF11DEE0FFF1FEE0F4A
:10E7B000FF1FEB54FF4EC080D180E280F3809601B2
:10E7C000A701B5018E859F850E94DDDB18161CF41C
:10E7D0005601EE86FF869601A701B30188899989C3
:10E7E0000E948DD587FFD9CF3601E88AF98AD5CF27
:10E7F000930148895989B5018E859F850E94B7D9B3
:10E8000020E030E040E05FE30E94F2D5A2019101F8
:10E810000E94B7D92B013C012DEB37E346E855EBBD
:10E820000E94DDDB87FD0AC02DEB37E346E855E3A8
:10E83000C301B2010E948DD518165CF580E00E94DC
:10E84000E88035E0D32E45E0C42EDA949FEFD91648
:10E8500001F105E0CD9C500111240150B0F3750188
:10E86000E00EF11CC701880F991F880F991FFC014A
:10E87000EB54FF4E7F01A30192016081718182817F
:10E8800093810E94B6D9F701608371838283938359
:10E89000E4CF86E50E945451882399F00E94BB8002
:10E8A000882379F0E2E7FAE184917F012FEFE21A01
:10E8B000F20A882321F00E94B951F701F5CF0E9496
:10E8C000ECAE8AE50E945451882321F00E941D512C
:10E8D0000E948BC2812F0E94E880111103C0EFE6D5
:10E8E000FEE11CC08091FD178111F9CFEAE5FEE140
:10E8F00084918F010F5F1F4F882321F00E94B9512F
:10E90000F801F6CFE3E5FAE184918F010F5F1F4F25
:10E91000882329F30E94B951F801F6CF84918F0121
:10E920000F5F1F4F882321F00E94B951F801F6CFE5
:10E930008091FD17811103C06FE073E002C06BE0AE
:10E9400073E085E49AE10E9453B78AE00E94B951CE
:10E95000EFE6FEE184918F010F5F1F4F882321F0C6
:10E960000E94B951F801F6CFE8E3FAE184918F01F2
:10E970000F5F1F4F882321F00E94B951F801F6CF95
:10E98000C090FE17D090FF17E0900018F09001188B
:10E9900020E030E0A901C701B6010E94DDDB1816B6
:10E9A0004CF442E0C701B6010E9460558AE00E9423
:10E9B000B9510CC0E3E3FAE184918F010F5F1F4F5F
:10E9C000882321F00E94B951F801F6CF4CE050E0C5
:10E9D00069E274E0CE0101960E94EFDC892BC9F058
:10E9E00061960FB6F894DEBF0FBECDBFDF91CF9119
:10E9F0001F910F91FF90EF90DF90CF90BF90AF905D
:10EA00009F908F907F906F905F904F903F902F904E
:10EA10005AC761960FB6F894DEBF0FBECDBFDF9127
:10EA2000CF911F910F91FF90EF90DF90CF90BF900B
:10EA3000AF909F908F907F906F905F904F903F909E
:10EA40002F90089580916F00982F927081FF05C0DC
:10EA500080916F008D7F80936F0080910C0A80936E
:10EA60000B0A80930A0A8093090A84E68093080AB5
:10EA700028EE33E03093591020935810992329F051
:10EA800080916F00826080936F0081E08093181006
:10EA9000BFDB0E94155C8091FD17882321F088EB75
:10EAA00095E00E944BB88CE0E8EBF5E0A9E2B4E019
:10EAB00001900D928A95E1F70C94A6502F923F9207
:10EAC0004F925F926F927F928F929F92AF92BF927E
:10EAD000CF92DF92EF92FF920F931F93CF93DF932A
:10EAE000CDB7DEB7CD54D1090FB6F894DEBF0FBE57
:10EAF000CDBF85E40E949D51882321F00E94ED50F6
:10EB00007B0102C0E12CF12C83E40E949D518823FB
:10EB100021F00E94ED506AA302C005E00AA385E53A
:10EB20000E949D51882319F00E940E5103C085E573
:10EB30000E9454518CA7F7FC07C0812C912C16E140
:10EB4000A12E13E4B12E06C0812C912CBCE8AB2E73
:10EB5000B2E4BB2E83E50E949D51882321F00E94E0
:10EB60001D514B015C01E114F10411F410925C1091
:10EB70001092C505ED820E9402C52B013C011D814A
:10EB800017FF05C00CE310E022E0298304C003E274
:10EB900010E035E03983D301C2018C53964FAF4F5B
:10EBA000BF4F8093521090935310A0935410B09382
:10EBB000551061E06E0D623080F0E5EFF9E184916F
:10EBC0008F010F5F1F4F1A830983882309F45FC3E6
:10EBD0000E94B951E981FA81F2CFEFE1FAE1849123
:10EBE0007F012FEFE21AF20A882321F00E94B95127
:10EBF000F701F5CF0E94639B3D8137FF04C08FE78B
:10EC000080935B1008C04D81E42F440FFF0BE65A40
:10EC1000FF4E8FE78083C501B4010E94FBDA072E07
:10EC2000000C880B990B0E9493D56A877B878C8791
:10EC30009D878981482F50E09801A8EEB3E00E949B
:10EC4000A7D96DA77EA78FA798AB8B019C01040D58
:10EC5000151D261D371D0AAF1BAF2CAF3DAF81E040
:10EC6000809334021D811F3F39F40FE519E11FAF76
:10EC70000EAF09E219E106C00DE419E11FAF0EAFB6
:10EC800006E119E122961FAF0EAF22974CA25DA2BA
:10EC90006EA27FA249AA5AAA6BAA7CAA1DAA1EAA82
:10ECA0001FAA18AE19AE188E10E4198F0CE10A8F46
:10ECB00016E41B8F1C8E1D8E1E8E1F8E1C8A1D8AB5
:10ECC0001E8A1F8A188A198A1A8A1B8A19821A822E
:10ECD0001B821C828FE790E0A0E0B0E08E839F83D0
:10ECE000A887B987FFE7CF2ED12CE12CF12C18A6ED
:10ECF00019A61AA61BA611E01F861E862D961FAE0A
:10ED00002D97212C312C2E961FAE2E970D81802F02
:10ED1000000F990B9C01265A3F4E24963FAF2EAF11
:10ED20002497880F991F880F991FDC01AD5BBB4F9B
:10ED3000B9A3A8A3CA01052E000CAA0BBB0B2896E9
:10ED40008CAF9DAFAEAFBFAF28974C5F5F4FCA018E
:10ED5000550FAA0BBB0B2C968CAF9DAFAEAFBFAFC0
:10ED60002C97AAA10A2E000CBB0BBBA3AAA38091CF
:10ED70003402882309F489C20E9402C54B015C0158
:10ED800080915710882309F4D4C00E944B9A0D81BA
:10ED900007FD0CC0A8A1B9A1BC912D96BFAF2D97BE
:10EDA000E8A1F9A12180328003810BC000913D04CC
:10EDB0002D960FAF2D9720903E0430903F04009188
:10EDC00040042E960FAF2E972D962FAD2D97322DF6
:10EDD000432D2E965FAD2E976C8D7D8D8E8D9F8DE4
:10EDE0000E948DD587FF0AC02D960FAD2D970C8FF1
:10EDF0002D8E3E8E2E960FAD2E970F8F288D398D2E
:10EE00004A8D5B8D2D966FAD2D97722D832D2E968D
:10EE10009FAD2E970E948DD587FF0AC02D960FAD0E
:10EE20002D97088F298E3A8E2E960FAD2E970B8F29
:10EE30008091521090915310A0915410B0915510A0
:10EE4000A5019401281B390B4A0B5B0B57FD10C021
:10EE50000E946A9AD501C4018C53964FAF4FBF4FA1
:10EE60008093521090935310A0935410B093551068
:10EE70002D962FAD2D97322D432D2E965FAD2E97CB
:10EE80006A857B858C859D851123E9F10E948DD54E
:10EE900087FF4FC0B501A4014419550966097709D8
:10EEA000DB01CA0188589341A109B109B7FD41C0EE
:10EEB000D701C6010E811F8128853985801B910BE2
:10EEC000A20BB30B1D81B595A7959795879517FF55
:10EED00003C080935B1005C02496EEADFFAD249770
:10EEE000808348A759A76AA77BA70A850C8F1B8533
:10EEF0001D8F0C850E8F1D851F8F8CA29DA2AEA22B
:10EF0000BFA210E016C00E94DDDB181694F4D501F4
:10EF1000C4012CA13DA14EA15FA1821B930BA40BA8
:10EF2000B50BAC01BD01485853416109710977FF28
:10EF3000CBC120E030E040EA51E46A857B858C85D6
:10EF40009D850E94B7D92D962FAD2D97322D432D3B
:10EF50002E965FAD2E970E948DD587FF10C0E1E8F9
:10EF6000F9E184918F010F5F1F4F1A830983882372
:10EF700009F48BC10E94B951E981FA81F2CFD50120
:10EF8000C40129A93AA94BA95CA9821B930BA40B24
:10EF9000B50BB7FD96C00E9465988AE00E94B951F2
:10EFA000D501C4018053984FAF4FBF4F89AB9AAB87
:10EFB000ABABBCAB0DA9011163C02EA93FA948ADF5
:10EFC00059AD2D966FAD2D97722D832D2E969FAD39
:10EFD0002E970E94DDDB18160CF041C028966CAD10
:10EFE0007DAD8EAD9FAD28970E9493D52D962FAD08
:10EFF0002D97322D432D2E965FAD2E970E94B7D9B7
:10F000006EAB7FAB88AF99AF2DA53EA54FA558A994
:10F01000280D391D4A1D5B1D2AAF3BAF4CAF5DAFBC
:10F020002C966CAD7DAD8EAD9FAD2C970E9493D587
:10F030009B01AC016A857B858C859D850E94B6D934
:10F040002D962FAD2D97322D432D2E965FAD2E97F9
:10F050000E948DD5881F8827881F8DAB32C0D501AF
:10F06000C4012AAD3BAD4CAD5DAD821B930BA40B2F
:10F07000B50BB7FD26C04EAD5FAD62E779E11EC0AE
:10F0800020E030E040EA51E46A857B858C859D85EF
:10F090000E94B6D99B01AC012D966FAD2D97722DB4
:10F0A000832D2E969FAD2E970E948DD587FF09C088
:10F0B00022964EAD5FAD22976DE379E18D810E947E
:10F0C000829BD501C401880F991FAA1FBB1F2CA1C9
:10F0D0003DA14EA15FA1821B930BA40BB50B84191C
:10F0E0009509A609B70981389F44A241B10580F06E
:10F0F000E8EFF8E184918F010F5F1F4F1A830983B6
:10F10000882309F4C2C00E94B951E981FA81F2CF83
:10F110002AA13BA14E855F85241735070CF027CE29
:10F12000EBE9F8E184918F010F5F1F4F1F830E837E
:10F13000882329F00E94B951EE81FF81F3CF1D8110
:10F1400017FD03C00EE013E002C007EF13E01F83BA
:10F150000E836E817F818AE898E10E9453B74981CE
:10F160005A816B817C8186E898E10E941DB78AE014
:10F170000E94B9516E817F8185E798E10E9453B763
:10F18000488959896A897B8981E798E10E941DB77E
:10F190008AE00E94B9516E817F8180E698E10E94E9
:10F1A00053B74C895D896E897F898CE598E10E940F
:10F1B0001DB78AE00E94B9511CA5112309F467C04C
:10F1C0000D8107FF31C029813A814B815C812093F9
:10F1D00042103093431040934410509345102CEA52
:10F1E00035EC47E25EE3688979898A899B890E94C8
:10F1F000F2D560933E1070933F108093401090932F
:10F2000041102CEA35EC47E25EE36C897D898E89FA
:10F210009F890E9493DA60933A1070933B10809319
:10F220003C1090933D1033C089819A81AB81BC81A1
:10F2300080934A1090934B10A0934C10B0934D10B4
:10F240002CEA35EC47E25EE3688979898A899B89F3
:10F250000E94F2D560934610709347108093481037
:10F26000909349102CEA35EC47E25EE36C897D8986
:10F270008E899F890E9493DA60934E1070934F108D
:10F28000809350109093511002C00E94639B81E0C4
:10F290008093C505C35BDF4F0FB6F894DEBF0FBE8A
:10F2A000CDBFDF91CF911F910F91FF90EF90DF9035
:10F2B000CF90BF90AF909F908F907F906F905F9016
:10F2C0004F903F902F9008950E851F85012B09F4D4
:10F2D0002DC148A459A46AA47BA4480E591E6A1ED5
:10F2E0007B1E28A539A54AA55BA5281B390B4A0B0F
:10F2F0005B0B6E817F81888599850E946CD9A30103
:10F3000092010E94B3DCDA01C9018C0D9D1DAE1D76
:10F31000BF1D84319105A105B105FCF06C017D0193
:10F320008C3E9105A105B1052CF05BEEC52ED12CCC
:10F33000E12CF12C20E8C216D104E104F104DCF048
:10F340008EEF90E0A0E0B0E08C199D09AE09BF09F6
:10F350008E839F83A887B98712C044E1C42ED12C25
:10F36000E12CF12C04E110E020E030E00E831F835B
:10F370002887398704C0CE82DF82E886F986EDEEE1
:10F38000F9E184918F010F5F1F4F882321F00E94C4
:10F39000B951F801F6CFC701B6010E944655E8EE13
:10F3A000F9E184918F010F5F1F4F882321F00E94A4
:10F3B000B951F801F6CF6E817F81888599850E94C9
:10F3C0004655488D598D6A8D7B8D81EE99E10E945D
:10F3D0001DB74C8D5D8D6E8D7F8D8AED99E10E94FC
:10F3E0001DB70E851F85033011050CF49FC06E817B
:10F3F0007F81888599850E9493D520E030E040E8A0
:10F4000050E40E94F2D569837A838B839C83288D94
:10F41000398D4A8D5B8D6C8D7D8D8E8D9F8D0E947B
:10F42000B6D92BED3FE049E450E40E94F2D520E04C
:10F4300030E040E05FE30E94F2D59B01AC016981BE
:10F440007A818B819C810E9493DA69837A838B8392
:10F450009C83C301B2010E9493D52FE632E143E8B9
:10F460005AE30E94F2D52B013C0149815A816B81FC
:10F470007C8184ED99E10E941DB7B301A2018EEC5D
:10F4800099E10E941DB72AE939E949E15FE3698101
:10F490007A818B819C810E94F2D569837A838B83E8
:10F4A0009C839B01AC010E94B7D9A30192010E94E9
:10F4B00093DA688B798B8A8B9B8B29813A814B817C
:10F4C0005C81C301B2010E94F2D520E030E040E04F
:10F4D0005EE30E94F2D56C8B7D8B8E8B9F8BEEEB67
:10F4E000F9E184918F010F5F1F4F882321F00E9463
:10F4F000B951F801F6CF49815A816B817C8188EB43
:10F5000099E10E941DB7488959896A897B8982EBF4
:10F5100099E10E941DB74C895D896E897F898CEACB
:10F5200099E10E941DB78AE00E94B9518E819F81A6
:10F53000A885B9858C0D9D1DAE1DBF1D1D81B5957E
:10F54000A7959795879517FF03C080935B1005C01B
:10F550002496EEADFFAD249780830E851F850F5F47
:10F560001F4F1F870E871A85188F0B85098F1C85E3
:10F570001A8F0D850B8F2401350111E0DACCCF9362
:10F58000DF93EFE6FEE18491EF012196882321F0DD
:10F590000E94B951FE01F7CF83E50E9454518823A0
:10F5A00021F00E940E5180932102ECE4F8E1849155
:10F5B000EF012196882321F00E94B951FE01F7CF77
:10F5C00080912102811103C0E8E4F8E102C0E4E483
:10F5D000F8E18491EF012196882321F00E94B9512E
:10F5E000FE01F7CFECE3F8E18491EF012196882347
:10F5F00021F00E94B951FE01F7CF20910E04309105
:10F600000F0440911004509111046091AC05709169
:10F61000AD058091AE059091AF050E94B7D9AB01C1
:10F62000BC018AE398E10E941DB720911204309139
:10F63000130440911404509115046091B005709129
:10F64000B1058091B2059091B3050E94B7D9AB0185
:10F65000BC0187E398E10E941DB720911604309108
:10F66000170440911804509119046091B4057091E9
:10F67000B5058091B6059091B7050E94B7D9AB0149
:10F68000BC0184E398E10E941DB7ECE2F8E18491AB
:10F69000EF012196882321F00E94B951FE01F7CF96
:10F6A00020910E0430910F044091100450911104E8
:10F6B00060911502709116028091170290911802C4
:10F6C0000E94B7D9AB01BC018AE298E10E941DB744
:10F6D00020911204309113044091140450911504A8
:10F6E0006091190270911A0280911B0290911C0284
:10F6F0000E94B7D9AB01BC0187E298E10E941DB717
:10F700002091160430911704409118045091190467
:10F7100060911D0270911E0280911F029091200243
:10F720000E94B7D9AB01BC0184E298E10E941DB7E9
:10F730008AE0DF91CF910C94B951CF93DF9381E5AB
:10F740000E9454518823C1F080910C0490910D04C3
:10F75000009739F04AE050E060E070E00E940CD47D
:10F7600003C060E070E0CB0160933E0670933F06FB
:10F77000809340069093410683E50E94545188236C
:10F7800051F00E941D516093460670934706809386
:10F7900048069093490684E50E945451882351F00D
:10F7A0000E941D5160934206709343068093440665
:10F7B0009093450688E50E945451882351F00E9499
:10F7C0001D5160930E0670930F0680931006909360
:10F7D000110689E50E945451882351F00E941D5161
:10F7E0006093120670931306809314069093150687
:10F7F0008AE50E9454518823E9F00E941D516093CC
:10F8000016067093170680931806909319062DEC30
:10F810003CEC4CEC5DE30E948DD518165CF0E2EFF9
:10F82000F7E18491EF012196882321F00E94B951DC
:10F83000FE01F7CF85E40E945451882351F00E94C5
:10F840001D5160931A0670931B0680931C069093BB
:10F850001D06DF91CF910895FF920F931F93CF93D1
:10F86000DF93F82E092F162FEDEEF7E18491EF01CB
:10F870002196882321F00E94B951FE01F7CFEF2D88
:10F88000F02F8491EF012196882321F00E94B95135
:10F89000FE01F7CFEBEEF7E18491EF01219688238B
:10F8A00021F00E94B951FE01F7CF612F70E080E096
:10F8B00090E00E9446558AE0DF91CF911F910F9111
:10F8C000FF900C94B9514F925F926F927F928F92FA
:10F8D0009F92AF92BF92CF92DF92EF92FF92CF931F
:10F8E000DF9320910E0430910F0440911004509149
:10F8F00011046091290470912A0480912B04909145
:10F900002C040E94B7D9AB01BC0180EB9BE10E94A3
:10F910001DB72091120430911304409114045091AA
:10F92000150460912D0470912E0480912F04909104
:10F9300030040E94B7D9AB01BC018CEA9BE10E9464
:10F940001DB720911604309117044091180450916E
:10F9500019046091310470913204809133049091C4
:10F9600034040E94B7D9AB01BC0188EA9BE10E9434
:10F970001DB7409135045091360460913704709161
:10F98000380484EA9BE10E941DB780916F00982F94
:10F99000927081FF05C080916F008D7F80936F0012
:10F9A00040902510509026106090271070902810DD
:10F9B0008090291090902A10A0902B10B0902C10BD
:10F9C000C0902D10D0902E10E0902F10F09030109D
:10F9D000992329F080916F00826080936F00EAE99B
:10F9E000FBE18491EF012196882321F00E94B95117
:10F9F000FE01F7CFC301B2010E944655E6E9FBE1E3
:10FA00008491EF012196882321F00E94B951FE01D3
:10FA1000F7CFC501B4010E944655E2E9FBE18491AC
:10FA2000EF012196882321F00E94B951FE01F7CF02
:10FA3000C701B6010E9446558AE0DF91CF91FF9041
:10FA4000EF90DF90CF90BF90AF909F908F907F907E
:10FA50006F905F904F900C94B95183E50E949D5137
:10FA6000882399F00E941D5120E030E04AE754E4D9
:10FA70000E94F2D50E9400DB60932302709324025F
:10FA80008093250290932602089588E50E945451A0
:10FA9000811111C089E50E94545181110CC08AE581
:10FAA0000E945451811107C085E40E945451811174
:10FAB00002C00C9494A90E94087188E50E945451D8
:10FAC000882331F05F9A809128048E7F80932804E8
:10FAD00089E50E945451882339F08A9A479A809187
:10FAE00028048D7F809328048AE50E94545188233E
:10FAF00061F0809108018095817080930601479A9A
:10FB0000809128048B7F8093280485E40E945451BF
:10FB1000882311F0129A089508952F923F924F92E0
:10FB20005F926F927F928F929F92AF92BF92CF928D
:10FB3000DF92EF92FF920F931F93CF93DF93CDB796
:10FB4000DEB762970FB6F894DEBF0FBECDBF8091CF
:10FB50004B0683FDA4C183E50E949D518C878111D2
:10FB600006C082E50E949D51882309F498C10E9435
:10FB70001D510E94FBDA6E3671050CF08DC1709339
:10FB80003C0460933B040E941F990E941D5120E099
:10FB900030E040EA50E40E94DDDB181614F40E94C5
:10FBA0002C9BE6E8FBE18491FB83EA83882371F0D8
:10FBB000082E000C990B0E94A7924A815B814F5F2F
:10FBC0005F4F5B834A83FA018491F0CF8DE090E030
:10FBD0000E94A7928AE090E00E94A79281E0809321
:10FBE00034021092C5058091C40580935C101A827E
:10FBF0001B821C821D82188619861A861B86198212
:10FC00001D86FCE3FE872CE12F8736E4388B312CF0
:10FC1000212C40E8498B5FEB5A8B812C912C5401AD
:10FC200060913B0470913C04072E000C880B990BEB
:10FC30000E9493D57B018C019B01AC01632D722D39
:10FC400089899A890E948DD5882341F120913D04AC
:10FC500030913E0440913F04509140048C85B7019F
:10FC600081110CC0C8010E948DD5881F8827881F6C
:10FC700089833E2C2F2C098B1A8B10C0C8010E943F
:10FC80008DD587FF06C0EAE8FBE18491FB83EA8318
:10FC9000E7C03E2C2F2C098B1A8B19820E9402C5BB
:10FCA0006B017C01DC01CB01288539854A855B85A8
:10FCB000821B930BA40BB50BB7FD3BC0D701C6014C
:10FCC00088519C4FAF4FBF4F88879987AA87BB87C2
:10FCD0000E946598EEE8FBE184913F019FEF691A6D
:10FCE000790A882321F00E94B951F301F5CF8114DC
:10FCF0009104A104B104B9F0D501C401805F984D0D
:10FD0000AF4FBF4FBC01CD016C197D098E099F0912
:10FD100028EE33E040E050E00E947BD9CA01B901EF
:10FD20000E94465503C08FE30E94B9518AE00E94A9
:10FD3000B9510E9452580E9402C56093C605709343
:10FD4000C7058093C8059093C905A0913D04AE8373
:10FD5000B0913E04BF8300913F04109140040E9483
:10FD600014312E813F81A801632D722D89899A89D2
:10FD70000E94B6D92B013C0120E030E0A9010E948D
:10FD8000DDDB87FF04C077FA709477F870948114F4
:10FD90009104A104B10459F420E030E040E85FE3AD
:10FDA000C301B2010E948DD587FF0DC00AC020E0BB
:10FDB00030E040E450E4C301B2010E94DDDB1816DC
:10FDC00014F446015701E981EE2391F12A813B8128
:10FDD0004C815D81211531054105510541F0D70167
:10FDE000C601821B930BA40BB50BB7FD21C02E815E
:10FDF0003F81A8016D857E858F8598890E94B6D93F
:10FE000020E030E040EC5FE30E948DD587FD3BCFE2
:10FE1000D701C601805A9541AF4FBF4F8A839B835C
:10FE2000AC83BD839E819D87AF81AE870F87188B82
:10FE300080913402882309F426CF81149104A1040F
:10FE4000B10409F4EDCEB0E1CB1AB7E2DB0AE10868
:10FE5000F108C818D908EA08FB08F7FE14CFE0CE6D
:10FE6000882361F0082E000C990B0E94A792EA816A
:10FE7000FB813196FB83EA838491F2CF8DE090E0A1
:10FE80000E94A7928AE090E00E94A792809134029B
:10FE900081E08093C50503C06EE670E070CE629687
:10FEA0000FB6F894DEBF0FBECDBFDF91CF911F918B
:10FEB0000F91FF90EF90DF90CF90BF90AF909F9009
:10FEC0008F907F906F905F904F903F902F9008950C
:10FED0009F92AF92BF92CF92DF92EF92FF920F93D9
:10FEE0001F93CF93DF938FE4A82E82E0B82E00EE0D
:10FEF00015E0C9E2D4E09EE0C92E94E0D92E2AE1B3
:10FF0000E22E24E0F22E912CF50181915F010E94F6
:10FF10005451882309F10E941D51F70120812111BC
:10FF200004C020911E04222339F0288139814A819E
:10FF30005B810E94B7D90AC0F3E09F1639F0F60141
:10FF400020813181428153810E94B6D9F8016083BA
:10FF500071838283938309C088819981AA81BB813F
:10FF6000F80180839183A283B38393940C5F1F4F26
:10FF70002496F4E0CF0ED11C2FEFE21AF20A84E0AF
:10FF80009812C2CF86E40E949D518823C9F00E9436
:10FF90001D5120E030E0A9010E94DDDB181684F439
:10FFA0000E941D5120E030E040E752E40E9493DAC5
:10FFB00060934B0270934C0280934D0290934E02DB
:10FFC000DF91CF911F910F91FF90EF90DF90CF9035
:10FFD000BF90AF909F9008952F923F924F925F9263
:10FFE0006F927F929F92AF92BF92CF92DF92EF92E9
:10FFF000FF920F931F93CF93DF93CDB7DEB7649734
:020000021000EC
:100000000FB6F894DEBF0FBECDBF1A012B01922EA2
:10001000F32EC82ED12CF601E255F84EE491AA2415
:10002000A3941E160CF4A12CBB24B39420E030E062
:10003000A901C201B1010E94DDDB18160CF0B12C40
:10004000CC0CDD1CCC0CDD1CC601875D9B4F3C013C
:10005000FC0110821182128213820E94A650F301C9
:100060002082318242825382E090C40520E030E059
:10007000A901B801892D9F2D0E948DD581110AC03B
:10008000F601E459F74D85919591A591B4918C01B4
:100090009A2EFB2EC801A92DBF2D898B9A8BAB8B75
:1000A000BC8B8091310490913204A0913304B091C3
:1000B000340440912D0450912E0460912F047091CE
:1000C00030040091290410912A0420912B043091CE
:1000D0002C0409831A832B833C834D835E836F83B7
:1000E000788789879A87AB87BC871D861E861F867F
:1000F000188AAE01475F5F4FBE016B5F7F4FCE0135
:1001000001960E94B2AECE010D966C018E010F5E7B
:100110001F4F25E334E0AE01475F5F4FBE016B5FC9
:100120007F4F0C970E94E4600E940871AB1459F055
:1001300080917906882319F01092790604C084E230
:100140009BE10E940D5864960FB6F894DEBF0FBE77
:10015000CDBFDF91CF911F910F91FF90EF90DF9076
:10016000CF90BF90AF909F907F906F905F904F9097
:100170003F902F900895EF92FF921F93CF93DF93BC
:1001800085EBE82E80E1F82E15E0C0E0D0E020E01D
:1001900030E0A901F701EC0FFD1F608171818281C0
:1001A00093810E948DD581110CC02496C431D10554
:1001B00071F7115084E1E80EF11C1111E6CF80E0D7
:1001C00001C081E0DF91CF911F91FF90EF900895E2
:1001D000CF939091FD179817C9F0C82F0E9408710E
:1001E000C11112C041E354E06DE274E089E294E091
:1001F0000E94B2AE80E08093FD17882339F089E237
:1002000094E0CF910C944BB8B6DFF5CFCF91089521
:100210008F929F92AF92BF92EF92FF920F931F9394
:10022000CF93DF9300D01F92CDB7DEB7182F809108
:1002300028048770873069F48FE40E949D518823D9
:1002400019F00E940E5103C08FE40E945451811195
:10025000BDC00E94087180E0BBDF80914B0290918D
:100260004C02A0914D02B0914E02809353069093A0
:100270005406A0935506B0935606809102029091C1
:100280000302909352068093510684E690E0909387
:1002900003028093020281E08093680611111BC063
:1002A00088E50E945451F82E89E50E945451082F88
:1002B0008AE50E945451E82EF11006C0011109C0D0
:1002C000811107C0F02E0CC0002319F0F02E182F5A
:1002D00008C010E006C0FF24F39401E0EE24E3948C
:1002E00011E00E94AF5182E50E949D51882361F088
:1002F0000E941D514B015C0120E030E0A9010E94E9
:100300008DD5882371F106C0812C912C80EAA82E0E
:1003100080E4B82E111104C0F11002C0002391F145
:100320008092E8059092E905A092EA05B092EB056B
:10033000A5019401609131047091320480913304DD
:10034000909134040E948DD587FF0BC019821A82C8
:100350001B821C82BE016F5F7F4F88EE95E00E947A
:100360006DC2111105C0F11003C0011106C00AC011
:1003700080E00E94B5561123C1F381E00E94B5567A
:10038000111102C0EE2019F082E00E94B5560E94C1
:10039000A6508091670680936806809153069091DD
:1003A0005406A0915506B091560680934B02909347
:1003B0004C02A0934D02B0934E0280915106909151
:1003C000520690930302809302027DDA0F900F9001
:1003D0000F900F90DF91CF911F910F91FF90EF90B1
:1003E000BF90AF909F908F900895CF92DF92EF9241
:1003F0000F931F93CF93DF93CDB7DEB760970FB600
:10040000F894DEBF0FBECDBFE090C405E9E2F4E092
:1004100080859185A285B3854481558166817781E8
:10042000008111812281338109831A832B833C83CC
:100430004D835E836F83788789879A87AB87BC8774
:100440001D861E861F86188AAE01475F5F4FBE015C
:100450006B5F7F4FCE0101960E94B2AECE010D962A
:100460006C010BE412E025E334E0AE01475F5F4F1F
:10047000BE016B5F7F4F0C970E94E46060960FB6E1
:10048000F894DEBF0FBECDBFDF91CF911F910F91CA
:10049000EF90DF90CF9008950F931F93CF93DF934A
:1004A00094E0899FE00111248E01025F1B4FFE0141
:1004B000E759F94FDE01AD52BA4F2D913D914D9163
:1004C0005C9160817181828193810E94B7D9F8012A
:1004D0006083718382839383FE01E45FF44E859190
:1004E0009591A591B491FE01E455FA4F80839183D3
:1004F000A283B383FE01E85EF44E85919591A591A8
:10050000B491CB5EDD4F88839983AA83BB83DF914F
:10051000CF911F910F910895EF92FF920F931F9328
:10052000CF93DF937C0184E50E949D51D82F8823CF
:1005300049F10E94FD50C82F181604F5EFE6FEE1C0
:1005400084918F010F5F1F4F882321F00E94B951C2
:10055000F801F6CF8DE40E94B951B70180E090E038
:100560004AE00E94DB546C2FCC0F770B89EF9AE1A5
:100570000E943AB78AE00E94B95108C080935C108B
:10058000D0E004C08091C40580935C108D2FDF9172
:10059000CF911F910F91FF90EF9008952F923F926E
:1005A0004F925F926F927F928F929F92AF92BF9283
:1005B000CF92DF92EF92FF920F931F93CF93DF932F
:1005C000CDB7DEB762970FB6F894DEBF0FBECDBFD2
:1005D0008DE690E0A1DF8111C5C180914B0683FDBE
:1005E000C1C183E50E949D518C87811106C082E5BF
:1005F0000E949D5189838823B1F00E941D510E9461
:10060000FBDACB010E9445910E941D5120E030E0B1
:1006100044EB52E40E948DD518160CF49EC10E9442
:100620004E9B21E02983E6E7FBE184918F0188233B
:1006300051F0082E000C990B0E94A7920F5F1F4FDC
:10064000F8018491F4CF8DE090E00E94A7928AE0B7
:1006500090E00E94A7920E947DB9F981FF2309F4DE
:1006600081C181E0809334021092C5051A821B82F9
:100670001C821D82188619861A861B8619821D8681
:100680002CE32E873CE13F8746E4488B312C212C1C
:1006900050E8598B8FEB8A8B812C912C54016091FF
:1006A000410470914204072E000C880B990B0E94A4
:1006B00093D57B018C019B01AC01632D722D89893F
:1006C0009A890E948DD5882359F120914304309155
:1006D000440440914504509146049C85B701802F05
:1006E00091110CC0912F0E948DD5881F8827881FDB
:1006F00089833E2C2F2C098B1A8B12C0912F0E94BC
:100700008DD587FF08C080913402EEE7FBE184912C
:10071000FB83EA83E7C03E2C2F2C098B1A8B1982AE
:100720000E9402C56B017C01DC01CB012885398563
:100730004A855B85821B930BA40BB50BB7FD3BC0B1
:10074000D701C60188519C4FAF4FBF4F888799870B
:10075000AA87BB870E946598E2E8FBE184913F018C
:100760009FEF691A790A882321F00E94B951F30199
:10077000F5CF81149104A104B104B9F0D501C401ED
:10078000805F984DAF4FBF4FBC01CD016C197D0903
:100790008E099F0928EE33E040E050E00E947BD9AB
:1007A000CA01B9010E94465503C08FE30E94B951A6
:1007B0008AE00E94B9510E9452580E9402C560937B
:1007C000C6057093C7058093C8059093C905A0918D
:1007D0004304AE83B0914404BF830091450410915B
:1007E00046040E9414312E813F81A801632D722D91
:1007F00089899A890E94B6D92B013C0120E030E01A
:10080000A9010E94DDDB87FF04C077FA709477F8B6
:10081000709481149104A104B10459F420E030E0F3
:1008200040E85FE3C301B2010E948DD587FF0DC090
:100830000AC020E030E040E450E4C301B2010E946D
:10084000DDDB181614F446015701E981EE2391F11E
:100850002A813B814C815D8121153105410551057E
:1008600041F0D701C601821B930BA40BB50BB7FD5A
:1008700021C02E813F81A8016D857E858F85988955
:100880000E94B6D920E030E040EC5FE30E948DD5B5
:1008900087FD39CFD701C601805A9541AF4FBF4F71
:1008A0008A839B83AC83BD839E819D87AF81AE8706
:1008B0000F87188B80913402882309F424CF811488
:1008C0009104A104B10409F4EACEB0E1CB1AB7E275
:1008D000DB0AE108F108C818D908EA08FB08F7FEA6
:1008E00012CFDDCE882361F0082E000C990B0E94F8
:1008F000A792EA81FB813196FB83EA838491F2CF50
:100900008DE090E00E94A7928AE090E00E94A7927A
:100910008091970E8130E9F4EAE7FBE18491FB8353
:10092000EA83882371F0082E000C990B0E94A7928D
:100930004A815B814F5F5F4F5B834A83FA018491F9
:10094000F0CF8DE090E00E94A7928AE090E00E94B4
:10095000A79281E08093C50505C00E942C9B31E0E1
:10096000398361CE62960FB6F894DEBF0FBECDBF5D
:10097000DF91CF911F910F91FF90EF90DF90CF907B
:10098000BF90AF909F908F907F906F905F904F90AF
:100990003F902F900895EF92FF920F931F93CF9364
:1009A000DF93CDB7DEB76D970FB6F894DEBF0FBEFD
:1009B000CDBF80918A0A882309F486C082E59CE035
:1009C0000E944BBF82E59CE00E94B4A21092880A6C
:1009D0001092870A80918A0A882309F475C00091D1
:1009E0003218109133180E94D094B801CE014C9661
:1009F0000E94E4968C01892B09F466C06C8D7D8D74
:100A00006115710511F06C5F7F4F19821C8222E025
:100A1000A801CE0101960E9447A8811102C0F12CC5
:100A200014C0CE0101960E943E948823C1F361E078
:100A3000CE0101960E94BDA2009789F325EEFC012C
:100A400020831C820E94F4BCF82ECE0101960E94E5
:100A5000A951FF2009F1E1E4FBE184917F019FEFBF
:100A6000E91AF90A882321F00E94B951F701F5CF5C
:100A7000F80181918F01882319F00E94B951F8CFB4
:100A80008AE00E94B9511092030D1092040D109249
:100A9000050D1092060D18C0EFE4FBE184917F0173
:100AA0009FEFE91AF90A882321F00E94B951F70152
:100AB000F5CFF80181918F01882319F00E94B95177
:100AC000F8CF8EE20E94B9516D960FB6F894DEBF52
:100AD0000FBECDBFDF91CF911F910F91FF90EF908F
:100AE0000895CF93DF938B3D9240B1F0EAE5FEE1AC
:100AF0008491EF012196882321F00E94B951FE01D3
:100B0000F7CFE3EBFBE18491EF012196882331F0ED
:100B10000E94B951FE01F7CF80E001C081E0DF9172
:100B2000CF9108952F923F924F925F926F927F9252
:100B30008F929F92AF92BF92CF92DF92EF92FF92ED
:100B40000F931F93CF93DF93CDB7DEB7C757D1096C
:100B50000FB6F894DEBF0FBECDBF2DB63EB6A7963A
:100B60001FAE1EAEA79784E690E0A9969FAF8EAF0A
:100B7000A99701E09E012B593F4F44E050E0BE0190
:100B8000655A7F4FCE0189599F4F0E948FBB9E01AE
:100B90002B593F4F42E050E0BE0167597F4FCE01D5
:100BA00089599F4F0E948FBB43E050E0BE01655AB8
:100BB0007F4F87ED92E00E943EDD892B09F43FC014
:100BC0006F968FAD6F97882339F08FE36C968FAF58
:100BD0006C976D961FAE6D97EFE6FEE184917F01F5
:100BE0002FEFE21AF20A811103C0E6E7FCE104C02C
:100BF0000E94B951F701F2CF84917F013FEFE31AD0
:100C0000F30A882321F00E94B951F701F5CFBE0104
:100C1000655A7F4F8DE69CE10E9453B7EFE5FCE1FA
:100C200084917F019FEFE91AF90A882321F00E943D
:100C3000B951F701F5CF81E08093570654C5EDB760
:100C4000FEB7E696FFAFEEAFE6976B961CAE1DAE15
:100C50001EAE1FAE6B97A7961FAE1EAEA79701E004
:100C60009E012B593F4F41E050E0BE0160597F4F3C
:100C7000CE0189599F4F0E948FBB80E1E3E5F2E0EE
:100C8000DE01919601900D928A95E1F780E1E3E60D
:100C9000F2E0DE01519601900D928A95E1F780E134
:100CA000E3E7F2E0DE01119601900D928A95E1F7FB
:100CB000E1964FADE19750E04D5F5F4F440F551FF8
:100CC000440F551F2DB73EB7241B350B0FB6F894B4
:100CD0003EBF0FBE2DBF8DB79EB701967C0100E0D1
:100CE0009E012B593F4FBC01CE0189599F4F0E9455
:100CF0008FBB9E012B593F4F44E050E06EE376E0FE
:100D0000CE0189599F4F0E948FBBE1968FACE1972E
:100D1000912C93E0890E911C880C991C880C991CCD
:100D2000EDB7FEB7E819F9090FB6F894FEBF0FBE8C
:100D3000EDBF2DB73EB72F5F3F4F69018DB79EB70F
:100D4000881999090FB6F8949EBF0FBE8DBFEDB7F5
:100D5000FEB731965F019E012B593F4FA401B601AA
:100D6000CE0189599F4F0E948FBB9E012B593F4F47
:100D7000A401B501CE0189599F4F0E948FBB1091EC
:100D80005806112309F4A7C000E09E012B593F4FDC
:100D900044E050E066E276E0CE0189599F4F0E9420
:100DA0008FBB9E012B593F4F44E050E06AE276E052
:100DB000CE0189599F4F0E948FBB9E012B593F4FF7
:100DC00044E050E062E276E0CE0189599F4F0E94F4
:100DD0008FBB9E012B593F4F44E050E066E476E024
:100DE000CE0189599F4F0E948FBB9E012B593F4FC7
:100DF00044E050E062E476E0CE0189599F4F0E94C2
:100E00008FBB9E012B593F4F40E150E06EE076E0F2
:100E1000CE0189599F4F0E948FBB9E012B593F4F96
:100E200044E050E0BE01695A7F4FCE0189599F4F7F
:100E30000E948FBB9E012B593F4F4CE050E069E66A
:100E400076E0CE0189599F4F0E948FBB9E012B599E
:100E50003F4F44E050E062E271E1CE0189599F4F7B
:100E60000E948FBB9E012B593F4F44E050E0BE01D2
:100E7000695A7F4FCE0189599F4F0E948FBB01E075
:100E80009E012B593F4F41E050E0BE0161597F4F19
:100E9000CE0189599F4F0E948FBB9E012B593F4F16
:100EA00041E050E0BE0162597F4FCE0189599F4F0A
:100EB0000E948FBB11118AC06B968CAD9DADAEADFB
:100EC000BFAD6B978093B1109093B210A093B31005
:100ED000B093B4107BC0E1968FADE19790E002969D
:100EE0002EE236E0E4963FAF2EAFE497B501DE0187
:100EF0001196EEE58E2EE1E19E2EAE014F5E5F4F24
:100F0000FEE3AF2EF1E1BF2EE896FFAEEEAEE8971E
:100F10007E0131E2E30EF11C20E030E082179307FE
:100F20002CF0E896EEADFFADE89701C0F7014080E8
:100F3000518062807380F501419251926192719269
:100F40005F018217930714F0F60101C0FA01408097
:100F5000518062807380F40141925192619271924A
:100F60004F018217930734F0FB014080518062806B
:100F7000738005C04D905D906D907C901397E496C2
:100F8000EEADFFADE4974192519261927192E49679
:100F9000FFAFEEAFE4972F5F3F4F6C5F7F4F14962C
:100FA000F4E0CF0ED11C4C5F5F4FE896EEADFFAD85
:100FB000E8973496E896FFAFEEAFE897F4E0EF0ECF
:100FC000F11C2430310509F0A9CFDECEE0968FADBB
:100FD000E097853099F4AF968FADAF97853071F477
:100FE00000E09E012B593F4F44E650E065EB70E175
:100FF000CE0189599F4F0E948FBB24C0111102C09E
:101000000E949FAFE0968FADE097AF96CFACAF97C1
:101010008C9D60011124E12CF12CEC14FD0491F065
:1010200000E09E012B593F4F44E050E0BE01695A59
:101030007F4FCE0189599F4F0E948FBB2FEFE21A3D
:10104000F20AEBCF00E09E012B593F4F44E050E005
:10105000BE016D5A7F4FCE0189599F4F0E948FBBB1
:101060001AE0115079F000E09E012B593F4F44E007
:1010700050E0BE01695A7F4FCE0189599F4F0E94AF
:101080008FBBEFCF01E09E012B593F4F41E050E075
:10109000BE0163597F4FCE0189599F4F0E948FBB7C
:1010A0009E012B593F4F41E050E0BE0164597F4FF4
:1010B000CE0189599F4F0E948FBB00E09E012B59A2
:1010C0003F4F44E050E0BE01635C7F4FCE01895941
:1010D0009F4F0E948FBB9E012B593F4F44E050E031
:1010E000BE016F5C7F4FCE0189599F4F0E948FBB1D
:1010F000AE968FADAE97AD96CFACAD978C9D60019F
:101100001124E12CF12C00E09E012B593F4FCE140D
:10111000DF0471F044E050E0BE01695A7F4FCE0118
:1011200089599F4F0E948FBB3FEFE31AF30AEBCF21
:1011300041E050E0BE016F587F4FCE0189599F4F6B
:101140000E948FBB9E012B593F4F41E050E0BE01F2
:1011500065597F4FCE0189599F4F0E948FBB9E01D9
:101160002B593F4F44E050E0BE01695A7F4FCE01FA
:1011700089599F4F0E948FBB9E012B593F4F44E0DE
:1011800050E0BE01695A7F4FCE0189599F4F0E949E
:101190008FBB9E012B593F4F44E050E066E271E166
:1011A000CE0189599F4F0E948FBB9E012B593F4F03
:1011B00044E050E0BE01615B7F4FCE0189599F4FF3
:1011C0000E948FBB9E012B593F4F44E050E0BE016F
:1011D000655B7F4FCE0189599F4F0E948FBB9E0157
:1011E0002B593F4F44E050E0BE01695B7F4FCE0179
:1011F00089599F4F0E948FBB10E000E09E012B5940
:101200003F4F44E050E0BE01695A7F4FCE018959FB
:101210009F4F0E948FBB111110C06B96CCACDDAC00
:10122000EEACFFAC6B9720E030E84BE355E4C70130
:10123000B6010E948DD5811103C054E0F52E33C054
:1012400080915806811108C0C0924A10D0924B106C
:10125000E0924C10F0924D1000E09E012B593F4F50
:1012600044E050E066E470E1CE0189599F4F0E944E
:101270008FBB9E012B593F4F44E050E06EE470E17C
:10128000CE0189599F4F0E948FBB9E012B593F4F22
:1012900044E050E0BE01695A7F4FCE0189599F4F0B
:1012A0000E948FBB12C0FA94FF2079F000E09E01EB
:1012B0002B593F4F44E050E0BE01695A7F4FCE01A9
:1012C00089599F4F0E948FBBEECF1F5F153009F0E9
:1012D00094CF00E09E012B593F4F42E050E0BE0109
:1012E0006D597F4FCE0189599F4F0E948FBB9E0140
:1012F0002B593F4F44E050E0BE01695A7F4FCE0169
:1013000089599F4F0E948FBB6B96CCACDDACEEAC85
:10131000FFAC6B9720E030E84BE355E4C701B60122
:101320000E948DD5882329F180915806811108C02B
:10133000C0924210D0924310E0924410F0924510B7
:1013400000E09E012B593F4F44E050E06EE370E116
:10135000CE0189599F4F0E948FBB9E012B593F4F51
:1013600044E050E06AE370E1CE0189599F4F0E944A
:101370008FBB00E09E012B593F4F42E050E0BE0181
:101380006F597F4FCE0189599F4F0E948FBB9E019D
:101390002B593F4F41E050E0BE016F587F4FCE01C7
:1013A00089599F4F0E948FBB19E0115000E09E01A8
:1013B0002B593F4F112359F044E050E0BE01695AC8
:1013C0007F4FCE0189599F4F0E948FBBEECF41E0E6
:1013D00050E069E171E1CE0189599F4F0E948FBBB6
:1013E000F12C00E09E012B593F4F44E050E0BE013C
:1013F000695A7F4FCE0189599F4F0E948FBB109130
:101400005806111110C0F1100EC06B968CAD9DAD39
:10141000AEADBFAD6B9780931E1190931F11A0933B
:101420002011B0932111F39485E0F812DACF111155
:1014300002C00E949EB64CE0F42EFA94F11003C054
:101440003CE0F32E0FC000E09E012B593F4F42E0DD
:1014500050E0BE01615A7F4FCE0189599F4F0E94D3
:101460008FBBEBCFFA9400E09E012B593F4FFF203A
:1014700059F044E050E0BE016D5B7F4FCE018959C9
:101480009F4F0E948FBBEECF46E050E0BE01635CF1
:101490007F4FCE0189599F4F0E948FBB9E012B59D0
:1014A0003F4F44E050E06EE176E0CE0189599F4F16
:1014B0000E948FBB9E012B593F4F4CE050E0BE0174
:1014C0006F5C7F4FCE0189599F4F0E948FBB2CE1EB
:1014D000F22EFA94F11003C094E0F92E1DC000E042
:1014E0009E012B593F4F44E050E0BE01695A7F4FA7
:1014F000CE0189599F4F0E948FBBEBCF00E09E0128
:101500002B593F4F44E050E0BE01695A7F4FCE0156
:1015100089599F4F0E948FBBFA94F110EFCF8BE057
:10152000F82EFA94FF2079F000E09E012B593F4FEE
:1015300044E050E0BE01695A7F4FCE0189599F4F68
:101540000E948FBBEECFA9968EAD9FADA997845612
:101550009109C7DA80935706882309F1EFE6FEE187
:1015600084917F019FEFE91AF90A882321F00E94F4
:10157000B951F701F5CFA9966EAD7FADA997645625
:10158000710987E59CE10E943AB76BED72E08FE448
:101590009CE10E943AB78AE00E94B95199C0A7968F
:1015A0002EAD3FADA797AB968EAD9FADAB972817ED
:1015B000390709F44BC081E080935706EAE5FEE164
:1015C00084917F012FEFE21AF20A811103C0EFE24A
:1015D000FCE104C00E94B951F701F2CF84917F0170
:1015E0003FEFE31AF30A882321F00E94B951F70173
:1015F000F5CFAB966EAD7FADAB9780E090E04AE063
:101600000E94DB54EAE2FCE184917F019FEFE91A3A
:10161000F90A882321F00E94B951F701F5CFA79666
:101620006EAD7FADA79780E090E04AE00E94DB546A
:10163000EAE1FCE184917F012FEFE21AF20A8823AC
:1016400009F446C00E94B951F701F4CF111142C00C
:10165000EFE6FEE184917F013FEFE31AF30A811187
:1016600003C007ED12E004C00E94B951F701F2CFA8
:10167000F80181918F01882319F00E94B951F8CFA8
:10168000A9966EAD7FADA997645671098DEF9BE168
:101690000E943AB7A7964EAD5FADA79760E070E0A5
:1016A00080EF9BE10E9400B7EDEEFBE184917F01AA
:1016B0002FEFE21AF20A811107C0809157068111BB
:1016C00009C00E944EBC06C00E94B951F701EECF7E
:1016D000112399F3E6968EAD9FADE6970FB6F89479
:1016E0009EBF0FBE8DBF80915806811102C00E941F
:1016F0006CB09091570681E089270FB6F8943EBEF2
:101700000FBE2DBEC958DF4F0FB6F894DEBF0FBE17
:10171000CDBFDF91CF911F910F91FF90EF90DF90A0
:10172000CF90BF90AF909F908F907F906F905F9081
:101730004F903F902F90089581E080935806F2D902
:10174000109258068111EEC90E94DBB481E0089521
:101750008F929F92AF92BF92CF92DF92EF92FF92C1
:101760000F931F93CF93DF93CDB7DEB7CA5AD1093A
:101770000FB6F894DEBF0FBECDBFE9961CAE1DAE0E
:101780001EAE1FAEE9978091FB039091FC03A091E0
:10179000FD03B091FE03ED968CAF9DAFAEAFBFAF32
:1017A000ED97C556DF4F19821882CB59D04084E699
:1017B00090E0C356DF4F99838883CD59D040109273
:1017C00057069E0125563F4F44E050E0BE01675842
:1017D0007F4FCE0183569F4F0E94DBBBC356DF4F26
:1017E00088819981CD59D0400296C356DF4F9983A5
:1017F0008883CD59D040C556DF4F19821882CB5906
:10180000D04081E0CD55DF4F8883C35AD0409E0140
:1018100025563F4F41E050E0BE016D557F4FCE0150
:1018200083569F4F0E94DBBB9E0125563F4F40E1F0
:1018300050E06EE371E1CE0183569F4F0E94DBBB07
:101840009E0125563F4F44E050E06EE376E0CE0126
:1018500083569F4F0E94DBBB9E0125563F4F40E1C0
:1018600050E06EE571E1CE0183569F4F0E94DBBBD5
:101870009E0125563F4F40E150E06EE276E0CE01FA
:1018800083569F4F0E94DBBB9E0125563F4F44E08D
:1018900050E066E276E0CE0183569F4F0E94DBBBAC
:1018A0009E0125563F4F44E050E06AE276E0CE01CB
:1018B00083569F4F0E94DBBB9E0125563F4F44E05D
:1018C00050E062E276E0CE0183569F4F0E94DBBB80
:1018D0009E0125563F4F44E050E066E476E0CE019D
:1018E00083569F4F0E94DBBB9E0125563F4F44E02D
:1018F00050E062E476E0CE0183569F4F0E94DBBB4E
:101900009E0125563F4F40E150E06EE076E0CE016B
:1019100083569F4F0E94DBBB8AE097EDA3EABCE3AE
:10192000E9968CAF9DAFAEAFBFAFE9979E0125564C
:101930003F4F44E050E0BE016B587F4FCE018356CD
:101940009F4F0E94DBBB9E0125563F4F4CE050E06D
:1019500069E676E0CE0183569F4F0E94DBBB809103
:10196000FE179091FF17A0910018B0910118C3586D
:10197000DF4F88839983AA83BB83CD57D0409E01D4
:1019800025563F4F44E050E0BE0163587F4FCE01E3
:1019900083569F4F0E94DBBB85E0CC55DF4F888389
:1019A000C45AD040CB55DF4F8883C55AD0409E01E2
:1019B00025563F4F44E050E061EB70E1CE01835685
:1019C0009F4F0E94DBBB9E0125563F4F41E050E0F8
:1019D000BE016C557F4FCE0183569F4F0E94DBBBEB
:1019E0009E0125563F4F41E050E0BE016B557F4FB1
:1019F000CE0183569F4F0E94DBBB9E0125563F4F71
:101A000044E650E065EB70E1CE0183569F4F0E94A3
:101A1000DBBBCF57DF4F188219821A821B82C15855
:101A2000D0409E0125563F4F44E050E0BE016F5725
:101A30007F4FCE0183569F4F0E94DBBBE9961CAEC1
:101A40001DAE1EAE1FAEE9971AE0115071F09E0157
:101A500025563F4F44E050E0BE016B587F4FCE010A
:101A600083569F4F0E94DBBBF0CF83E0CA55DF4F08
:101A70008883C65AD040C955DF4F8883C75AD040A3
:101A8000CB57DF4F188219821A821B82C558D0406B
:101A9000C757DF4F188219821A821B82C958D0405B
:101AA000E9961CAE1DAE1EAE1FAEE9979E012556EF
:101AB0003F4F41E050E0BE016A557F4FCE01835653
:101AC0009F4F0E94DBBB9E0125563F4F41E050E0F7
:101AD000BE0169557F4FCE0183569F4F0E94DBBBED
:101AE0009E0125563F4F44E050E0BE0167577F4FAF
:101AF000CE0183569F4F0E94DBBB9E0125563F4F70
:101B000044E050E0BE016B577F4FCE0183569F4F9C
:101B10000E94DBBB0AE010E00150110971F09E0148
:101B200025563F4F44E050E0BE016B587F4FCE0139
:101B300083569F4F0E94DBBBEFCFC855DF4F188203
:101B4000C85AD0408FEFC755DF4F8883C95AD0405D
:101B50009E0125563F4F41E050E0BE0168557F4F42
:101B6000CE0183569F4F0E94DBBB9E0125563F4FFF
:101B700041E050E0BE0167557F4FCE0183569F4F35
:101B80000E94DBBBE9961CAE1DAE1EAE1FAEE997F0
:101B90009E0125563F4F44E050E0BE016B587F4FF9
:101BA000CE0183569F4F0E94DBBB9E0125563F4FBF
:101BB00044E050E0BE016B587F4FCE0183569F4FEB
:101BC0000E94DBBB9E0125563F4F44E050E066E299
:101BD00071E1CE0183569F4F0E94DBBB809183024F
:101BE00090918402A0918502B0918602C357DF4F85
:101BF00088839983AA83BB83CD58D0408091870284
:101C000090918802A0918902B0918A02CF56DF4F4D
